:020000040000FA
:04000000A8EF09F06C
:08000800236E060E03D0236EE7
:10001000040E00D00A6E2450205C02E123501F5CC5
:10002000040ED8B0010ED8B4020E0A14D8A4010EE2
:100030001200086A276E286A00960850D8B4008615
:10004000050E076E270E246E100E0CD8030E246EBC
:10005000E80E08D8246A640E05D8246A0A0E02D86D
:10006000275008D0236E2850206E27501F6EE8ECD2
:1000700001F01F501F6E074E0096085003E0075C0A
:10008000D8B008D01F50D8A4009600B603D0300FC7
:10009000D9EF00F0120005C01FF006C020F0010EDD
:1000A000236E246A0F0EEA6E02C0E9FF00002AD810
:1000B000D8A015D0232EFAD7FF0E2426D8B0F6D715
:1000C0001F26D8A02026D8A01200640E236E246A12
:1000D000EDD70F0EEA6E02C0E9FF14D8FEE256D843
:1000E0002D6A080E246E53D80DD8D8B02D3E233279
:1000F000242EF9D730AA2D6A30BA239E48D8D8804A
:1001000023501200120EE9260950EF1202C0E9FF37
:10011000EF1430BC0918FF0F12002B6E0F0EEA6EA1
:10012000E26E0250E96E120FE16E800E0A16080EA2
:100130002C6ED890D8B00A3E12D82B322C2EFAD77B
:10014000000030BA0A300BD800D000D000D0D880E0
:1001500006D80650246E055052EC01F0120030AE65
:100160000BD0EF50091030AC0918EF6EE7500910B2
:10017000D8A00918E76E0BD0EF500910D8A00918C5
:1001800030BC0918EF6E091CE71601D00A8C3050FC
:100190001F0B000F206E2F50050FD8B0202A0AAC7D
:1001A0005FEF01F00A9C1F6E020E43EC02F05FEF5E
:1001B00001F001BA8DEF00F001B202D001B0FCEF06
:1001C00000F0008800A8009800BA03D0008A33D855
:1001D00027E2009444D8C58642D8C95000B407D05D
:1001E00000B804D0C588C5B8FED700B819D8D890D3
:1001F000236E1DD0008800A8009800BC05D0FE0B1F
:100200000A6E008CD89013D000BE06D02B6E008EE4
:1002100014D8D8B005D02B5014D802E200A807D0CB
:10022000C584C5B4FED7009C009E009A00942D8022
:10023000D8A02D9012000DD801D005D80A5000BAD0
:100240000109C96E0AD094869488C580C5B0FED7CE
:100250001200C582C5B2FED71200C7B4FED723680C
:10026000C5501F0B00D0D890D8B41200232EF8D759
:10027000D8801200AA6AA96EA66AA680A850A94AC8
:10028000AA2A1200AA6AA86EA66AA684550EA76EAC
:10029000AA0EA76EA682A6B2FED7A694A94AAA2A3B
:1002A0001200246A236EFF0E2326242200D0D8A039
:1002B0001200030E206EE30E02D8F5D7206AF40F69
:1002C0001F6E201EFE0ED8A003D01F26D8B0FDD76B
:1002D0001F260000203EF9D700001FB000D01FB03D
:1002E00000D01200010F2C6E0A0E236E246A70D803
:1002F0002C2EFDD727501200010F066E0A0E276E16
:10030000286A296A2A6A04D8062EF8D727501200CC
:1003100022502A18800BF46E22AE06D0D880000E30
:100320001F562056215622562AAE06D0D880000EDF
:100330002756285629562A56236A246A256A266A89
:10034000376A386A396A3A6A2A5029102810271001
:1003500023E0200EF36ED8901F3620362136223649
:100360003736383639363A362750375C28503858C1
:10037000295039582A503A5809E32750375E2850F7
:10038000385A2950395A2A503A5AD88023362436B6
:1003900025362636F32EDFD7F4AE06D0D880000EF1
:1003A000235624562556265623C01FF024C020F07D
:1003B00025C021F026C022F037C027F038C028F031
:1003C00039C029F03AC02AF01200206A246A236E4C
:1003D000286A276A100EF36E2034273628362350F9
:1003E000275C2450285805E32350275E2450285AC0
:1003F000D8801F362036F32EEFD71F501200200E64
:100400002B6E376A386A396A3A6AD8901FA00ED0C4
:10041000275037262850D8B0283C38262950D8B045
:10042000293C39262A50D8B02A3C3A263A32393269
:10043000383237322232213220321F322B2EE5D78A
:100440001200236A246A04D020321F322336243655
:10045000FF0FFAE224C020F023501F6E12001F6E1F
:1004600022BE02D81F5012001F1E201E211E221E57
:100470001F2AD8B0202AD8B0212AD8B0222A1200A8
:10048000D89020321F32FF0FFBE21F501200FC0EEB
:10049000DBCFE6FFFD0EDBCFE6FFFE0EDBCFE6FF98
:1004A000FF0EDBCFE6FFDD52DD52DD52DD521200E2
:1004B000FE0EDBCFE6FFFF0EDBCFE6FFDD52DD52A7
:1004C000120014BE15D11352D8B412D13EC02BF075
:1004D0003E8C7E0E135C2C6E7E0E136E1A6A196AA9
:1004E000186A7F0E176EF30E165C040ED8A0050E68
:1004F000155C350ED8A0360E145C03E3B1EC07F0A2
:1005000004D0132AB1EC07F02C0616C01FF015C05A
:1005100020F014C021F013C022F0710E1A6E5F0E8D
:10052000196E550E186E800E176EB3EC07F01FC0D3
:100530001AF020C019F021C018F022C017F0B5EC55
:1005400008F0C60E1A6EF50E196E1F0E186E800E8C
:10055000176EB3EC07F016C023F015C024F014C0DA
:1005600025F013C026F01FC016F020C015F021C0E2
:1005700014F022C013F08A0E1A6E120E196E790E44
:10058000186E7D0E176EB5EC08F0F60E1A6E460E5C
:10059000196E550E186E7E0E176EB3EC07F023C061
:1005A0001AF024C019F025C018F026C017F04DEC41
:1005B00008F016C023F015C024F014C025F013C0B5
:1005C00026F02250136E176E2150146E186E2050B4
:1005D000156E196E1F50166E1A6EB5EC08F016C027
:1005E00031F015C032F014C033F013C034F023C022
:1005F0001AF024C019F025C018F026C017F0B5EC89
:1006000008F01FC01AF020C019F021C018F022C055
:1006100017F0B5EC08F031C01AF032C019F033C051
:1006200018F034C017F017661706B1EC07F01FC0BA
:100630001AF020C019F021C018F022C017F0B3EC56
:1006400007F02C5256E016C031F015C032F014C03D
:1006500033F013C034F02CC016F0000E16BEFF0E9F
:10066000156E146E136E65EC09F016C01FF015C000
:1006700020F014C021F013C022F0830E1A6E800EF9
:10068000196EDE0E186E720E176EB5EC08F031C0E2
:100690001AF032C019F033C018F034C017F0B3ECC0
:1006A00007F016C031F015C032F014C033F013C09B
:1006B00034F01FC016F020C015F021C014F022C085
:1006C00013F01A6A800E196E310E186E7E0E176EB8
:1006D000B5EC08F031C01AF032C019F033C018F090
:1006E00034C017F0B3EC07F02BBC03D03E9C01D014
:1006F0003E8A165012003A6A16C022F015C021F048
:1007000014C020F013501F6E05E014AE03D03A80E1
:10071000800E201A20BE21D0010E225C000E21582E
:10072000000E20587F0E1F5818E3166A156A146AC7
:100730007F0E136E22C01AF021C019F020C018F0ED
:100740001FC017F04DEC08F016C022F015C021F0C4
:1007500014C020F013C01FF03A820A0E166E890EE4
:10076000156E340E146E7C0E136E22C01AF021C06A
:1007700019F020C018F01FC017F0B5EC08F022C027
:100780001AF021C019F020C018F01FC017F0B5EC06
:1007900008F07C0E1A6E790E196E350E186E810EE9
:1007A000176EB3EC07F022C01AF021C019F020C078
:1007B00018F01FC017F0B5EC08F022C01AF021C0E5
:1007C00019F020C018F01FC017F0B5EC08F03F0E6C
:1007D0001A6E020E196E330E186E830E176EB3EC7E
:1007E00007F022C01AF021C019F020C018F01FC075
:1007F00017F0B5EC08F022C01AF021C019F020C0A3
:1008000018F01FC017F0B5EC08F0330E1A6E8C0EFE
:10081000196E1E0E186E830E176EB3EC07F016C01D
:1008200026F015C025F014C024F013C023F0225088
:10083000166E2150156E2050146E1F50136E22C07C
:100840001AF021C019F020C018F01FC017F0B5EC45
:1008500008F01B0E1A6EE40E196E350E186E820E1D
:10086000176EB3EC07F022C01AF021C019F020C0B7
:1008700018F01FC017F0B5EC08F022C01AF021C024
:1008800019F020C018F01FC017F0B5EC08F0A40E46
:100890001A6EDB0E196E670E186E830E176EB3ECB0
:1008A00007F022C01AF021C019F020C018F01FC0B4
:1008B00017F0B5EC08F022C01AF021C019F020C0E2
:1008C00018F01FC017F0B5EC08F0330E1A6E8C0E3E
:1008D000196E1E0E186E830E176EB3EC07F016C05D
:1008E0002AF015C029F014C028F013C027F022C048
:1008F00016F021C015F020C014F01FC013F026C060
:100900001AF025C019F024C018F023C017F0B5EC78
:1009100008F02AC01AF029C019F028C018F027C022
:1009200017F04DEC08F016C01AF015C019F014C0FD
:1009300018F013C017F03AA20AD0DB0E166E0F0E95
:10094000156E490E146E7F0E136EB1EC07F03AA0CF
:1009500002D0800E141A1650120016C032F015C0C4
:1009600033F014C034F013C031F01BD816C01CF0A3
:1009700015C01DF014C01EF013C01BF032C016F0DD
:1009800033C015F034C014F031C013F00CD81CC0C3
:100990001AF01DC019F01EC018F01BC017F04DEF63
:1009A00008F0010E01D0000E276E3EC029F03E8CEB
:1009B0002A6A276602D014BE2A8E149E880E1360FF
:1009C0003E8A16C01FF015C020F014C021F013C0DD
:1009D00022F0830E1A6EF90E196E220E186E7F0E1B
:1009E000176EB5EC08F03E9C05EC09F03E8C16A0A5
:1009F00004D0162A000E15221422070E1614286E93
:100A0000030E286404D0800E2A1A040E285E136A8E
:100A100065EC09F01350266E6DE016C023F015C08A
:100A200024F014C025F01A6A0F0E196EC90E186E44
:100A30007E0E176EB5EC08F01FC01AF020C019F03A
:100A400021C018F022C017F0B3EC07F016C01FF059
:100A500015C020F014C021F013C022F023C016F0FE
:100A600024C015F025C014F026C013F01A6AA20E97
:100A7000196EDA0E186E6E0E176EB5EC08F01FC008
:100A80001AF020C019F021C018F022C017F0B3EC02
:100A900007F016C01FF015C020F014C021F013C0DD
:100AA00022F023C016F024C015F025C014F026C093
:100AB00013F0200E1A6EA20E196E850E186E5C0EC3
:100AC000176EB5EC08F01FC01AF020C019F021C055
:100AD00018F022C017F0B3EC07F01350226E176E17
:100AE0001450216E186E1550206E196E16501F6E20
:100AF0001A6E0CD02250136E176E2150146E186EA1
:100B00002050156E196E1F50166E1A6EB5EC08F057
:100B100016C023F015C024F014C025F013C026F031
:100B200028302818010B271851E0CE0E1A6EF50E4A
:100B3000196E4C0E186E6F0E176EB5EC08F01A0E8B
:100B40001A6E060E196EB60E186E750E176EB3EC91
:100B500007F023C01AF024C019F025C018F026C0F1
:100B600017F0B5EC08F0A50E1A6EAA0E196E2A0E33
:100B7000186E7A0E176EB3EC07F023C01AF024C07B
:100B800019F025C018F026C017F0B5EC08F023C006
:100B90001AF024C019F025C018F026C017F0B5ECE3
:100BA00008F023C01AF024C019F025C018F026C0A0
:100BB00017F017661706B1EC07F03E9C1A6A196A1F
:100BC000186A7F0E176EB3EC07F05AD0F90E1A6E42
:100BD000680E196E360E186E6C0E176EB5EC08F0B6
:100BE000C00E1A6E070E196ED00E186E720E176EAA
:100BF000B3EC07F023C01AF024C019F025C018F098
:100C000026C017F0B5EC08F0840E1A6E880E196E27
:100C1000080E186E780E176EB3EC07F023C01AF0AA
:100C200024C019F025C018F026C017F0B5EC08F064
:100C3000AB0E1A6EAA0E196E186E7C0E176EB3EC00
:100C400007F023C01AF024C019F025C018F026C000
:100C500017F0B5EC08F01FC01AF020C019F021C041
:100C600018F022C017F0B5EC08F03E9C1FC01AF037
:100C700020C019F021C018F022C017F0B3EC07F023
:100C8000800E275202E028B22A1A2ABE141A29BC62
:100C90003E8C1650120014BEB1D01352D8B4AFD04F
:100CA00013C028F03EC029F03E8C7F0E136E1A6AE6
:100CB000196A186A176EB1EC07F016C01FF015C05C
:100CC00020F014C021F013C022F0130E1A6ECB0EC8
:100CD000196E030E186E840E176EB3EC07F01FC06A
:100CE0001AF020C019F021C018F022C017F0B5EC9E
:100CF00008F0BC0E1A6E5A0E196E050E186E860E8E
:100D0000176EB3EC07F01FC01AF020C019F021C015
:100D100018F022C017F0B5EC08F0830E1A6E300EF2
:100D2000196E720E186E850E176EB3EC07F016C0B2
:100D300023F015C024F014C025F013C026F01FC006
:100D400016F020C015F021C014F022C013F08E0E52
:100D50001A6ED70E196E6B0E186E810E176EB5ECEB
:100D600008F0B50E1A6E290E196E4E0E186E840E0E
:100D7000176EB3EC07F01FC01AF020C019F021C0A5
:100D800018F022C017F0B5EC08F0800E1A6E300E85
:100D9000196E720E186E840E176EB3EC07F023C036
:100DA0001AF024C019F025C018F026C017F04DEC39
:100DB00008F01FC01AF020C019F021C018F022C09E
:100DC00017F0B5EC08F01A6A196A186A7F0E176EE8
:100DD000B3EC07F028B00AD0F30E1A6E040E196EA9
:100DE000350E186E7F0E176EB5EC08F07F0E2826B4
:100DF0002830136E29BC03D03E9C01D03E8A165089
:100E0000120018501418406E40BE30D018BE17D0D3
:100E10001750135CD8A0000CD8A4010C1850145C17
:100E2000D8A0000CD8A4010C1950155CD8A0000C57
:100E3000D8A4010C1A50165CD8A0000C010C135059
:100E4000175CD8A0000CD8A4010C1450185CD8A0D2
:100E5000000CD8A4010C1550195CD8A0000CD8A423
:100E6000010C16501A5CD8A0000C010C14AE010C39
:100E7000000C18501418406E40BE34D018BE19D063
:100E80001750135CD8A0000CD8A4010C1850145CA7
:100E9000D8A0000CD8A4010C1950155CD8A0000CE7
:100EA000D8A4010C1A50165CD8A0000CD8A4010CD0
:100EB000000C1350175CD8A0000CD8A4010C1450DF
:100EC000185CD8A0000CD8A4010C1550195CD8A04F
:100ED000000CD8A4010C16501A5CD8A0000CD8A4A1
:100EE000010C000C14AE010C000C14501818406ECC
:100EF00040BE34D014BE19D01350175CD8A0000CDB
:100F0000D8A4010C1450185CD8A0000CD8A4010C73
:100F10001550195CD8A0000CD8A4010C16501A5C0E
:100F2000D8A0000CD8A4010C000C1750135CD8A05A
:100F3000000CD8A4010C1850145CD8A0000CD8A444
:100F4000010C1950155CD8A0000CD8A4010C1A5043
:100F5000165CD8A0000CD8A4010C000C18AE010C33
:100F6000000C800E181A1750135C3D6E19E23D6C90
:100F700013C03FF017C013F03FC017F014C03FF08C
:100F800018C014F03FC018F015C03FF019C015F09C
:100F90003FC019F016C03FF01AC016F03FC01AF05B
:100FA0001A0E3D6078D0175276E03C6A14503F6EBE
:100FB0001818416E148E188E080E3D5E08E31AC094
:100FC0003CF019C01AF018C019F0186AF5D73D2680
:100FD00007E0D890183219321A323C323D2EF9D738
:100FE00041AE35D01A50165E1950155A1850145A81
:100FF00007E2D880000E165615561456800E3F1A7A
:101000003C6C04E01606000E155A145A040E3D6E90
:1010100014660DD015C014F016C015F03CC016F0C3
:101020003C6A080E135E2DE33D2EF2D72AD014BE83
:1010300008D0D8903C36163615361436132EF7D70E
:1010400020D03EAC26D03CAE24D03C6A11D01A5001
:101050001626195015221850142206E314321532A0
:1010600016323C32134A0FD03EAC13D03CAE11D0F6
:10107000163E0FD0153E0DD0143E0BD0D8801690E2
:10108000EDD7136A02D03E821368166A156A800E85
:10109000146E3FAE149E165012001450396E18187C
:1010A000416E175053E0135254E0135E7F0E03E27B
:1010B000132603E24DD013264EE216C037F015C0BA
:1010C00038F0398E188E180E3F6E166A156A146A3B
:1010D0000BD01A50375C1950385811E3386E396A02
:1010E0001A50375E0BD004E21850395CF2E007E387
:1010F0001A50375E1950385A1850395AD880163657
:10110000153614363736383639363F2EECD714BEFE
:1011100007D013521DE0413213063F2A4136E3D770
:101120003EAC1FD007E21A50375E1950385A18509B
:10113000395A17E3163E15D0153E13D0143E11D080
:10114000143215321632133E0CD005D03E8604D030
:101150003E84136A02D03E821368166A156A800EB6
:10116000146E41AE149E165012001450396E1818A9
:10117000416E1350D8A417503CE013267E0E03E3B3
:10118000135E03E338D0135E33E316C037F015C0A7
:1011900038F0398E188E166A156A146A180E3F6E6A
:1011A00039323832373206E31A50162619501522D2
:1011B000185014221432153216323F2EF1D714BEB5
:1011C00007D0163615361436135212E0130639348A
:1011D0003EAC17D016E3163E14D0153E12D0143E86
:1011E00010D0D880143215321632133E0AD003D0F4
:1011F0003E84136A02D03E821368166A156A800E16
:10120000146E41AE149E1650120014C041F07F0EB1
:10121000135C3F6E3FE3148E136A376A17083F6E04
:101220000BE2080E3F2638E314C013F015C014F08B
:1012300016C015F0166A0CD0080E3F5E08E316C003
:1012400037F015C016F014C015F0146AF5D73F2614
:101250003F5208E0D890133214321532163237322A
:101260003F2EF8D713BE18D03EAC0BD037AE09D006
:10127000163E07D0153E05D0143E03D0142A13BEE7
:101280000BD041AE10D0D880000E1656155614560D
:10129000135609D0000E02D03E82FF0E136E146E5C
:1012A000156E166E139E16501200136E146A156A90
:1012B000166A13C03CF016C013F03CC016F015C0FF
:1012C0003CF014C015F03CC014F0960E3F6E416A1D
:1012D00013AE07D0D880000E165615561456135666
:1012E000418E135218E03EAC0DD016AE0BD0153E19
:1012F00009D0143E07D0133E05D0D88013321432E3
:1013000015323F2A080E3F2615C016F014C015F0FE
:1013100013C014F015D0146613D0080E3F5E15509C
:1013200005E1080E3F5E165011E0166A146E16C0F5
:1013300015F0166A05D0D8901636153614363F06C5
:1013400014AEF9D73FC013F041AE149E16501200F0
:10135000F86A400E3E6E006AAB6A280EC66E040E36
:10136000C86E800EC76E070EB46E0F0EC16E2EEEE5
:10137000C0F0860ED56E0EEEFFF0ED6AE950EA1071
:10138000FCE1EF6A2F0E926E070E936E870E946E3D
:10139000956A966A3F0E976E200E986E836B826BED
:1013A000916B010E936F900E926F946B0A0E896F82
:1013B0008B6B8C6B88958D6B0601376B0001889168
:1013C000B36BB26BB56BB46B889B010EB66F010E3D
:1013D000B76FC86B0B0E8A6F88998897CB6BCC6BF5
:1013E000D06BD66BD56BD46BD36B0101216B010E27
:1013F00008011C6F0101276B266B296B286B050107
:10140000216B206B1F6B1E6B256B246B236B226B78
:10141000296B286B276B266B2D6B2C6B2B6B2A6B28
:101420002F6B2E6B336B326B316B306B08011B6B88
:101430001A6B196B186B790E0501346F366B356BAF
:1014400001012D6B2C6B2B6B2A6BA30E476FA20E29
:10145000486FAB0E496FAA0E4A6F0001846B800E75
:10146000845DD8B040EF0AF002EE1AF0D8908435CF
:10147000E926000EEA22EE6AEF6A842BD8A4EFD7A1
:10148000846B800E845DD8B052EF0AF003EE1AF040
:10149000D8908435E926000EEA22EE6AEF6A842BA2
:1014A000D8A4EFD7846B800E845DD8B064EF0AF0C7
:1014B00004EE1AF0D8908435E926000EEA22EE6A8E
:1014C000EF6A842BD8A4EFD7846B150E845DD8B057
:1014D00076EF0AF001EE74F0D8908435E926000E1C
:1014E000EA22EE6AEF6A842BD8A4EFD7846B290E28
:1014F000845DD8B088EF0AF001EE9EF0D890843574
:10150000E926000EEA22EE6AEF6A842BD8A4EFD710
:10151000846B150E845DD8B09AEF0AF001EEF0F0FE
:10152000D8908435E926000EEA22EE6AEF6A842B11
:10153000D8A4EFD7C9EFC3F008016B6B0001835348
:10154000D8A483EF0BF001013493020E225D000159
:10155000D8A4B0EF0AF0010134830001BFEF0AF014
:10156000030E0101225D0001D8A4BCEF0AF00101C5
:1015700034830001BEEF0AF0010134930001D896D4
:10158000010134A3D8860001D8B64DEF0BF0080155
:101590006B2B0A0E6B5D0001D8A4D1EF0AF0ADEF02
:1015A00097F0850E026E800E096E306ABC0E2F6EAB
:1015B000066A056A200E016E240E8DEC00F0500EB6
:1015C0008DEC00F0530E8DEC00F0520E8DEC00F01F
:1015D000460E8DEC00F0310E8DEC00F0300E8DECEF
:1015E00000F0330E8DEC00F02C0E8DEC00F0340E7C
:1015F0008DEC00F02C0E8DEC00F0310E8DEC00F037
:101600002C0E8DEC00F0310E8DEC00F02C0E8DECDC
:1016100000F0310E8DEC00F02A0E8DEC00F0320E51
:101620008DEC00F0300E8DEC00F00D0E8DEC00F026
:101630000A0E8DEC00F0800E026E040E096E400E54
:10164000306EBC0E2F6E070E066ED00E056E4BEC84
:1016500000F0D8A09CD75208D8A4F9D74BEC00F0E2
:10166000D8A095D74D08D8A4F2D74BEC00F0D8A05D
:101670008ED74308D8A4EBD70B6AD8804BEC00F088
:10168000D8A085D708EE24F00B5023C0EBFF0B2A1F
:101690000B504008F2E181EF0BF0800E026E040E59
:1016A000096E400E306EBC0E2F6E070E066ED00E09
:1016B000056E4BEC00F0D8A0ADEF97F05208D8A41F
:1016C000F8D74BEC00F0D8A0ADEF97F04D08D8A4B8
:1016D000F0D74BEC00F0D8A0ADEF97F04308D8A4BA
:1016E000E8D70B6AD8804BEC00F0D8A0ADEF97F0AC
:1016F00008EE24F00B5023C0EBFF0B2A0B504008E0
:10170000F1E19CEF0CF0470E0801246F500E256F9D
:10171000520E266F4D0E276F430E286F2C0E296F29
:10172000300E2A6F310E2B6F310E2C6F340E2D6F51
:10173000330E2E6F370E2F6F2E0E306F300E316F2F
:10174000300E326F300E336F2C0E346F410E356F0A
:101750002C0E366F340E376F320E386F340E396FF1
:10176000340E3A6F2E0E3B6F300E3C6F300E3D6FD5
:10177000300E3E6F300E3F6F2C0E406F4E0E416F9D
:101780002C0E426F300E436F380E446F330E456F90
:10179000300E466F300E476F2E0E486F300E496F79
:1017A000300E4A6F300E4B6F300E4C6F2C0E4D6F5B
:1017B000570E4E6F2C0E4F6F696B06EE38F0D890B7
:1017C00006013735E926000EEA22EECF1FF0EFCFF3
:1017D00020F0030E72EC01F00801696F69C850F83F
:1017E000696B06EE38F0D89006013735E926000E11
:1017F000EA22EECF1FF0EFCF20F0020E72EC01F0E4
:101800000801696F69C851F82E0E526F696B06EEB8
:1018100038F0D89006013735E926000EEA22EECFDF
:101820001FF0EFCF20F0010E72EC01F00801696F9C
:1018300069C853F8696B06EE38F0D8900601373561
:10184000E926000EEA22EECF1FF0EFCF20F0000EC7
:1018500072EC01F00801696F69C854F82C0E556FDD
:10186000696B07EE28F0D89006013735E926000E9F
:10187000EA22EECF1FF0EFCF20F0020E72EC01F063
:101880000801696F69C856F8696B07EE28F0D890AF
:1018900006013735E926000EEA22EECF1FF0EFCF22
:1018A00020F0010E72EC01F00801696F69C857F869
:1018B000696B07EE28F0D89006013735E926000E4F
:1018C000EA22EECF1FF0EFCF20F0000E72EC01F015
:1018D0000801696F69C858F82E0E596F380E5A6F93
:1018E000350E5B6F2C0E5C6F320E5D6F300E5E6FCF
:1018F000300E5F6F380E606F300E616F380E626FA2
:101900002C0E636F2C0E646F2A0E656F310E666F9E
:10191000360E676F360E686F0601372B780E375D0F
:101920000001D8A096EF0CF00601376B0001010E04
:10193000246E900E52EC01F00801236B0001400E62
:101940000801235D0001D8B0DFEF0CF008EE24F0B1
:1019500008012351EBCF0BF000EE42F023510BC0F6
:10196000EBFF08EE24F02351EB500F6E960EF66E4F
:10197000190EF76E2368232A235009080001D8A006
:10198000D5EF0CF00900F55009000F5CF4E123C01D
:101990000BF0D5EF0CF0300C310C320C330C340C56
:1019A000350C360C370C380C390C00EE42F00801BF
:1019B00023510BC0EBFF232B0001D8A4BFD712008B
:1019C00008016C6B00010A0E08016C5D0001D8B0C3
:1019D0003AEF0DF00101215108016C5D0001D8B012
:1019E00015EF0DF008016C510101215D316E326A75
:1019F000D8A03206310404EE1AF0D890E836E92671
:101A0000000EEA22EECF0BF0EFCF0CF008EE6FF0F5
:101A1000D89008016C35E926000EEA220BC0EEFFD3
:101A20000CC0EFFF000134EF0DF07F0E0101212506
:101A3000326A316E323608016C51315C04EE1AF0B4
:101A4000D890E836E926000EEA22EECF0BF0EFCF71
:101A50000CF008EE6FF0D8906C35E926000EEA2203
:101A60000BC0EEFF0CC0EFFF000108016C2B000162
:101A7000D8A4A8D708016C6B00010A0E08016C5DA0
:101A80000001D8B0DBEF0DF004EE1AF0D8900101A0
:101A90002135E926000EEA22EECF1FF0EFCF20F02D
:101AA000020E72EC01F00B6E030E0B5C0001D8A469
:101AB0008DEF0DF008EE6FF0D89008016C35E92637
:101AC000000EEA22EECF1FF0EFCF20F0020E72ECF4
:101AD00001F00B6E0B520001D8A48CEF0DF008EE54
:101AE0006FF0D89008016C35E926000EEA22EECF9F
:101AF0000FF0EFCF10F0680E0F240B6E010E1020C8
:101B00000C6E08EE6FF0D8906C35E926000EEA22D4
:101B10000BC0EEFF0CC0EFFF000104EE1AF0D890EE
:101B200001012135E926000EEA22EECF1FF0EFCFAA
:101B300020F0020E72EC01F00B6E0B520001D8A4E3
:101B4000D6EF0DF008EE6FF0D89008016C35E9265D
:101B5000000EEA22EECF1FF0EFCF20F0020E72EC63
:101B600001F00B6E030E0B5C0001D8A4D5EF0DF055
:101B700008EE6FF0D89008016C35E926000EEA22D5
:101B8000EECF0FF0EFCF10F00F5068080B6E010E84
:101B900010540C6E08EE6FF0D8906C35E926000EEC
:101BA000EA220BC0EEFF0CC0EFFF000108016C2B16
:101BB0000001D8A461D708016E6B6D6B6C6B0001DE
:101BC0000A0E08016C5D0001D8B0FBEF0DF008EEC5
:101BD0006FF0D89008016C35E926000EEA22EECFAE
:101BE0000BF0EFCF0CF00B506D270C506E236C2BCD
:101BF0000001D8A4E4D76EC820F06DC81FF0246A95
:101C00000A0E236EE8EC01F008016D6F20C06EF83B
:101C100004EE1AF0D89001012135E926000EEA22DF
:101C2000EECF0BF0EFCF0CF00B5008016D5D0C50B8
:101C30006E590001D8B033EF0EF004EE1AF0D890D0
:101C400001012135E926000EEA22EECF0BF0EFCF9D
:101C50000CF008016D510B5C836F6E510C58846F52
:101C6000000146EF0EF004EE1AF0D8900101213584
:101C7000E926000EEA22EECF0BF0EFCF0CF00B506E
:101C800008016D5D836F0C506E59846F000108016F
:101C900084530001D8A463EF0EF0030E0801835DA6
:101CA0000001D8B063EF0EF004EE1AF0D8900101F5
:101CB0002135E926000EEA22EECF6DF8EFCF6EF85F
:101CC000000168EF0EF0010E08016E6F680E6D6F77
:101CD00000016DC8DEFF6EC8DEFF120018EE87F04F
:101CE00058EC02F018EE85F058EC02F0080185512E
:101CF000875D865188590001D8B08FEF0EF008013A
:101D00008751855D896F885186598A6F8951680826
:101D1000896F010E8A558A6F000196EF0EF0080157
:101D20008551875D896F865188598A6F0001080146
:101D30008A51010A680ED8B489190001D8A4A6EF07
:101D40000EF0010E08018A6F670E896F000189C8C5
:101D5000DEFF8AC8DEFF1200FF0EDB50DD520101FC
:101D60003485E8A0349518EE8DF058EC02F018EEAA
:101D70008BF058EC02F008018B518D5D8C518E591F
:101D80000001D8B0D4EF0EF008018D518B5D8F6F3C
:101D90008E518C59906F8F516808916F010E90553C
:101DA000926F0001E1EF0EF008018B518D5D8F6F96
:101DB0008C518E59906F8F516808916F010E90551C
:101DC000926F0001080191518F5D9251905900016D
:101DD000D8B0F1EF0EF090C894F88FC893F8F5EFF3
:101DE0000EF092C894F891C893F8D896010134A5E2
:101DF000D8860001D8B626EF0FF008018B518D5D13
:101E00008C518E590001D8B017EF0FF00801915195
:101E10008F5D925190590001D8B013EF0FF0520E20
:101E2000856F15EF0FF04C0E856F26EF0FF0080150
:101E300091518F5D925190590001D8B024EF0FF06D
:101E40004C0E856F26EF0FF0520E856F08019451EE
:101E5000010A680ED8B493190001D8A435EF0FF029
:101E6000010E0801946F670E936F000193C8DEFFA7
:101E700094C8DEFF120018EEA1F058EC02F004EE58
:101E80001AF0D89001012135E926000EEA22EECFA2
:101E90000BF0EFCF0CF00BC0DEFF0CC0DEFFA1C8D3
:101EA000DEFFA2C8DEFFDE6A000156DF18EE95F005
:101EB00058EC02F095C813F096C814F057EC09F0EE
:101EC000DB0E1A6E0F0E196E490E186E800E176E0D
:101ED000B5EC08F016C0A0F815C09FF814C09EF825
:101EE00013C09DF81A6A196A340E186E860E176EA2
:101EF000A0C816F09FC815F09EC814F09DC813F036
:101F00004DEC08F016C0A0F815C09FF814C09EF85C
:101F100013C09DF8A0C816F09FC815F09EC814F015
:101F20009DC813F0D1EC04F016C09CF815C09BF8C6
:101F300014C09AF813C099F808019A9F03EE1AF09A
:101F4000D89001012135E926000EEA22EECF0BF0F0
:101F5000EFCF0CF00BC013F00CC014F057EC09F0ED
:101F60009CC81AF09BC819F09AC818F099C817F0C5
:101F7000B5EC08F005EC09F015C098F80801976F6A
:101F800097C8DEFF98C8DEFF00011200D89688AD22
:101F9000D886D8B6D1EF0FF00801AC6BAB6B00015F
:101FA000889D04EE1AF0D89001012135E926000E33
:101FB000EA22EECFA3F8EFCFA4F8A4C820F0A3C87C
:101FC0001FF0020E72EC01F00801A66BA56F010173
:101FD00021530001D8B4FEEF0FF0010121050B6E73
:101FE00004EE1AF0D8900B34E926000EEA22EECF68
:101FF000A7F8EFCFA8F8000102EF10F018C5A7F876
:1020000019C5A8F8A8C820F0A7C81FF0020E72ECE6
:1020100001F00801AA6BA96FA951A55D0B6EAA5129
:10202000A6590C6E0B50030A0C100001D8A420EF27
:1020300010F00801A7516808A76F010EA855A86FF6
:1020400000010801A551A95D0B6EA651AA590C6E9D
:102050000B50030A0C100001D8A434EF10F0680EE6
:102060000801A327010EA42300010801A351A75DC5
:10207000A451A8590001D8B059EF10F00801AB2BBA
:10208000040EAC5D0001D8A056EF10F0888104EE7C
:102090001AF0D89001012135E926000EEA22EECF90
:1020A00086F0EFCF87F0000158EF10F00801AC6B1D
:1020B00000010801A751A35DA851A4590001D8B09F
:1020C0007DEF10F00801AC2B040EAB5D0001D8A031
:1020D0007AEF10F0888104EE1AF0D89001012135D2
:1020E000E926000EEA22EECF86F0EFCF87F000015E
:1020F0007CEF10F00801AB6B00011200A1C0B1F839
:10210000A0C0B0F89FC0AFF89EC0AEF8A5C0B5F8AB
:10211000A4C0B4F8A3C0B3F8A2C0B2F8A9C0B9F87B
:10212000A8C0B8F8A7C0B7F8A6C0B6F8ADC0BDF84B
:10213000ACC0BCF8ABC0BBF8AAC0BAF81A6A7C0E37
:10214000196E120E186E920E176E96C013F097C08D
:1021500014F098C015F099C016F059EC09F04DEC48
:1021600008F016C0C1F815C0C0F814C0BFF813C0FD
:10217000BEF8CC5155EC09F0C1C81AF0C0C819F02E
:10218000BFC818F0BEC817F0B3EC07F016C0C1F80E
:1021900015C0C0F814C0BFF813C0BEF8530E01013B
:1021A0005A5D0001D8A4D8EF10F0800E0801BF1BC3
:1021B00000011A6A7C0E196E120E186E920E176EBE
:1021C0009AC013F09BC014F09CC015F09DC016F08F
:1021D00059EC09F04DEC08F016C0C5F815C0C4F86C
:1021E00014C0C3F813C0C2F8CD5155EC09F0C5C8EE
:1021F0001AF0C4C819F0C3C818F0C2C817F0B3EC7D
:1022000007F016C0C5F815C0C4F814C0C3F813C051
:10221000C2F8570E0101645D0001D8A413EF11F05C
:10222000800E0801C31B0001CC5155EC09F0DB0EF8
:102230001A6E0F0E196E490E186E800E176EB5ECE1
:1022400008F016C034F015C033F014C032F013C0DB
:1022500031F01A6A196A340E186E860E176E34C081
:1022600016F033C015F032C014F031C013F04DEC4D
:1022700008F016C013F915C012F914C011F913C0F3
:1022800010F913C916F012C915F011C914F010C9CC
:1022900013F0D1EC04F016C013F915C012F914C0F4
:1022A00011F913C010F9BDC816F0BCC815F0BBC8B1
:1022B00014F0BAC813F0B5C81AF0B4C819F0B3C80E
:1022C00018F0B2C817F0B1EC07F016C034F015C022
:1022D00033F014C032F013C031F034C016F033C004
:1022E00015F032C014F031C013F013C91AF012C93E
:1022F00019F011C918F010C917F0B5EC08F016C0A4
:10230000E1F815C0E0F814C0DFF813C0DEF8B9C872
:1023100016F0B8C815F0B7C814F0B6C813F0B1C8B5
:102320001AF0B0C819F0AFC818F0AEC817F0B1EC89
:1023300007F016C0E5F815C0E4F814C0E3F813C0C0
:10234000E2F8C5C816F0C4C815F0C3C814F0C2C876
:1023500013F0B5C81AF0B4C819F0B3C818F0B2C871
:1023600017F0B1EC07F016C034F015C033F014C00C
:1023700032F013C031F034C016F033C015F032C063
:1023800014F031C013F013C91AF012C919F011C9B1
:1023900018F010C917F0B5EC08F016C0EDF815C02C
:1023A000ECF814C0EBF813C0EAF8C1C816F0C0C8C6
:1023B00015F0BFC814F0BEC813F0B1C81AF0B0C809
:1023C00019F0AFC818F0AEC817F0B1EC07F016C09E
:1023D000E9F815C0E8F814C0E7F813C0E6F8B1C88A
:1023E00016F0B0C815F0AFC814F0AEC813F0C1C8ED
:1023F0001AF0C0C819F0BFC818F0BEC817F0B1EC89
:1024000007F016C0F9F815C0F8F814C0F7F813C0B3
:10241000F6F8B5C816F0B4C815F0B3C814F0B2C8D1
:1024200013F0C5C81AF0C4C819F0C3C818F0C2C860
:1024300017F0B1EC07F016C034F015C033F014C03B
:1024400032F013C031F034C016F033C015F032C092
:1024500014F031C013F013C91AF012C919F011C9E0
:1024600018F010C917F0B5EC08F016C0FFF815C049
:10247000FEF814C0FDF813C0FCF8E9C8C9F8E8C8B4
:10248000C8F8E7C8C7F80801C79FE6C8C6F8FFC87C
:10249000CDF8FEC8CCF8FDC8CBF8CB9FFCC8CAF875
:1024A000CDC816F0CCC815F0CBC814F0CAC813F0CC
:1024B000C9C81AF0C8C819F0C7C818F0C6C817F0BC
:1024C00001EC07F001080001D8B471EF12F0C9C89F
:1024D00017F9C8C816F9C7C815F9C6C814F979EFAD
:1024E00012F0CDC817F9CCC816F9CBC815F9CAC86F
:1024F00014F90A0E166ED70E156E230E146E780E92
:10250000136E17C91AF016C919F015C918F014C9B5
:1025100017F001EC07F00108D8B49AEF12F00901A6
:102520000F6B010E0E6F860E0D6F3C0E0C6F0001CF
:1025300084EF15F0EDC816F0ECC815F0EBC814F0F8
:10254000EAC813F0E1C81AF0E0C819F0DFC818F0C3
:10255000DEC817F0B5EC08F016C0C9F815C0C8F809
:1025600014C0C7F813C0C6F8E9C816F0E8C815F0DB
:10257000E7C814F0E6C813F0E5C81AF0E4C819F08B
:10258000E3C818F0E2C817F0B5EC08F016C0CDF8B3
:1025900015C0CCF814C0CBF813C0CAF8C9C816F0DF
:1025A000C8C815F0C7C814F0C6C813F0CDC81AF0D3
:1025B000CCC819F0CBC818F0CAC817F0B3EC07F0B4
:1025C00016C0D5F815C0D4F814C0D3F813C0D2F88B
:1025D000E1C816F0E0C815F0DFC814F0DEC813F04B
:1025E000E1C81AF0E0C819F0DFC818F0DEC817F02B
:1025F000B5EC08F016C0C9F815C0C8F814C0C7F883
:1026000013C0C6F8E5C816F0E4C815F0E3C814F026
:10261000E2C813F0E5C81AF0E4C819F0E3C818F0EE
:10262000E2C817F0B5EC08F016C0CDF815C0CCF82C
:1026300014C0CBF813C0CAF8C9C816F0C8C815F042
:10264000C7C814F0C6C813F0CDC81AF0CCC819F02A
:10265000CBC818F0CAC817F0B3EC07F016C0D1F811
:1026600015C0D0F814C0CFF813C0CEF8D5C816F0F6
:10267000D4C815F0D3C814F0D2C813F0D1C81AF0DA
:10268000D0C819F0CFC818F0CEC817F04DEC08F03C
:1026900016C0D9F815C0D8F814C0D7F813C0D6F8AA
:1026A000E1C816F0E0C815F0DFC814F0DEC813F07A
:1026B000F9C81AF0F8C819F0F7C818F0F6C817F0FA
:1026C000B5EC08F016C0C9F815C0C8F814C0C7F8B2
:1026D00013C0C6F8E5C816F0E4C815F0E3C814F056
:1026E000E2C813F0FFC81AF0FEC819F0FDC818F0D0
:1026F000FCC817F0B5EC08F016C0CDF815C0CCF842
:1027000014C0CBF813C0CAF8C9C816F0C8C815F071
:10271000C7C814F0C6C813F0CDC81AF0CCC819F059
:10272000CBC818F0CAC817F0B1EC07F016C0DDF836
:1027300015C0DCF814C0DBF813C0DAF8DDC816F0F9
:10274000DCC815F0DBC814F0DAC813F0D1C81AF0F1
:10275000D0C819F0CFC818F0CEC817F04DEC08F06B
:1027600016C0DDF815C0DCF814C0DBF813C0DAF8C9
:10277000D9C816F0D8C815F0D7C814F0D6C813F0C9
:102780001A6A196A186A176A01EC07F03B6ED9C811
:1027900016F0D8C815F0D7C814F0D6C813F01A6AC6
:1027A000196A186A7F0E176E39EC07F0010A3B149C
:1027B000D8B414EF14F0D1C816F0D0C815F0CFC8B3
:1027C00014F0CEC813F04BEC06F016C0C9F815C0D3
:1027D000C8F814C0C7F813C0C6F8DDC8CDF8DCC807
:1027E000CCF8DBC8CBF80801CB9FDAC8CAF8C9C857
:1027F00016F0C8C815F0C7C814F0C6C813F0CDC885
:102800001AF0CCC819F0CBC818F0CAC817F0B5EC4C
:1028100008F016C00BF915C00AF914C009F913C065
:1028200008F900013AEF15F0EDC816F0ECC815F004
:10283000EBC814F0EAC813F0EDC81AF0ECC819F0B0
:10284000EBC818F0EAC817F0B5EC08F016C0C9F8E4
:1028500015C0C8F814C0C7F813C0C6F8E9C816F008
:10286000E8C815F0E7C814F0E6C813F0E9C81AF094
:10287000E8C819F0E7C818F0E6C817F0B5EC08F09A
:1028800016C0CDF815C0CCF814C0CBF813C0CAF8E8
:10289000C9C816F0C8C815F0C7C814F0C6C813F0E8
:1028A000CDC81AF0CCC819F0CBC818F0CAC817F0B8
:1028B000B3EC07F016C003F915C002F914C001F912
:1028C00013C000F9C5C816F0C4C815F0C3C814F089
:1028D000C2C813F0BDC81AF0BCC819F0BBC818F0C4
:1028E000BAC817F0B1EC07F016C034F015C033F0D9
:1028F00014C032F013C031F034C016F033C015F0FC
:1029000032C014F031C013F013C91AF012C919F013
:1029100011C918F010C917F0B5EC08F016C0F5F899
:1029200015C0F4F814C0F3F813C0F2F8C1C816F0DB
:10293000C0C815F0BFC814F0BEC813F0B9C81AF06B
:10294000B8C819F0B7C818F0B6C817F0B1EC07F05E
:1029500016C0F1F815C0F0F814C0EFF813C0EEF887
:10296000F5C816F0F4C815F0F3C814F0F2C813F067
:10297000F5C81AF0F4C819F0F3C818F0F2C817F047
:10298000B5EC08F016C0C9F815C0C8F814C0C7F8EF
:1029900013C0C6F8F1C816F0F0C815F0EFC814F06F
:1029A000EEC813F0F1C81AF0F0C819F0EFC818F02B
:1029B000EEC817F0B5EC08F016C0CDF815C0CCF88D
:1029C00014C0CBF813C0CAF8C9C816F0C8C815F0AF
:1029D000C7C814F0C6C813F0CDC81AF0CCC819F097
:1029E000CBC818F0CAC817F0B3EC07F016C007F947
:1029F00015C006F914C005F913C004F903C916F08F
:102A000002C915F001C914F000C913F007C91AF082
:102A100006C919F005C918F004C917F001EC07F050
:102A20000108D8B428EF15F003C916F002C915F053
:102A300001C914F000C913F04BEC06F016C00BF9F5
:102A400015C00AF914C009F913C008F93AEF15F0D6
:102A500007C916F006C915F005C914F004C913F02A
:102A60004BEC06F016C00BF915C00AF914C009F9B1
:102A700013C008F9600E166E5F0E156E290E146EE7
:102A8000960E136E0BC91AF00AC919F009C918F08D
:102A900008C917F0B5EC08F016C00BF915C00AF913
:102AA00014C009F913C008F9166A1E0E156E430EFC
:102AB000146E8F0E136E0BC91AF00AC919F009C9EA
:102AC00018F008C917F001EC07F00108D8B471EF4D
:102AD00015F009010B6B1E0E0A6F430E096F8F0E66
:102AE000086F00010BC916F00AC915F009C914F0E6
:102AF00008C913F005EC09F013C00FF914C00EF962
:102B000015C00DF909010C6F00010CC9DEFF0DC9DC
:102B1000DEFF0EC9DEFF0FC9DEFF120019EE35F031
:102B200058EC02F019EE18F047EC02F019EE33F011
:102B300058EC02F018C913F019C914F01AC915F0AD
:102B40001BC916F059EC09F016C01FF915C01EF983
:102B500014C01DF913C01CF935C9DEFF36C9DEFFEC
:102B600033C9DEFF34C9DEFFDE6AACEC0EF019EECD
:102B700037F058EC02F0090138530001D8A4C8EF2F
:102B800015F00B0E0901375D0001D8A0B9EF16F062
:102B900001013C510901185D01013D51090119591B
:102BA00001013E5109011A5901013F5109011B5907
:102BB0001B5101013F19D8B0800A0001D8B8AFEF0E
:102BC00016F038C914F037C913F057EC09F016C0E5
:102BD00023F915C022F914C021F913C020F9DB0E26
:102BE000166E0F0E156E490E146E800E136E23C9ED
:102BF0001AF022C919F021C918F020C917F0B5EC54
:102C000008F016C034F015C033F014C032F013C011
:102C100031F01A6A196A340E186E860E176E34C0B7
:102C200016F033C015F032C014F031C013F04DEC83
:102C300008F016C023F915C022F914C021F913C0F9
:102C400020F9090138530001D8A438EF16F0050E19
:102C50000901375D0001D8B038EF16F01FC92BF914
:102C60001EC92AF91DC929F91CC928F97EEF16F0D9
:102C7000090138530001D8A445EF16F0AB0E090145
:102C8000375D0001D8A04FEF16F01FC92BF91EC900
:102C90002AF91DC929F91CC928F97DEF16F023C9A5
:102CA00016F022C915F021C914F020C913F0D3EC95
:102CB00004F016C032F915C031F914C030F913C050
:102CC0002FF90901309F1FC916F01EC915F01DC943
:102CD00014F01CC913F032C91AF031C919F030C907
:102CE00018F02FC917F04DEC08F016C02BF915C0DD
:102CF0002AF914C029F913C028F900012BC916F0CC
:102D00002AC915F029C914F028C913F005EC09F0F7
:102D100013C027F914C026F915C025F90901246F3D
:102D2000D89627BFD8860001D8B6ACEF16F03D0E76
:102D30000901245D860E2559010E2659000E2759DA
:102D40000001D8A0ACEF16F00901276B010E266F29
:102D5000860E256F3C0E246F0001B7EF16F01BC9DD
:102D600027F91AC926F919C925F918C924F9C1EF93
:102D700016F01BC927F91AC926F919C925F918C966
:102D800024F924C9DEFF25C9DEFF26C9DEFF27C9D5
:102D9000DEFF120019EE3FF047EC02F019EE39F0B9
:102DA00058EC02F039C913F03AC914F057EC09F0A5
:102DB0004A0E1A6E9F0E196E240E186E810E176E33
:102DC000B5EC08F016C03EF915C03DF914C03CF949
:102DD00013C03BF93EC916F03DC915F03CC914F0CB
:102DE0003BC913F005EC09F015C03AF90901396F38
:102DF00042C922F041C921F040C920F03FC91FF06B
:102E00002A6A296A030E286EE80E276EFFEC01F08D
:102E100022C042F921C041F920C040F91FC03FF94A
:102E2000166A156A146A7F0E136E3EC91AF03DC900
:102E300019F03CC918F03BC917F001EC07F0010884
:102E40000001D8B445EF17F042C916F041C915F09A
:102E500040C914F03FC913F059EC09F03EC91AF00B
:102E60003DC919F03CC918F03BC917F04DEC08F00A
:102E700005EC09F013C048F914C047F915C046F92C
:102E80000901456F00014CEF17F00901486B476BD2
:102E9000170E466F340E456F0001D896090148BFE2
:102EA000D8860001D8B669EF17F0090148530AE146
:102EB000475108E1350E455D170E46590001D8A06F
:102EC00069EF17F00901486B476B170E466F340E18
:102ED000456F000146C944F945C943F943C9DEFFBE
:102EE00044C9DEFF120019EE49F047EC02F019EE7A
:102EF0004DF047EC02F019EE51F047EC02F019EEFC
:102F000055F047EC02F001013497166A156A146A0D
:102F1000136A4CC91AF04BC919F04AC918F049C9CB
:102F200017F001EC07F001080001D8B4AFEF17F07B
:102F3000166A156A146A136A54C91AF053C919F04B
:102F400052C918F051C917F001EC07F00108D8B4C4
:102F5000ACEF17F0010134870001C0EF17F0090151
:102F600051530001D8B4BFEF17F0D896090152AF02
:102F7000D8860001D8B6BFEF17F0010134870001F1
:102F8000166A156A146A136A50C91AF04FC919F003
:102F90004EC918F04DC917F001EC07F00108D8B47C
:102FA000E9EF17F0166A156A146A136A58C91AF01D
:102FB00057C919F056C918F055C917F001EC07F0B8
:102FC0000108D8B4E6EF17F0010134870001FAEFE9
:102FD00017F0090155530001D8B4F9EF17F0D8964E
:102FE000090156AFD8860001D8B6F9EF17F00101F4
:102FF00034870001DB0E0901646F0F0E636F490E09
:10300000626F800E616FDB0E686F0F0E676F490E87
:10301000666F810E656FDB0E6C6F0F0E6B6F490E66
:103020006A6F7E0E696F58C916F057C915F056C9F8
:1030300014F055C913F005EC09F0936F935155EC5A
:1030400009F016C097F915C096F914C095F913C088
:1030500094F997C916F096C915F095C914F094C95A
:1030600013F064C91AF063C919F062C918F061C994
:1030700017F0B5EC08F016C034F015C033F014C0EA
:1030800032F013C031F01A6A196A340E186E860EC7
:10309000176E34C016F033C015F032C014F031C0D2
:1030A00013F04DEC08F016C097F915C096F914C04E
:1030B00095F913C094F997C916F096C915F095C9FA
:1030C00014F094C913F0D1EC04F016C097F915C0B0
:1030D00096F914C095F913C094F958C9A3F957C9C2
:1030E000A2F956C9A1F9A19F55C9A0F954C9A7F9D8
:1030F00053C9A6F952C9A5F9A59F51C9A4F950C948
:10310000ABF94FC9AAF94EC9A9F9A99F4DC9A8F9A8
:103110004CC9AFF94BC9AEF94AC9ADF9AD9F49C920
:10312000ACF9A3C916F0A2C915F0A1C914F0A0C941
:1031300013F0ABC91AF0AAC919F0A9C918F0A8C9A7
:1031400017F0B1EC07F016C09BF915C09AF914C03E
:1031500099F913C098F9A7C916F0A6C915F0A5C921
:1031600014F0A4C913F0AFC91AF0AEC919F0ADC973
:1031700018F0ACC917F0B1EC07F016C034F015C068
:1031800033F014C032F013C031F034C016F033C045
:1031900015F032C014F031C013F097C91AF096C977
:1031A00019F095C918F094C917F0B5EC08F016C0DD
:1031B0009FF915C09EF914C09DF913C09CF99BC9D5
:1031C00016F09AC915F099C914F098C913F09BC963
:1031D0001AF09AC919F099C918F098C917F0B5EC06
:1031E00008F016C074F915C073F914C072F913C051
:1031F00071F99FC916F09EC915F09DC914F09CC9BC
:1032000013F09FC91AF09EC919F09DC918F09CC906
:1032100017F0B5EC08F016C078F915C077F914C0AE
:1032200076F913C075F978C916F077C915F076C923
:1032300014F075C913F074C91AF073C919F072C982
:1032400018F071C917F0B3EC07F016C078F915C083
:1032500077F914C076F913C075F978C916F077C9F3
:1032600015F076C914F075C913F04BEC06F016C0D2
:1032700084F915C083F914C082F913C081F9166A64
:10328000CC0E156E580E146E8F0E136E84C91AF084
:1032900083C919F082C918F081C917F0B5EC08F09C
:1032A00016C084F915C083F914C082F913C081F9DE
:1032B00084C916F083C915F082C914F081C913F0CE
:1032C0001A6A196A7A0E186E890E176E75EC07F075
:1032D0003B6EE86A010134B7010E3B140001D8B41B
:1032E000ABEF1CF09BC974F99AC973F999C972F9CB
:1032F0000901729F98C971F99FC978F99EC977F938
:103300009DC976F9769F9CC975F974C916F073C981
:1033100015F072C914F071C913F078C91AF077C9A1
:1033200019F076C918F075C917F04DEC08F016C001
:1033300078F915C077F914C076F913C075F978C912
:1033400016F077C915F076C914F075C913F07BEC47
:1033500003F016C080F915C07FF914C07EF913C0C0
:103360007DF9166A156A340E146E860E136E80C9C6
:103370001AF07FC919F07EC918F07DC917F0B5ECB5
:1033800008F016C034F015C033F014C032F013C08A
:1033900031F034C016F033C015F032C014F031C033
:1033A00013F064C91AF063C919F062C918F061C951
:1033B00017F04DEC08F016C080F915C07FF914C065
:1033C0007EF913C07DF9166A500E156E430E146E09
:1033D0008F0E136E80C91AF07FC919F07EC918F0DC
:1033E0007DC917F0B5EC08F016C074F915C073F973
:1033F00014C072F913C071F9166A156A146A136A57
:1034000058C91AF057C919F056C918F055C917F01C
:1034100001EC07F001080001D8B45DEF1BF0166A5B
:10342000156A146A136A54C91AF053C919F052C9BB
:1034300018F051C917F001EC07F00108D8B4BFEF3C
:103440001AF0166A156A146A136A9BC91AF09AC9A7
:1034500019F099C918F098C917F001EC07F00108A4
:10346000D8B479EF1AF0166A156A146A136A9FC9FC
:103470001AF09EC919F09DC918F09CC917F001EC0B
:1034800007F00108D8B45FEF1AF0166A156A070E44
:10349000146E870E136E80C91AF07FC919F07EC9A9
:1034A00018F07DC917F0B1EC07F016C080F915C00F
:1034B0007FF914C07EF913C07DF977EF1AF0166A10
:1034C000156A340E146E850E136E80C91AF07FC90A
:1034D00019F07EC918F07DC917F0B3EC07F016C0DB
:1034E00080F915C07FF914C07EF913C07DF9BDEFD6
:1034F0001AF0166A156A146A136A9FC91AF09EC9EF
:1035000019F09DC918F09CC917F001EC07F00108EB
:10351000D8B4A5EF1AF0166A156A070E146E870E56
:10352000136E80C91AF07FC919F07EC918F07DC9E1
:1035300017F0B3EC07F016C080F915C07FF914C07E
:103540007EF913C07DF9BDEF1AF0166A156A340EC4
:10355000146E850E136E80C91AF07FC919F07EC9EA
:1035600018F07DC917F0B1EC07F016C080F915C04E
:103570007FF914C07EF913C07DF95BEF1BF0166A6A
:10358000156A146A136A9BC91AF09AC919F099C985
:1035900018F098C917F001EC07F00108D8B417EF3C
:1035A0001BF0166A156A146A136A9FC91AF09EC93D
:1035B00019F09DC918F09CC917F001EC07F001083B
:1035C000D8B4FDEF1AF0166A156A340E146E850E23
:1035D000136E80C91AF07FC919F07EC918F07DC931
:1035E00017F0B3EC07F016C080F915C07FF914C0CE
:1035F0007EF913C07DF915EF1BF0166A156A070EE8
:10360000146E870E136E80C91AF07FC919F07EC937
:1036100018F07DC917F0B1EC07F016C080F915C09D
:103620007FF914C07EF913C07DF95BEF1BF0166AB9
:10363000156A146A136A9FC91AF09EC919F09DC9C8
:1036400018F09CC917F001EC07F00108D8B443EF5B
:103650001BF0166A156A340E146E850E136E80C93F
:103660001AF07FC919F07EC918F07DC917F0B1ECC6
:1036700007F016C080F915C07FF914C07EF913C099
:103680007DF95BEF1BF0166A156A070E146E870E44
:10369000136E80C91AF07FC919F07EC918F07DC970
:1036A00017F0B3EC07F016C080F915C07FF914C00D
:1036B0007EF913C07DF9A9EF1CF0166A156A146A29
:1036C000136A54C91AF053C919F052C918F051C9F4
:1036D00017F001EC07F00108D8B40DEF1CF0166AE2
:1036E000156A146A136A9BC91AF09AC919F099C924
:1036F00018F098C917F001EC07F00108D8B4C7EF2B
:103700001BF0166A156A146A136A9FC91AF09EC9DB
:1037100019F09DC918F09CC917F001EC07F00108D9
:10372000D8B4ADEF1BF0166A156A070E146E870E3B
:10373000136E80C91AF07FC919F07EC918F07DC9CF
:1037400017F0B3EC07F016C080F915C07FF914C06C
:103750007EF913C07DF9C5EF1BF0166A156A340EA9
:10376000146E850E136E80C91AF07FC919F07EC9D8
:1037700018F07DC917F0B1EC07F016C080F915C03C
:103780007FF914C07EF913C07DF90BEF1CF0166AA7
:10379000156A146A136A9FC91AF09EC919F09DC967
:1037A00018F09CC917F001EC07F00108D8B4F3EF4A
:1037B0001BF0166A156A070E146E870E136E80C909
:1037C0001AF07FC919F07EC918F07DC917F0B1EC65
:1037D00007F016C080F915C07FF914C07EF913C038
:1037E0007DF90BEF1CF0166A156A340E146E850E07
:1037F000136E80C91AF07FC919F07EC918F07DC90F
:1038000017F0B3EC07F016C080F915C07FF914C0AB
:103810007EF913C07DF9A9EF1CF0166A156A146AC7
:10382000136A9BC91AF09AC919F099C918F098C976
:1038300017F001EC07F00108D8B465EF1CF0166A28
:10384000156A146A136A9FC91AF09EC919F09DC9B6
:1038500018F09CC917F001EC07F00108D8B44BEF41
:103860001CF0166A156A340E146E850E136E80C92C
:103870001AF07FC919F07EC918F07DC917F0B1ECB4
:1038800007F016C080F915C07FF914C07EF913C087
:103890007DF963EF1CF0166A156A070E146E870E29
:1038A000136E80C91AF07FC919F07EC918F07DC95E
:1038B00017F0B3EC07F016C080F915C07FF914C0FB
:1038C0007EF913C07DF9A9EF1CF0166A156A146A17
:1038D000136A9FC91AF09EC919F09DC918F09CC9B6
:1038E00017F001EC07F00108D8B491EF1CF0166A4C
:1038F000156A340E146E850E136E80C91AF07FC9D6
:1039000019F07EC918F07DC917F0B3EC07F016C0A6
:1039100080F915C07FF914C07EF913C07DF9A9EFB5
:103920001CF0166A156A070E146E870E136E80C996
:103930001AF07FC919F07EC918F07DC917F0B1ECF3
:1039400007F016C080F915C07FF914C07EF913C0C6
:103950007DF97DEF25F058C916F057C915F056C905
:1039600014F055C913F064C91AF063C919F062C99B
:1039700018F061C917F0B5EC08F016C034F015C0A6
:1039800033F014C032F013C031F01A6A196A340EE1
:10399000186E860E176E34C016F033C015F032C0A4
:1039A00014F031C013F04DEC08F016C058F915C0F2
:1039B00057F914C056F913C055F954C916F053C934
:1039C00015F052C914F051C913F064C91AF063C953
:1039D00019F062C918F061C917F0B5EC08F016C00B
:1039E00034F015C033F014C032F013C031F01A6A4D
:1039F000196A340E186E860E176E34C016F033C076
:103A000015F032C014F031C013F04DEC08F016C0C0
:103A100054F915C053F914C052F913C051F950C9E3
:103A200016F04FC915F04EC914F04DC913F064C912
:103A30001AF063C919F062C918F061C917F0B5EC42
:103A400008F016C034F015C033F014C032F013C0C3
:103A500031F01A6A196A340E186E860E176E34C069
:103A600016F033C015F032C014F031C013F04DEC35
:103A700008F016C050F915C04FF914C04EF913C024
:103A80004DF94CC916F04BC915F04AC914F049C993
:103A900013F064C91AF063C919F062C918F061C95A
:103AA00017F0B5EC08F016C034F015C033F014C0B0
:103AB00032F013C031F01A6A196A340E186E860E8D
:103AC000176E34C016F033C015F032C014F031C098
:103AD00013F04DEC08F016C04CF915C04BF914C0AA
:103AE0004AF913C049F94CC916F04BC915F04AC937
:103AF00014F049C913F054C91AF053C919F052C946
:103B000018F051C917F0B1EC07F016C074F915C0E0
:103B100073F914C072F913C071F974C916F073C93E
:103B200015F072C914F071C913F068C91AF067C9A9
:103B300019F066C918F065C917F04DEC08F016C009
:103B400078F915C077F914C076F913C075F978C9FA
:103B500016F077C915F076C914F075C913F005ECA5
:103B600009F015C092F90901916F91C913F092C93A
:103B700014F057EC09F068C91AF067C919F066C962
:103B800018F065C917F0B5EC08F016C060F915C05B
:103B90005FF914C05EF913C05DF974C916F073C9FA
:103BA00015F072C914F071C913F060C91AF05FC939
:103BB00019F05EC918F05DC917F0B1EC07F016C036
:103BC00060F915C05FF914C05EF913C05DF95D536B
:103BD0000001D8B40EEF1EF0D89609015EAFD8866A
:103BE0000001D8B60EEF1EF060C916F05FC915F0DF
:103BF0005EC914F05DC913F068C91AF067C919F0FD
:103C000066C918F065C917F0B3EC07F016C060F983
:103C100015C05FF914C05EF913C05DF954C916F000
:103C200053C915F052C914F051C913F04CC91AF018
:103C30004BC919F04AC918F049C917F0B1EC07F09F
:103C400016C074F915C073F914C072F913C071F974
:103C500074C916F073C915F072C914F071C913F064
:103C600068C91AF067C919F066C918F065C917F074
:103C70004DEC08F016C078F915C077F914C076F944
:103C800013C075F978C916F077C915F076C914F024
:103C900075C913F005EC09F015C092F90901916F8F
:103CA00091C913F092C914F057EC09F068C91AF0E1
:103CB00067C919F066C918F065C917F0B5EC08F0C6
:103CC00016C05CF915C05BF914C05AF913C059F954
:103CD00074C916F073C915F072C914F071C913F0E4
:103CE0005CC91AF05BC919F05AC918F059C917F024
:103CF000B1EC07F016C05CF915C05BF914C05AF9B5
:103D000013C059F959530001D8B4A9EF1EF0D89641
:103D100009015AAFD8860001D8B6A9EF1EF05CC9D8
:103D200016F05BC915F05AC914F059C913F068C9E7
:103D30001AF067C919F066C918F065C917F0B3EC35
:103D400007F016C05CF915C05BF914C05AF913C02E
:103D500059F958C974F957C973F956C972F9090163
:103D60005551D8B43E84D8A45505716F74C916F066
:103D700073C915F072C914F071C913F06CC91AF047
:103D80006BC919F06AC918F069C917F0B3EC07F0EC
:103D900016C074F915C073F914C072F913C071F923
:103DA00074C916F073C915F072C914F071C913F013
:103DB000ADEC04F016C074F915C073F914C072F9B3
:103DC00013C071F950C978F94FC977F94EC976F91E
:103DD0004D51D8B43E84D8A44D05756F78C916F0FE
:103DE00077C915F076C914F075C913F06CC91AF0CB
:103DF0006BC919F06AC918F069C917F0B3EC07F07C
:103E000016C078F915C077F914C076F913C075F9A2
:103E100078C916F077C915F076C914F075C913F092
:103E2000ADEC04F016C078F915C077F914C076F936
:103E300013C075F978C916F077C915F076C914F072
:103E400075C913F074C91AF073C919F072C918F062
:103E500071C917F04DEC08F016C070F915C06FF974
:103E600014C06EF913C06DF970C916F06FC915F062
:103E70006EC914F06DC913F061EC02F016C070F950
:103E800015C06FF914C06EF913C06DF950C916F062
:103E90004FC915F04EC914F04DC913F058C91AF0A6
:103EA00057C919F056C918F055C917F0B1EC07F009
:103EB00016C074F915C073F914C072F913C071F902
:103EC00071530001D8B470EF1FF0D896090172AF9A
:103ED000D8860001D8B670EF1FF0800E0901721B62
:103EE000000172BF0DD0DC0E0901745D240E735900
:103EF000340E7259500E71590001D8B094EF1FF072
:103F000058C916F057C915F056C914F055C913F021
:103F1000D1EC04F016C07CF915C07BF914C07AF915
:103F200013C079F9C8EF1FF050C916F04FC915F04A
:103F30004EC914F04DC913F058C91AF057C919F0F9
:103F400056C918F055C917F0B1EC07F016C074F94E
:103F500015C073F914C072F913C071F974C916F061
:103F600073C915F072C914F071C913F070C91AF051
:103F70006FC919F06EC918F06DC917F04DEC08F053
:103F800016C07CF915C07BF914C07AF913C079F911
:103F900060C916F05FC915F05EC914F05DC913F071
:103FA0005CC91AF05BC919F05AC918F059C917F061
:103FB00001EC07F00108D8B4B7EF21F060C974F93B
:103FC0005FC973F95EC972F95DC971F9166A156A3C
:103FD000146A136A70C91AF06FC919F06EC918F023
:103FE0006DC917F001EC07F00108D8B426EF20F0F6
:103FF00074C916F073C915F072C914F071C913F0C1
:1040000070C91AF06FC919F06EC918F06DC917F0B0
:104010004DEC08F016C078F915C077F914C076F9A0
:1040200013C075F978C916F077C915F076C914F080
:1040300075C913F07BEC03F016C078F915C077F959
:1040400014C076F913C075F934EF21F009016D53EE
:104050000001D8A48AEF20F0166A156A146A136A60
:1040600074C91AF073C919F072C918F071C917F040
:1040700001EC07F00108D8B44EEF20F064C978F9DC
:1040800063C977F962C976F909016151D8B43E84F0
:10409000D8A46105756F000188EF20F00901715304
:1040A0000001D8B482EF20F0D896090172AFD8860B
:1040B0000001D8B682EF20F0166A156A146A136AF6
:1040C00064C91AF063C919F062C918F061C917F020
:1040D000B1EC07F016C034F015C033F014C032F064
:1040E00013C031F034C078F933C077F932C076F9B3
:1040F0003150D8B43E84D8A431040901756F000151
:1041000087EF20F00901806B7F6B7E6B7D6B000178
:1041100034EF21F009016D530001D8B434EF21F0E0
:10412000D89609016EAFD8860001D8B634EF21F0D9
:10413000090171530001D8B4EEEF20F0D8960901BF
:1041400072AFD8860001D8B6EEEF20F074C916F031
:1041500073C915F072C914F071C913F070C91AF05F
:104160006FC919F06EC918F06DC917F04DEC08F061
:1041700016C078F915C077F914C076F913C075F92F
:1041800078C916F077C915F076C914F075C913F01F
:104190007BEC03F016C078F915C077F914C076F9F6
:1041A00013C075F978C916F077C915F076C914F0FF
:1041B00075C913F064C91AF063C919F062C918F01F
:1041C00061C917F0B1EC07F016C078F915C077F99E
:1041D00014C076F913C075F934EF21F074C916F0E4
:1041E00073C915F072C914F071C913F070C91AF0CF
:1041F0006FC919F06EC918F06DC917F04DEC08F0D1
:1042000016C078F915C077F914C076F913C075F99E
:1042100078C916F077C915F076C914F075C913F08E
:104220007BEC03F016C078F915C077F914C076F965
:1042300013C075F978C916F077C915F076C914F06E
:1042400075C913F064C91AF063C919F062C918F08E
:1042500061C917F0B3EC07F016C078F915C077F90B
:1042600014C076F913C075F978C916F077C915F03E
:1042700076C914F075C913F068C91AF067C919F046
:1042800066C918F065C917F04DEC08F016C074F94E
:1042900015C073F914C072F913C071F974C916F01E
:1042A00073C915F072C914F071C913F005EC09F067
:1042B00015C092F90901916F91C913F092C914F0D8
:1042C00057EC09F068C91AF067C919F066C918F007
:1042D00065C917F0B5EC08F016C080F915C07FF974
:1042E00014C07EF913C07DF978C916F077C915F0AE
:1042F00076C914F075C913F080C91AF07FC919F096
:104300007EC918F07DC917F0B1EC07F016C080F92E
:1043100015C07FF914C07EF913C07DF97D530001EB
:10432000D8B4B5EF21F0D89609017EAFD886000148
:10433000D8B6B5EF21F080C916F07FC915F07EC957
:1043400014F07DC913F068C91AF067C919F066C97D
:1043500018F065C917F0B3EC07F016C080F915C066
:104360007FF914C07EF913C07DF986EF23F05CC994
:1043700074F95BC973F95AC972F9800E0901721B8D
:1043800059C971F9166A156A146A136A70C91AF064
:104390006FC919F06EC918F06DC917F001EC07F07C
:1043A00001080001D8B403EF22F074C916F073C9F4
:1043B00015F072C914F071C913F070C91AF06FC901
:1043C00019F06EC918F06DC917F04DEC08F016C061
:1043D00078F915C077F914C076F913C075F978C962
:1043E00016F077C915F076C914F075C913F07BEC97
:1043F00003F016C078F915C077F914C076F913C028
:1044000075F905EF23F009016D530001D8A45BEFA6
:1044100022F0166A156A146A136A74C91AF073C90D
:1044200019F072C918F071C917F001EC07F0010812
:10443000D8B42BEF22F064C978F963C977F962C95F
:1044400076F909016151D8B43E84D8A46105756F2D
:10445000000159EF22F0090171530001D8B453EF64
:1044600022F0D896090172AFD8860001D8B653EF72
:1044700022F064C90EF063C90DF062C90CF0800E21
:104480000C1A61C90BF00EC078F90DC077F90CC099
:1044900076F90B50D8B43E84D8A40B040901756F8B
:1044A000000158EF22F00901806B7F6B7E6B7D6B02
:1044B000000105EF23F009016D530001D8B405EFA9
:1044C00023F0D89609016EAFD8860001D8B605EF63
:1044D00023F0090171530001D8B4BFEF22F0D89640
:1044E000090172AFD8860001D8B6BFEF22F074C9B7
:1044F00016F073C915F072C914F071C913F070C9C0
:104500001AF06FC919F06EC918F06DC917F04DECAB
:1045100008F016C078F915C077F914C076F913C001
:1045200075F978C916F077C915F076C914F075C910
:1045300013F07BEC03F016C078F915C077F914C0BE
:1045400076F913C075F978C916F077C915F076C9F0
:1045500014F075C913F064C91AF063C919F062C97F
:1045600018F061C917F0B1EC07F016C078F915C062
:1045700077F914C076F913C075F905EF23F074C903
:1045800016F073C915F072C914F071C913F070C92F
:104590001AF06FC919F06EC918F06DC917F04DEC1B
:1045A00008F016C078F915C077F914C076F913C071
:1045B00075F978C916F077C915F076C914F075C980
:1045C00013F07BEC03F016C078F915C077F914C02E
:1045D00076F913C075F978C916F077C915F076C960
:1045E00014F075C913F064C91AF063C919F062C9EF
:1045F00018F061C917F0B3EC07F016C078F915C0D0
:1046000077F914C076F913C075F978C916F077C92F
:1046100015F076C914F075C913F068C91AF067C9A6
:1046200019F066C918F065C917F04DEC08F016C00E
:1046300074F915C073F914C072F913C071F974C913
:1046400016F073C915F072C914F071C913F005ECB6
:1046500009F015C092F90901916F91C913F092C93F
:1046600014F057EC09F068C91AF067C919F066C967
:1046700018F065C917F0B5EC08F016C080F915C040
:104680007FF914C07EF913C07DF978C916F077C997
:1046900015F076C914F075C913F080C91AF07FC9F6
:1046A00019F07EC918F07DC917F0B1EC07F016C0FB
:1046B00080F915C07FF914C07EF913C07DF97D53D0
:1046C0000001D8B486EF23F0D89609017EAFD886D2
:1046D0000001D8B686EF23F080C916F07FC915F027
:1046E0007EC914F07DC913F068C91AF067C919F0C2
:1046F00066C918F065C917F0B3EC07F016C080F969
:1047000015C07FF914C07EF913C07DF9166A156AC9
:10471000340E146E860E136E80C91AF07FC919F01C
:104720007EC918F07DC917F0B5EC08F016C080F905
:1047300015C07FF914C07EF913C07DF980C916F049
:104740007FC915F07EC914F07DC913F064C91AF051
:1047500063C919F062C918F061C917F04DEC08F08F
:1047600016C080F915C07FF914C07EF913C07DF919
:10477000166A156A330E146E870E136E80C91AF00E
:104780007FC919F07EC918F07DC917F001EC07F058
:104790000108D8B4D4EF23F00901806B800E7F6F3D
:1047A000330E7E6F870E7D6F000160C916F05FC902
:1047B00015F05EC914F05DC913F05CC91AF05BC94D
:1047C00019F05AC918F059C917F001EC07F001089F
:1047D000D8B49BEF24F07CC916F07BC915F07AC9D8
:1047E00014F079C913F07CC91AF07BC919F07AC9A1
:1047F00018F079C917F0B5EC08F016C074F915C0B7
:1048000073F914C072F913C071F960C916F05FC969
:1048100015F05EC914F05DC913F060C91AF05FC9E4
:1048200019F05EC918F05DC917F0B5EC08F016C0B4
:1048300078F915C077F914C076F913C075F974C901
:1048400016F073C915F072C914F071C913F078C964
:104850001AF077C919F076C918F075C917F0B5ECD8
:1048600008F016C074F915C073F914C072F913C0BA
:1048700071F950C916F04FC915F04EC914F04DC961
:1048800013F058C91AF057C919F056C918F055C98C
:1048900017F0B1EC07F016C078F915C077F914C01D
:1048A00076F913C075F978C916F077C915F076C98D
:1048B00014F075C913F078C91AF077C919F076C9E0
:1048C00018F075C917F0B5EC08F016C078F915C0E6
:1048D00077F914C076F913C075F974C916F073C965
:1048E00015F072C914F071C913F078C91AF077C9BC
:1048F00019F076C918F075C917F0B3EC07F016C0B7
:1049000084F915C083F914C082F913C081F984C9F0
:1049100016F083C915F082C914F081C913F04BEC6D
:1049200006F016C084F915C083F914C082F913C0CB
:1049300081F949EF25F07CC916F07BC915F07AC9D9
:1049400014F079C913F07CC91AF07BC919F07AC93F
:1049500018F079C917F0B5EC08F016C074F915C055
:1049600073F914C072F913C071F95CC916F05BC910
:1049700015F05AC914F059C913F05CC91AF05BC993
:1049800019F05AC918F059C917F0B5EC08F016C05B
:1049900078F915C077F914C076F913C075F974C9A0
:1049A00016F073C915F072C914F071C913F078C903
:1049B0001AF077C919F076C918F075C917F0B5EC77
:1049C00008F016C074F915C073F914C072F913C059
:1049D00071F950C916F04FC915F04EC914F04DC900
:1049E00013F058C91AF057C919F056C918F055C92B
:1049F00017F0B1EC07F016C078F915C077F914C0BC
:104A000076F913C075F978C916F077C915F076C92B
:104A100014F075C913F078C91AF077C919F076C97E
:104A200018F075C917F0B5EC08F016C078F915C084
:104A300077F914C076F913C075F974C916F073C903
:104A400015F072C914F071C913F078C91AF077C95A
:104A500019F076C918F075C917F0B3EC07F016C055
:104A600084F915C083F914C082F913C081F984C98F
:104A700016F083C915F082C914F081C913F04BEC0C
:104A800006F016C084F915C083F914C082F913C06A
:104A900081F9166A156A480E146E850E136E84C964
:104AA0001AF083C919F082C918F081C917F001EC16
:104AB00007F00108D8B462EF25F00901846B836B1D
:104AC000826B816B0001320E166EA50E156E420EC2
:104AD000146E950E136E84C91AF083C919F082C939
:104AE00018F081C917F0B5EC08F016C084F915C0AC
:104AF00083F914C082F913C081F982BF0DD0400E32
:104B00000901845DD70E8359340E8259900E815964
:104B10000001D8B0A1EF25F084C916F083C915F0C3
:104B200082C914F081C913F005EC09F013C088F9AB
:104B300014C087F915C086F90901856F0001A9EF36
:104B400025F00901886B020E876FD30E866F5D0E0C
:104B5000856F000180C916F07FC915F07EC914F079
:104B60007DC913F005EC09F013C08CF914C08BF962
:104B700015C08AF90901896F8CC922F08BC921F00F
:104B80008AC920F089C91FF02A6A0F0E296E420EC9
:104B9000286E400E276EFFEC01F022C08CF921C078
:104BA0008BF920C08AF91FC089F9906B8F6B8E6BCF
:104BB0008D6B855189258D6F86518A218E6F875126
:104BC0008B218F6F88518C21906F8DC9DEFF8EC92C
:104BD000DEFF8FC9DEFF90C9DEFF00011200010E6B
:104BE0000601396F4D0E386F010E3B6F2C0E3A6F78
:104BF000010E3D6F2C0E3C6F010E3F6F2C0E3E6F71
:104C0000010E416F2C0E406F010E436F2C0E426F50
:104C1000010E456F2C0E446F010E476F2C0E466F30
:104C2000010E496F900E486F010E4B6FF40E4A6FE4
:104C3000020E4D6F580E4C6F020E4F6FBC0E4E6F32
:104C4000030E516F200E506F030E536F840E526F80
:104C5000030E556FE80E546F030E576FE80E566F34
:104C6000030E596FE80E586F030E5B6FE80E5A6F14
:104C7000030E5D6FE80E5C6F030E5F6FE80E5E6FF4
:104C8000030E616FE80E606F030E636FE80E626FD4
:104C9000030E656FE80E646F030E676FE80E666FB4
:104CA000030E696FE80E686F030E6B6FE80E6A6F94
:104CB000030E6D6FE80E6C6F030E6F6FE80E6E6F74
:104CC000040E716F4C0E706F040E736FB00E726F26
:104CD000050E756F140E746F050E776F780E766F74
:104CE000050E796FDC0E786F050E7B6F780E7A6F8C
:104CF000050E7D6F140E7C6F040E7F6FB00E7E6FFD
:104D0000030E816FE80E806F030E836FDE0E826FDD
:104D1000030E856FD40E846F030E876FCA0E866FE5
:104D2000030E896FD40E886F030E8B6FDE0E8A6FB1
:104D3000030E8D6FE80E8C6F040E8F6F4C0E8E6F0E
:104D4000040E916FB00E906F040E936FB00E926FC1
:104D5000040E956FB00E946F040E976FB00E966FA1
:104D6000040E996FB00E986F040E9B6FB00E9A6F81
:104D7000040E9D6FB00E9C6F040E9F6FB00E9E6F61
:104D8000040EA16FB00EA06F030EA36FE80EA26F0A
:104D9000030EA56FDE0EA46F030EA76FD40EA66FD1
:104DA000030EA96FCA0EA86F030EAB6FD40EAA6FC5
:104DB000030EAD6FDE0EAC6F030EAF6FE80EAE6F7D
:104DC000030EB16F840EB06F030EB36F200EB26F7F
:104DD000020EB56FBC0EB46F020EB76F580EB66FF1
:104DE000020EB96F580EB86F020EBB6F580EBA6F35
:104DF000020EBD6F580EBC6F020EBF6F580EBE6F15
:104E0000020EC16F580EC06F020EC36F580EC26FF4
:104E1000020EC56F580EC46F020EC76F580EC66FD4
:104E2000020EC96F580EC86F020ECB6F580ECA6FB4
:104E3000020ECD6F580ECC6F020ECF6F580ECE6F94
:104E4000020ED16F580ED06F020ED36F580ED26F74
:104E5000020ED56F580ED46F020ED76F580ED66F54
:104E6000020ED96F580ED86F020EDB6F580EDA6F34
:104E7000020EDD6F8A0EDC6F020EDF6F8A0EDE6FB0
:104E8000020EE16F8A0EE06F020EE36F8A0EE26F90
:104E9000020EE56F8A0EE46F020EE76F8A0EE66F70
:104EA000020EE96F8A0EE86F020EEB6F8A0EEA6F50
:104EB000020EED6F8A0EEC6F020EEF6F8A0EEE6F30
:104EC000020EF16F8A0EF06F020EF36F260EF26F74
:104ED000020EF56F260EF46F020EF76F260EF66FB8
:104EE000020EF96F260EF86F020EFB6F260EFA6F98
:104EF000020EFD6F260EFC6F020EFF6F260EFE6F78
:104F0000020E0701016F260E006F020E036F260EC0
:104F1000026F020E056F260E046F020E076F260E3B
:104F2000066F020E096F260E086F020E0B6F260E1B
:104F30000A6F020E0D6F260E0C6F020E0F6F260EFB
:104F40000E6F020E116F260E106F010E136FF40E0E
:104F5000126F010E156FC20E146F010E176F900EB7
:104F6000166F010E196F5E0E186F010E1B6F2C0E5F
:104F70001A6F010E1D6F2C0E1C6F010E1F6F2C0E71
:104F80001E6F010E216F2C0E206F010E236F2C0E51
:104F9000226F010E256F2C0E246F010E276F2C0E31
:104FA000266F296B286B2B6B140E2A6F2D6B280E26
:104FB0002C6F2F6B3C0E2E6F316B500E306F336B9E
:104FC000640E326F356B780E346F376B8C0E366F24
:104FD000396BA00E386F3B6BB40E3A6F3D6BC80E49
:104FE0003C6F3F6BB40E3E6F416BA00E406F436B46
:104FF0008C0E426F456B780E446F476B640E466FA4
:10500000496B500E486F4B6B3C0E4A6F4D6B280E30
:105010004C6F4F6B140E4E6F516B506B536B050EF4
:10502000526F556B0A0E546F576B0A0E566F596BC1
:105030000A0E586F5B6B0A0E5A6F5D6B0A0E5C6F3F
:105040005F6B0A0E5E6F616B0A0E606F636B0A0E18
:10505000626F656B0F0E646F676B140E666F696B22
:10506000190E686F6B6B1E0E6A6F6D6B230E6C6F83
:105070006F6B280E6E6F716B0A0E706F736B0F0E75
:10508000726F756B140E746F776B190E766F796B88
:105090001E0E786F7B6B230E7A6F7D6B280E7C6FF4
:1050A0007F6B2D0E7E6F816B320E806F836B370EA0
:1050B000826F856B3C0E846F876B3D0E866F896BAC
:1050C0003E0E886F8B6B3D0E8A6F8D6B3C0E8C6F26
:1050D0008F6B3B0E8E6F916B3A0E906F936B3B0E06
:1050E000926F956B460E946F976B500E966F996BFF
:1050F0005A0E986F9B6B640E9A6F9D6B6E0E9C6F31
:105100009F6B780E9E6FA16B820EA06FA36B8C0EAF
:10511000A26FA56B960EA46FA76BA00EA66FA96BCE
:10512000AA0EA86FAB6BB40EAA6FAD6BBE0EAC6FC0
:10513000AF6BC80EAE6FB16BD20EB06FB36BD30E48
:10514000B26FB56BD40EB46FB76BD30EB66FB96BCD
:10515000D40EB86FBB6BD30EBA6FBD6BD40EBC6FE1
:10516000BF6BD50EBE6FC16BD40EC06FC36BD50EB7
:10517000C26FC56BD60EC46FC76BDC0EC66FC96B32
:10518000F00EC86F010ECB6F040ECA6F010ECD6F0B
:10519000180ECC6F010ECF6F2C0ECE6F010ED16F9B
:1051A000400ED06F010ED36F540ED26F010ED56F2B
:1051B0005E0ED46F010ED76F5E0ED66F010ED96FE3
:1051C0005E0ED86F010EDB6F5E0EDA6F010EDD6FC3
:1051D000630EDC6FDF6BDE6BE16B0A0EE06FE36B7F
:1051E000140EE26FE56B1E0EE46FE76B280EE66FA0
:1051F000E96B320EE86FEB6B3C0EEA6FED6B460E1F
:10520000EC6FEF6B500EEE6FF16B5A0EF06FF36BAD
:105210005F0EF26FF56B5F0EF46FF76B5F0EF66F5C
:10522000F96B5F0EF86FFB6B5F0EFA6FFD6B5F0E35
:10523000FC6FFF6B5F0EFE6F0801016B5F0E006F6E
:10524000036B5F0E026F056B590E046F076B530EF5
:10525000066F096B4D0E086F0B6B470E0A6F0D6BD7
:10526000410E0C6F0F6B3B0E0E6F116B350E106FF6
:10527000136B2F0E126F156B290E146F176B230E05
:10528000166F00011200A30E0901D16FA20ED26F9A
:10529000AB0ED36FAA0ED46F01014B510A0DF3CFA1
:1052A00031F0F4CF32F04C5131240B6E0BC0B0F919
:1052B0004D510A0DF3CF31F0F4CF32F04E5131247D
:1052C0000B6E0BC0B1F94F510A0DF3CF31F0F4CF93
:1052D00032F0505131240B6E0BC0B2F952510A0D0D
:1052E000F3CF31F0F4CF32F0535131240B6E0BC0B9
:1052F000B3F954510A0DF3CF31F0F4CF32F05551D8
:1053000031240B6E0BC0B4F956510A0DF3CF31F0B6
:10531000F4CF32F0575131240B6E0BC0B5F9585110
:105320000A0DF3CF31F0F4CF32F0595131240B6E26
:105330000BC0B6F94E0E5A5D0001D8A4A4EF29F0B7
:105340006BC1B7F9AAEF29F00A0E01016B250B6EAC
:105350000BC0B7F9000101015B510A0DF3CF31F029
:10536000F4CF32F05C5131240B6E0BC0B8F95D51B3
:105370000A0DF3CF31F0F4CF32F05E5131240B6ED1
:105380000BC0B9F95F510A0DF3CF31F0F4CF32F011
:10539000605131240B6E0BC0BAF961510A0DF3CF85
:1053A00031F0F4CF32F0625131240B6E0BC0BBF9F7
:1053B000450E645D0001D8A4E7EF29F0140E010149
:1053C00063250B6E0BC0BCF90001EDEF29F01E0E3A
:1053D000010163250B6E0BC0BCF900010101655191
:1053E0000A0DF3CF31F0F4CF32F0665131240B6E59
:1053F0000BC0BDF967510A0DF3CF31F0F4CF32F095
:10540000685131240B6E0BC0BEF96C510A0DF3CFFD
:1054100031F0F4CF32F06D5131240B6E0BC0BFF977
:105420006E510A0DF3CF31F0F4CF32F06F513124C9
:105430000B6E0BC0C0F970510A0DF3CF31F0F4CFF1
:1054400032F0715131240B6E0BC0C1F972510A0D4B
:10545000F3CF31F0F4CF32F0735131240B6E0BC027
:10546000C2F905011A510A0DF3CF31F0F4CF32F031
:105470001B5131240B6E0BC0C3F91C510A0DF3CF25
:1054800031F0F4CF32F01D5131240B6E0BC0C4F952
:10549000EA0E0901C56FC66B0001160E0901C65D53
:1054A0000001D8B0D7EF2AF0D896BBBFD886D8B6BF
:1054B00067EF2AF0FE0EB85DFF0EB959010EBA591A
:1054C000000EBB59D8A067EF2AF038EF2BF0D89622
:1054D000BBBFD886D8B6B5EF2AF0000EBB5DD8A00A
:1054E000B5EF2AF011E1000EBA5DD8A0B5EF2AF0B1
:1054F0000BE1FF0EB95DD8A0B5EF2AF005E1FE0E75
:10550000B85DD8A0B5EF2AF0B82B000EB923BA23A6
:10551000BB23FF0EB85D0901C76FFF0E0001B9592B
:105520000901C86F000E0001BA590901C96F000EC8
:105530000001BB590901CA6FC8C9CCF9C7C9CBF969
:10554000D451FCEC00F0CC51FCEC00F0CB51FCEC65
:1055500000F009EEB0F0C651EB50FAEC00F0050E89
:1055600051EC01F00001D1EF2AF0B82B000EB92365
:10557000BA23BB23B9C0CCF9B8C0CBF90901D251C9
:10558000FCEC00F0CC51FCEC00F0CB51FCEC00F05A
:1055900009EEB0F0C651EB50FAEC00F0050E51ECFC
:1055A00001F000010901C62B0001D8A475D7BBC0CA
:1055B000CDF9BAC0CEF9B9C0CFF9B8C0D0F9090158
:1055C000D251FCEC00F00001BD51FCEC00F0BC51EC
:1055D000FCEC00F00901CD51FAEC00F0050E51ECA5
:1055E00001F0D251FCEC00F0010E0001BC25316E3F
:1055F000000EBD21326E3250FCEC00F03150FCEC5C
:1056000000F00901CE51FAEC00F0050E51EC01F06A
:10561000D251FCEC00F0020E0001BC25316E000EF0
:10562000BD21326E3250FCEC00F03150FCEC00F049
:105630000901CF51FAEC00F0050E51EC01F0D25106
:10564000FCEC00F0030E0001BC25316E000EBD2104
:10565000326E3250FCEC00F03150FCEC00F00901ED
:10566000D051FAEC00F0050E51EC01F000011200EF
:10567000010EB66FB7EF33F012000A0E895DD8A4A1
:105680004EEF2BF099ECADF09D0EDE6E200EDE6E2F
:10569000010EDE6E34EC9CF064EF31F00B0E895D90
:1056A000D8A45FEF2BF060ECADF02F0EDE6E0C0E89
:1056B000DE6E020EDE6E34EC9CF064EF31F00C0E08
:1056C000895DD8A470EF2BF060ECADF02D0EDE6E8E
:1056D0001B0EDE6E020EDE6E34EC9CF064EF31F0D9
:1056E0000D0E895DD8A481EF2BF060ECADF02B0E90
:1056F000DE6E0E0EDE6E020EDE6E34EC9CF064EF9B
:1057000031F0140E895DD8A491EF2BF099ECADF037
:105710009F0EDE6E140EDE6EDE6A34EC9CF064EFDB
:1057200031F0150E895DD8A4A9EF2BF0C2ECADF0D5
:10573000250EDE6E1B0EDE6EDE6A34EC9CF0330E40
:10574000DE6E0E0EDE6E0C0EDE6E34EC9CF064EF40
:1057500031F0160E895DD8A4C1EF2BF0C2ECADF08C
:10576000270EDE6E0C0EDE6EDE6A34EC9CF0350E1B
:10577000DE6E1B0EDE6E0C0EDE6E34EC9CF064EF03
:1057800031F0170E895DD8A4D9EF2BF0C2ECADF043
:10579000270EDE6E0C0EDE6EDE6A34EC9CF0330EED
:1057A000DE6E0E0EDE6E0C0EDE6E34EC9CF064EFE0
:1057B00031F01E0E895DD8A4EAEF2BF099ECADF024
:1057C000A30EDE6E110EDE6E010EDE6E34EC9CF06A
:1057D00064EF31F01F0E895DD8A402EF2CF0C2EC0B
:1057E000ADF0250EDE6E1B0EDE6EDE6A34EC9CF034
:1057F000970EDE6E210EDE6E0C0EDE6E34EC9CF02B
:1058000064EF31F0200E895DD8A41AEF2CF0C2ECC1
:10581000ADF0250EDE6E1B0EDE6EDE6A34EC9CF003
:10582000950EDE6E210EDE6E0C0EDE6E34EC9CF0FC
:1058300064EF31F0210E895DD8A432EF2CF0C2EC78
:10584000ADF0250EDE6E1B0EDE6EDE6A34EC9CF0D3
:10585000930EDE6E210EDE6E0C0EDE6E34EC9CF0CE
:1058600064EF31F0220E895DD8A44AEF2CF0C2EC2F
:10587000ADF0250EDE6E1B0EDE6EDE6A34EC9CF0A3
:10588000990EDE6E210EDE6E0C0EDE6E34EC9CF098
:1058900064EF31F0230E895DD8A462EF2CF0C2ECE6
:1058A000ADF0270EDE6E0C0EDE6EDE6A34EC9CF080
:1058B000950EDE6E210EDE6E0C0EDE6E34EC9CF06C
:1058C00064EF31F0240E895DD8A47AEF2CF0C2EC9D
:1058D000ADF0270EDE6E0C0EDE6EDE6A34EC9CF050
:1058E000930EDE6E210EDE6E0C0EDE6E34EC9CF03E
:1058F00064EF31F0250E895DD8A492EF2CF0C2EC54
:10590000ADF0270EDE6E0C0EDE6EDE6A34EC9CF01F
:10591000970EDE6E210EDE6E0C0EDE6E34EC9CF009
:1059200064EF31F0260E895DD8A4AAEF2CF0C2EC0A
:10593000ADF0270EDE6E0C0EDE6EDE6A34EC9CF0EF
:10594000990EDE6E210EDE6E0C0EDE6E34EC9CF0D7
:1059500064EF31F0270E895DD8A4C2EF2CF0C2ECC1
:10596000ADF0230EDE6E0E0EDE6EDE6A34EC9CF0C1
:10597000930EDE6E210EDE6E0C0EDE6E34EC9CF0AD
:1059800064EF31F0280E895DD8A4DAEF2CF0C2EC78
:10599000ADF0230EDE6E0E0EDE6EDE6A34EC9CF091
:1059A000950EDE6E210EDE6E0C0EDE6E34EC9CF07B
:1059B00064EF31F0290E895DD8A4F2EF2CF0C2EC2F
:1059C000ADF0230EDE6E0E0EDE6EDE6A34EC9CF061
:1059D000970EDE6E210EDE6E0C0EDE6E34EC9CF049
:1059E00064EF31F02A0E895DD8A40AEF2DF0C2ECE5
:1059F000ADF0230EDE6E0E0EDE6EDE6A34EC9CF031
:105A0000990EDE6E210EDE6E0C0EDE6E34EC9CF016
:105A100064EF31F0320E895DD8A41BEF2DF099ECC4
:105A2000ADF0030EDE6E340EDE6E020EDE6E34EC72
:105A30009CF064EF31F0330E895DD8A43BEF2DF07C
:105A4000C2ECADF0030EDE6E0A0EDE6E0C0EDE6EE4
:105A500034EC9CF0290EDE6E480EDE6E0D0EDE6E0E
:105A600034EC9CF0330EDE6E0E0EDE6EDE6A34EC2D
:105A70009CF064EF31F0340E895DD8A45BEF2DF01B
:105A8000C2ECADF0030EDE6E0A0EDE6E0C0EDE6EA4
:105A900034EC9CF0290EDE6E480EDE6E0D0EDE6ECE
:105AA00034EC9CF02F0EDE6E0C0EDE6EDE6A34ECF3
:105AB0009CF064EF31F0350E895DD8A482EF2DF0B3
:105AC000C2ECADF0030EDE6E0A0EDE6E0C0EDE6E64
:105AD00034EC9CF0290EDE6E480EDE6E0D0EDE6E8E
:105AE00034EC9CF0030EDE6E070EDE6EDE6A34ECE4
:105AF0009CF0410EDE6E450EDE6EDE6A34EC9CF0EC
:105B000064EF31F0360E895DD8A4AAEF2DF0C2EC17
:105B1000ADF0030EDE6E0A0EDE6E0C0EDE6E34ECA1
:105B20009CF0290EDE6E480EDE6E0D0EDE6E34EC3D
:105B30009CF0030EDE6E060EDE6EDE6A34EC9CF028
:105B4000190EDE6E440EDE6E010EDE6E34EC9CF03D
:105B500064EF31F0370E895DD8A4D1EF2DF0C2EC9F
:105B6000ADF0030EDE6E0A0EDE6E0C0EDE6E34EC51
:105B70009CF0290EDE6E480EDE6E0D0EDE6E34ECED
:105B80009CF0310EDE6E200EDE6EDE6A34EC9CF090
:105B9000030EDE6E470EDE6EDE6A34EC9CF064EFC0
:105BA00031F0380E895DD8A4F8EF2DF0C2ECADF0DD
:105BB000030EDE6E060EDE6E0C0EDE6E34EC9CF016
:105BC000190EDE6E440EDE6E0D0EDE6E34EC9CF0B1
:105BD000310EDE6E200EDE6EDE6A34EC9CF0030EBB
:105BE000DE6E470EDE6EDE6A34EC9CF064EF31F060
:105BF000390E895DD8A41FEF2EF0C2ECADF0330E44
:105C0000DE6E0E0EDE6EDE6A34EC9CF0650EDE6E2D
:105C1000DE6A0C0EDE6E34EC9CF0670EDE6E100E4B
:105C2000DE6E0C0EDE6E34EC9CF0690EDE6E210E24
:105C3000DE6E0C0EDE6E34EC9CF064EF31F03A0E4A
:105C4000895DD8A438EF2EF060ECADF0030EDE6E67
:105C5000340EDE6E010EDE6E34EC9CF0170EDE6E3E
:105C60002F0EDE6E040EDE6E34EC9CF064EF31F02D
:105C70003C0E895DD8A449EF2EF099ECADF0140EDE
:105C8000DE6E200EDE6E010EDE6E34EC9CF064EFF4
:105C900031F03D0E895DD8A45AEF2EF060ECADF0E6
:105CA000140EDE6E200EDE6E020EDE6E34EC9CF004
:105CB00064EF31F03E0E895DD8A491EF2EF0C2EC76
:105CC000ADF08B0EDE6E220EDE6EDE6A34EC9CF0E2
:105CD000240EDE6E350EDE6E010EDE6E34EC9CF0B0
:105CE0008A0EDE6E3C0EDE6EDE6A34EC9CF0200E18
:105CF000DE6E140EDE6E0C0EDE6E34EC9CF0240EA6
:105D0000DE6E270EDE6E0D0EDE6E34EC9CF0220E83
:105D1000DE6E2E0EDE6E0C0EDE6E34EC9CF064EF4A
:105D200031F03F0E895DD8A4B9EF2EF0C2ECADF092
:105D30008B0EDE6E220EDE6E0C0EDE6E34EC9CF0F0
:105D4000240EDE6E350EDE6E0D0EDE6E34EC9CF033
:105D50008A0EDE6E3C0EDE6E0C0EDE6E34EC9CF0B7
:105D60000B0EDE6E360EDE6EDE6A34EC9CF064EFF7
:105D700031F0400E895DD8A4E1EF2EF0C2ECADF019
:105D80000B0EDE6E360EDE6EDE6A34EC9CF0200EFC
:105D9000DE6E140EDE6E0C0EDE6E34EC9CF0240E05
:105DA000DE6E270EDE6E0D0EDE6E34EC9CF0220EE3
:105DB000DE6E2E0EDE6E0C0EDE6E34EC9CF064EFAA
:105DC00031F0460E895DD8A4F2EF2EF099ECADF0DB
:105DD000A50EDE6E0F0EDE6E010EDE6E34EC9CF054
:105DE00064EF31F0470E895DD8A403EF2FF060EC2B
:105DF000ADF0180EDE6E1E0EDE6E010EDE6E34ECA1
:105E00009CF064EF31F0480E895DD8A459EF2FF073
:105E100060ECADF0EB0EDE6E2A0EDE6EDE6A34EC68
:105E20009CF0010EB65DD8A429EF2FF0DE6A0F0EAC
:105E3000DE6E380EDE6E040EDE6E41ECADF04D0E01
:105E4000DE6E3F0EDE6E060EDE6E34EC9CF057EF1B
:105E50002FF0020EB65DD8A441EF2FF0DE6A0F0ED0
:105E6000DE6E380EDE6E040EDE6E41ECADF0590EC5
:105E7000DE6E450EDE6E060EDE6E34EC9CF057EFE5
:105E80002FF0030EB65DD8A457EF2FF0DE6A0F0E89
:105E9000DE6E380EDE6E040EDE6E41ECADF0550E99
:105EA000DE6E380EDE6E060EDE6E34EC9CF064EFB5
:105EB00031F0490E895DD8A472EF2FF0570EDE6ED7
:105EC000360EDE6E010EDE6E34EC9CF0230EDE6EBE
:105ED0000E0EDE6E030EDE6E34EC9CF060ECADF068
:105EE00064EF31F04A0E895DD8A4A2EF2FF060EC88
:105EF000ADF0550EDE6E380EDE6E010EDE6E34EC49
:105F00009CF0630EDE6E2C0EDE6E030EDE6E34EC45
:105F10009CF0010E8D5DD8A498EF2FF0F50EDE6E8B
:105F20003E0EDE6E060EDE6E34EC9CF0A0EF2FF01F
:105F3000F70EDE6E3E0EDE6E060EDE6E34EC9CF06C
:105F400064EF31F04B0E895DD8A4B3EF2FF060EC15
:105F5000ADF0170EDE6E2F0EDE6E030EDE6E34EC2D
:105F60009CF064EF31F04C0E895DD8A4CCEF2FF09B
:105F700060ECADF0410EDE6E410EDE6E020EDE6EA6
:105F800034EC9CF0110EDE6E180EDE6E030EDE6E2B
:105F900034EC9CF064EF31F04D0E895DD8A4DDEF58
:105FA0002FF060ECADF0160EDE6E250EDE6E010EEB
:105FB000DE6E34EC9CF064EF31F0500E895DD8A4B5
:105FC000EEEF2FF099ECADF0ED0EDE6E1F0EDE6EF3
:105FD000010EDE6E34EC9CF064EF31F0510E895D01
:105FE000D8A406EF30F060ECADF0E90EDE6E1C0ECA
:105FF000DE6EDE6A34EC9CF0ED0EDE6E1F0EDE6EA1
:10600000040EDE6E34EC9CF064EF31F0520E895DCC
:10601000D8A41EEF30F060ECADF0EB0EDE6E2A0E71
:10602000DE6EDE6A34EC9CF0ED0EDE6E1F0EDE6E70
:10603000040EDE6E34EC9CF064EF31F0530E895D9B
:10604000D8A437EF30F060ECADF0890EDE6E200E94
:10605000DE6E010EDE6E34EC9CF0ED0EDE6E1F0E79
:10606000DE6E040EDE6E34EC9CF064EF31F0540E04
:10607000895DD8A466EF30F060ECADF0A30EDE6E63
:10608000110EDE6EDE6A34EC9CF0080EDE6E130E2E
:10609000DE6E030EDE6E34EC9CF0010ECB5DD8A4F8
:1060A0005CEF30F0F50EDE6E390EDE6E060EDE6E43
:1060B00034EC9CF064EF30F0F70EDE6E390EDE6EDD
:1060C000060EDE6E34EC9CF064EF31F0550E895D07
:1060D000D8A48EEF30F060ECADF0020EDE6E240E30
:1060E000DE6E010EDE6E34EC9CF0010E835DD8A4F2
:1060F00084EF30F0F50EDE6E390EDE6E060EDE6ECB
:1061000034EC9CF08CEF30F0F70EDE6E390EDE6E64
:10611000060EDE6E34EC9CF064EF31F0560E895DB5
:10612000D8A4A7EF30F060ECADF0120EDE6E150EC5
:10613000DE6E010EDE6E34EC9CF0ED0EDE6E1F0E98
:10614000DE6E040EDE6E34EC9CF064EF31F0570E20
:10615000895DD8A4C0EF30F060ECADF0470EDE6E84
:10616000240EDE6E010EDE6E34EC9CF0ED0EDE6E63
:106170001F0EDE6E040EDE6E34EC9CF064EF31F028
:10618000580E895DD8A4D9EF30F060ECADF0030E65
:10619000DE6E340EDE6E010EDE6E34EC9CF0ED0E23
:1061A000DE6E1F0EDE6E040EDE6E34EC9CF064EFCD
:1061B00031F05A0E895DD8A41BEF31F01B0EDE6E54
:1061C0000D0EDE6E030EDE6E34EC9CF0630EDE6EA2
:1061D000190EDE6E0A0EDE6E34EC9CF0D70EDE6E0B
:1061E0006E0EDE6E090EDE6E34EC9CF0D90EDE6EA5
:1061F0006E0EDE6E0B0EDE6E34EC9CF04F0EDE6E1D
:106200003F0EDE6E0E0EDE6E34EC9CF0DF0EDE6EA8
:10621000780EDE6E0E0EDE6E34EC9CF0DB0EDE6E63
:106220006D0EDE6E0E0EDE6E34EC9CF0C80E51EC80
:1062300001F064EF31F05B0E895DD8A462EF31F0BC
:106240001B0EDE6E0D0EDE6E030EDE6E34EC9CF069
:10625000E10EDE6E3F0EDE6E0A0EDE6E34EC9CF05A
:10626000D70EDE6E6E0EDE6E080EDE6E34EC9CF027
:10627000D90EDE6E6E0EDE6E0C0EDE6E34EC9CF011
:10628000DF0EDE6E800EDE6E0A0EDE6E34EC9CF0EB
:10629000DB0EDE6E650EDE6E0A0EDE6E34EC9CF0FA
:1062A0004F0EDE6E3F0EDE6E0E0EDE6E34EC9CF098
:1062B000DD0EDE6E650EDE6E0E0EDE6E34EC9CF0D4
:1062C00064EF31F065EF31F012000101349D0001FF
:1062D000888336ECBFF0010E246EF40E52EC01F010
:1062E000206A89C01FF0000E72EC01F00B6E0B5299
:1062F000D8B47FEF31F089C08AF08AEF31F0280EF0
:10630000895DD8A488EF31F089C08AF08AEF31F036
:106310000B0E8A6F3DEC2BF0C20ED76EF70ED66EC9
:10632000F2940901ED6BEC6B010E246EF40E52EC4D
:1063300001F00001820E026E800E096E306A540E6A
:106340002F6E066A0B0E056E4BEC00F0D8A0B3EF73
:1063500031F00901EE6F6C0EEE5D0001D8A4B3EFD1
:1063600031F0B5EF5AF0F2A4BEEF31F0C20ED76EA5
:10637000F70ED66EF2940901EC4BED2B0001030EE3
:106380000901ED5D0001D8A0D2EF31F0D8A4D0EF23
:1063900031F0850E0901EC5D0001D8A0D2EF31F09B
:1063A000ADEC97F00101349B0001956B80A0DEEF0E
:1063B00031F00101348B030E0001956F81A2E6EFED
:1063C00031F00101348B040E0001956F80AAEEEFCD
:1063D00031F00101348B010E0001956F82A2F6EFBE
:1063E00031F00101348B020E0001956F82A0FEEFA7
:1063F00031F00101348B050E0001956FD896010133
:1064000034BBD8860001D8B68FEF32F0810E026E11
:10641000010E096E400E306E200E2F6E066A7B0E46
:10642000056E0B6AD8804BEC00F0D8A082D709EE3D
:10643000D9F00B5023C0EBFF0B2A0B501008F2E1F0
:106440000901E96B0001100E0901E95D0001D8B0F6
:106450008FEF32F009EED9F00901E951EB500B6EE4
:10646000030E0B5C0001D8A48AEF32F0030E090181
:10647000E92509EED9F0EB50EB6F206AEBC91FF06C
:10648000080E21EC02F0EA6F800EEA5D0001D8A44C
:1064900051EF32F0010E956F0101348D00018AEF4A
:1064A00032F0400E0901EA5D0001D8A45FEF32F03E
:1064B000020E956F0101348D00018AEF32F0200E3B
:1064C0000901EA5D0001D8A46DEF32F0030E956F6B
:1064D0000101348D00018AEF32F0100E0901EA5DEE
:1064E0000001D8A47BEF32F0040E956F0101348DCA
:1064F00000018AEF32F0080E0901EA5D0001D8A41C
:1065000089EF32F0050E956F0101348D00018AEF9D
:1065100032F0956B0901E92B0001D8A493D7010E45
:10652000955DD8A4D1EF32F05B0E895DD8A49BEFC6
:1065300032F0ADEF97F05E0EF66E650EF76E2368E3
:10654000232A23500B08D8A0BBEF32F00900F550E6
:106550000900895DF5E123C091F0BBEF32F0630CD7
:106560000C0C150C160C1F0C200C210C220C250CED
:10657000290C4A0C4C0C280E895DD8A4C2EF32F0CD
:10658000B7EF33F0206A89C01FF0000E72EC01F003
:106590000B6E0B52D8B4CFEF32F0B7EF33F0A2EF5F
:1065A00033F0020E955DD8A4F5EF32F089C01FF0EC
:1065B0000A0EE5EC01F0896F89510A0DF3CF31F035
:1065C000F4CF32F00A0E3124896F280E895DD8A4E9
:1065D000ECEF32F0320E896F640E895DD8A4F3EFD0
:1065E00032F00A0E896FA2EF33F0030E955DD8A446
:1065F00018EF33F089C01FF00A0EE5EC01F0896F47
:1066000089510A0DF3CF31F0F4CF32F00A0E315C2C
:10661000896F280E895DD8A410EF33F01E0E896FA4
:106620008953D8A416EF33F05A0E896FA2EF33F0D6
:10663000040E955DD8A458EF33F0892B0E0E895DBA
:10664000D8A425EF33F00A0E896F180E895DD8A4FF
:106650002CEF33F0140E896F2B0E895DD8A433EF25
:1066600033F01E0E896F3B0E895DD8A43AEF33F0EC
:10667000320E896F410E895DD8A441EF33F03C0E94
:10668000896F4E0E895DD8A448EF33F0460E896FAE
:10669000590E895DD8A44FEF33F0500E896F5C0E10
:1066A000895DD8A456EF33F05A0E896FA2EF33F00C
:1066B000050E955DD8A498EF33F08907090E895D22
:1066C000D8A465EF33F00D0E896F130E895DD8A441
:1066D0006CEF33F0170E896F1D0E895DD8A473EF30
:1066E00033F02A0E896F310E895DD8A47AEF33F02A
:1066F0003A0E896F3B0E895DD8A481EF33F0400ECE
:10670000896F450E895DD8A488EF33F04D0E896FEF
:106710004F0E895DD8A48FEF33F0580E896F590E54
:10672000895DD8A496EF33F05B0E896FA2EF33F04A
:106730009553D8A4A0EF33F099EF31F0A2EF33F0E6
:1067400099EF31F036ECBFF03DEC2BF0D89601011B
:1067500034ADD8860001D8B6B3EF33F0C80E51EC93
:1067600001F00101349D000199EF31F012003A0E61
:10677000895DD8A4BEEF33F02DEF34F03E0E895D75
:10678000D8A4C5EF33F02DEF34F03F0E895DD8A4C7
:10679000CCEF33F02DEF34F0400E895DD8A4D3EF69
:1067A00033F02DEF34F0470E895DD8A4DAEF33F0E3
:1067B0002DEF34F04A0E895DD8A4E1EF33F02DEFD0
:1067C00034F04D0E895DD8A4E8EF33F02DEF34F0AE
:1067D000510E895DD8A4EFEF33F02DEF34F0520E57
:1067E000895DD8A4F6EF33F02DEF34F0530E895DB8
:1067F000D8A4FDEF33F02DEF34F0540E895DD8A40A
:1068000004EF34F02DEF34F0550E895DD8A40BEF72
:1068100034F02DEF34F0560E895DD8A412EF34F029
:106820002DEF34F0570E895DD8A419EF34F02DEF19
:1068300034F0580E895DD8A420EF34F02DEF34F0F9
:106840005B0E895DD8A427EF34F02DEF34F09CEC7B
:106850000AF0010EDE6E54EC46F0826BD89688A3E7
:10686000D886D8B636EF34F036ECBFF00A01329154
:106870003A0E0001895DD8A440EF34F0D6EF34F031
:106880003D0E895DD8A447EF34F0D6EF34F03E0ECC
:10689000895DD8A44EEF34F0D6EF34F03F0E895D19
:1068A000D8A455EF34F0D6EF34F0400E895DD8A46B
:1068B0005CEF34F0D6EF34F0430E895DD8A463EF7B
:1068C00034F0D6EF34F0470E895DD8A46AEF34F087
:1068D000D6EF34F0480E895DD8A471EF34F0D6EFCE
:1068E00034F0490E895DD8A478EF34F0D6EF34F057
:1068F0004A0E895DD8A47FEF34F0D6EF34F04B0E0A
:10690000895DD8A486EF34F0D6EF34F04C0E895D63
:10691000D8A48DEF34F0D6EF34F04D0E895DD8A4B5
:1069200094EF34F0D6EF34F0510E895DD8A49BEF8C
:1069300034F0D6EF34F0520E895DD8A4A2EF34F0D3
:10694000D6EF34F0530E895DD8A4A9EF34F0D6EF1A
:1069500034F0540E895DD8A4B0EF34F0D6EF34F0A3
:10696000550E895DD8A4B7EF34F0D6EF34F0560E4B
:10697000895DD8A4BEEF34F0D6EF34F0570E895DB0
:10698000D8A4C5EF34F0D6EF34F0580E895DD8A402
:10699000CCEF34F0D6EF34F05B0E895DD8A4D3EFA2
:1069A00034F0D5EF34F00A0132810001D8960A01A3
:1069B00032A1D8860001D8B688EF35F08B53D8A421
:1069C000E6EF34F089C08BF0F2EF34F08C53D8A4AA
:1069D000F2EF34F08B51895DD8B4F2EF34F089C016
:1069E0008CF08885010E8D5DD8A488EF35F0D8969F
:1069F00088A5D886D8B688EF35F089C08EF004EE29
:106A00001AF0D89001012135E926000EEA22EECFD6
:106A10000BF0EFCF0CF0000192510B5C93510C582E
:106A2000D8A02CEF35F004EE1AF0D89001012135F2
:106A3000E926000EEA22EECF0BF0EFCF0CF00001BA
:106A400092510B5C0A01306F000193510C580A01FE
:106A5000316F000142EF35F004EE1AF0D8900101D9
:106A60002135E926000EEA22EECF0BF0EFCF0CF035
:106A70000B500001925D0A01306F0C5000019359D8
:106A80000A01316F00010A0131530001D8A452EF0D
:106A900035F05B0E0A01305D0001D8B052EF35F0E1
:106AA0008BC089F0010E0A01315D0001D8A065EFAD
:106AB00035F0D8A463EF35F00E0E0A01305D000109
:106AC000D8A065EF35F08BC089F00A013153000181
:106AD000D8A472EF35F05B0E0A01305D0001D8A03A
:106AE0007EEF35F0010E0A01315D0E0ED8B4305D37
:106AF0000001D8B07EEF35F08CC089F089518E5DF1
:106B0000D8B486EF35F0888336ECBFF088EF35F0E7
:106B10000B0E895DD8A47EEF36F0BFEC84F0010E39
:106B2000955DD8A49CEF35F0D89688B3D886D8B6B2
:106B30009CEF35F065EF31F0050E955DD8A4AFEF11
:106B400035F0D89688B3D886D8B6AFEF35F08AC07E
:106B50002FFA89C08AF02FCA89F0888308D6040EDC
:106B6000955DD8A4B6EF35F088EC64F0D89688A38C
:106B7000D886D8B6C6EF35F00101349F270EDE6EF9
:106B8000180EDE6EDE6A000134EC9CF079ECAFF09A
:106B900003EE1AF0D89001012135E926000EEA2211
:106BA000EECF0BF0EFCF0CF00BC0DEFF0CC0DEFF22
:106BB0000001F1EC74F0FF0EDB50DD520101348F67
:106BC000E8A0349FD89634AFD8860001D8B632EF0B
:106BD00036F0010121530001D8B415EF36F003EE71
:106BE0001AF0D89001012135E926000EEA22EECFF5
:106BF0000BF0EFCF0CF00BC0DEFF0CC0DEFF210569
:106C00000F6E03EE1AF0D8900F34E926000EEA2238
:106C1000EECF0BF0EFCF0CF00BC0DEFF0CC0DEFFB1
:106C20000001EFEC75F030EF36F003EE1AF0D8907B
:106C300001012135E926000EEA22EECF0BF0EFCF5D
:106C40000CF00BC0DEFF0CC0DEFF18C40BF019C443
:106C50000CF00BC0DEFF0CC0DEFF0001EFEC75F0A6
:106C600079EF36F0010121530001D8B45EEF36F020
:106C700003EE1AF0D89001012135E926000EEA2230
:106C8000EECF0BF0EFCF0CF00BC0DEFF0CC0DEFF41
:106C900021050F6E03EE1AF0D8900F34E926000E8E
:106CA000EA22EECF0BF0EFCF0CF00BC0DEFF0CC0F2
:106CB000DEFF0001B7EC75F079EF36F003EE1AF065
:106CC000D89001012135E926000EEA22EECF0BF023
:106CD000EFCF0CF00BC0DEFF0CC0DEFF18C40BF0D2
:106CE00019C40CF00BC0DEFF0CC0DEFF0001B7ECD6
:106CF00075F08893B7EF33F052EF46F00C0E895DD4
:106D0000D8A48DEF37F0BFEC84F0010E955DD8A4C8
:106D100094EF36F0D89688B3D886D8B692EF36F08E
:106D200065EF31F0AAEF36F0020E955DD8A4A0EF22
:106D300036F036ECBFF0888354EF96F0AAEF36F0C9
:106D4000030E955DD8A4AAEF36F036ECBFF0888329
:106D500054EF96F0040E955DD8A4B1EF36F088ECB0
:106D600064F0050E955DD8A4C5EF36F0D89688B3CB
:106D7000D886D8B6C5EF36F08AC02FFA89C08AF017
:106D80002FCA89F08883B7EF33F0D89688A3D886C6
:106D9000D8B6D5EF36F00101349F250EDE6E180E01
:106DA000DE6EDE6A000134EC9CF079ECAFF002EEAE
:106DB0001AF0D89001012135E926000EEA22EECF23
:106DC0000BF0EFCF0CF00BC0DEFF0CC0DEFF0001BC
:106DD000F1EC74F0FF0EDB50DD520101348FE8A0BE
:106DE000349FD89634AFD8860001D8B641EF37F03B
:106DF000010121530001D8B424EF37F002EE1AF05C
:106E0000D89001012135E926000EEA22EECF0BF0E1
:106E1000EFCF0CF00BC0DEFF0CC0DEFF21050F6EC4
:106E200002EE1AF0D8900F34E926000EEA22EECFD7
:106E30000BF0EFCF0CF00BC0DEFF0CC0DEFF00014B
:106E4000EFEC75F03FEF37F002EE1AF0D890010149
:106E50002135E926000EEA22EECF0BF0EFCF0CF041
:106E60000BC0DEFF0CC0DEFF18C30BF019C30CF023
:106E70000BC0DEFF0CC0DEFF0001EFEC75F088EF09
:106E800037F0010121530001D8B46DEF37F002EE65
:106E90001AF0D89001012135E926000EEA22EECF42
:106EA0000BF0EFCF0CF00BC0DEFF0CC0DEFF2105B6
:106EB0000F6E02EE1AF0D8900F34E926000EEA2287
:106EC000EECF0BF0EFCF0CF00BC0DEFF0CC0DEFFFF
:106ED0000001B7EC75F088EF37F002EE1AF0D890A9
:106EE00001012135E926000EEA22EECF0BF0EFCFAB
:106EF0000CF00BC0DEFF0CC0DEFF18C30BF019C393
:106F00000CF00BC0DEFF0CC0DEFF0001B7EC75F02B
:106F10008893B7EF33F052EF46F00D0E895DD8A499
:106F2000EFEF37F0BFEC84F0010E955DD8A4A1EF30
:106F300037F0D89688B3D886D8B6A1EF37F065EF8A
:106F400031F0050E955DD8A4B5EF37F0D89688B32B
:106F5000D886D8B6B5EF37F08AC02FFA89C08AF044
:106F60002FCA89F08883B7EF33F0040E955DD8A45B
:106F7000BCEF37F088EC64F0D89688A3D886D8B6F2
:106F8000D2EF37F0230EDE6E0E0EDE6E010EDE6ED9
:106F900034EC9CF03D0EDE6E860EDE6E060EDE6E6E
:106FA00034EC9CF004EE1AF0D89001012135E9266A
:106FB000000EEA22EECF0BF0EFCF0CF00BC0DEFF9D
:106FC0000CC0DEFFDE6A010EDE6E0A0EDE6E000110
:106FD00027EC76F08893B7EF33F052EF46F0150EBA
:106FE000895DD8A47FEF38F0BFEC84F0010E955D89
:106FF000D8A405EF38F0D89688B3D886D8B603EF72
:1070000038F065EF31F01BEF38F0020E955DD8A433
:1070100011EF38F036ECBFF0888354EF96F01BEF99
:1070200038F0030E955DD8A41BEF38F036ECBFF0B6
:10703000888354EF96F0040E955DD8A422EF38F0C3
:1070400088EC64F0050E955DD8A436EF38F0D8963C
:1070500088B3D886D8B636EF38F08AC02FFA89C000
:107060008AF02FCA89F08883B7EF33F0D89688A3C7
:10707000D886D8B64AEF38F0CD0EDE6EDE6ADE6A0C
:1070800034EC9CF03F0EDE6E860EDE6E090EDE6E78
:1070900034EC9CF002EE1AF0D89001012135E9267B
:1070A000000EEA22EECF0BF0EFCF0CF00BC0DEFFAC
:1070B0000CC0DEFF010EDE6EDE6A140EDE6E000115
:1070C00027EC76F004EE1AF0D89001012135E9267C
:1070D000000EEA22EECF0BF0EFCF0CF00BC0DEFF7C
:1070E0000CC0DEFFDE6A010EDE6E0A0EDE6E0001EF
:1070F00027EC76F08893B7EF33F052EF46F0160E98
:10710000895DD8A40FEF39F0BFEC84F0010E955DD6
:10711000D8A495EF38F0D89688B3D886D8B693EF30
:1071200038F065EF31F0ABEF38F0020E955DD8A482
:10713000A1EF38F036ECBFF0888354EF96F0ABEF58
:1071400038F0030E955DD8A4ABEF38F036ECBFF005
:10715000888354EF96F0040E955DD8A4B2EF38F012
:1071600088EC64F0050E955DD8A4C6EF38F0D8968B
:1071700088B3D886D8B6C6EF38F08AC02FFA89C04F
:107180008AF02FCA89F08883B7EF33F0D89688A3A6
:10719000D886D8B6DBEF38F0D10EDE6E050EDE6E87
:1071A000DE6A34EC9CF0CF0EDE6E900EDE6E090EC1
:1071B000DE6E34EC9CF003EE1AF0D890010121351C
:1071C000E926000EEA22EECF0BF0EFCF0CF00BC059
:1071D000DEFF0CC0DEFF010EDE6EDE6A140EDE6E18
:1071E000000127EC76F002EE1AF0D890010121356B
:1071F000E926000EEA22EECF0BF0EFCF0CF00BC029
:10720000DEFF0CC0DEFFDE6ADE6A0C0EDE6E000101
:1072100027EC76F08893B7EF33F052EF46F0170E75
:10722000895DD8A488EF39F0BFEC84F0010E955D3C
:10723000D8A423EF39F0D89688B3D886D8B623EFF0
:1072400039F065EF31F0050E955DD8A437EF39F0D0
:10725000D89688B3D886D8B637EF39F08AC02FFAD7
:1072600089C08AF02FCA89F08883B7EF33F0040E03
:10727000955DD8A43EEF39F088EC64F0D89688A3E9
:10728000D886D8B653EF39F0D10EDE6E050EDE6E1D
:10729000DE6A34EC9CF03F0EDE6E860EDE6E090E6A
:1072A000DE6E34EC9CF003EE1AF0D890010121352B
:1072B000E926000EEA22EECF0BF0EFCF0CF00BC068
:1072C000DEFF0CC0DEFF010EDE6EDE6A140EDE6E27
:1072D000000127EC76F004EE1AF0D8900101213578
:1072E000E926000EEA22EECF0BF0EFCF0CF00BC038
:1072F000DEFF0CC0DEFFDE6A010EDE6E0A0EDE6E01
:10730000000127EC76F08893B7EF33F052EF46F0A8
:107310001F0E895DD8A404EF3AF0BFEC84F0010E93
:10732000955DD8A49EEF39F0D89688B3D886D8B6A4
:107330009CEF39F065EF31F0B4EF39F0020E955D56
:10734000D8A4AAEF39F036ECBFF0888354EF96F05A
:10735000B4EF39F0030E955DD8A4B4EF39F036ECF4
:10736000BFF0888354EF96F0040E955DD8A4BBEF70
:1073700039F088EC64F0050E955DD8A4CFEF39F0B4
:10738000D89688B3D886D8B6CFEF39F08AC02FFA0E
:1073900089C08AF02FCA89F08883B7EF33F0D89676
:1073A00088A3D886D8B6E3EF39F0CD0EDE6EDE6A5C
:1073B000DE6A34EC9CF0CF0EDE6E900EDE6E080EB0
:1073C000DE6E34EC9CF002EE1AF0D890010121350B
:1073D000E926000EEA22EECF0BF0EFCF0CF00BC047
:1073E000DEFF0CC0DEFF010EDE6EDE6A140EDE6E06
:1073F000000127EC76F0020EDE6EE2ECB0F088932E
:10740000B7EF33F052EF46F0200E895DD8A480EF3D
:107410003AF0BFEC84F0010E955DD8A41AEF3AF073
:10742000D89688B3D886D8B618EF3AF065EF31F021
:1074300030EF3AF0020E955DD8A426EF3AF036EC24
:10744000BFF0888354EF96F030EF3AF0030E955D6D
:10745000D8A430EF3AF036ECBFF0888354EF96F0C2
:10746000040E955DD8A437EF3AF088EC64F0050E71
:10747000955DD8A44BEF3AF0D89688B3D886D8B6A5
:107480004BEF3AF08AC02FFA89C08AF02FCA89F0F0
:107490008883B7EF33F0D89688A3D886D8B65FEF45
:1074A0003AF0CD0EDE6EDE6ADE6A34EC9CF0D30E6E
:1074B000DE6E8E0EDE6E090EDE6E34EC9CF002EE99
:1074C0001AF0D89001012135E926000EEA22EECF0C
:1074D0000BF0EFCF0CF00BC0DEFF0CC0DEFF010E97
:1074E000DE6EDE6A140EDE6E000127EC76F0010E11
:1074F000DE6EE2ECB0F08893B7EF33F052EF46F077
:10750000210E895DD8A4FCEF3AF0BFEC84F0010EA7
:10751000955DD8A496EF3AF0D89688B3D886D8B6B9
:1075200094EF3AF065EF31F0ACEF3AF0020E955D72
:10753000D8A4A2EF3AF036ECBFF0888354EF96F06F
:10754000ACEF3AF0030E955DD8A4ACEF3AF036EC10
:10755000BFF0888354EF96F0040E955DD8A4B3EF86
:107560003AF088EC64F0050E955DD8A4C7EF3AF0C8
:10757000D89688B3D886D8B6C7EF3AF08AC02FFA23
:1075800089C08AF02FCA89F08883B7EF33F0D89684
:1075900088A3D886D8B6DBEF3AF0CD0EDE6EDE6A71
:1075A000DE6A34EC9CF03F0EDE6E860EDE6E090E57
:1075B000DE6E34EC9CF002EE1AF0D8900101213519
:1075C000E926000EEA22EECF0BF0EFCF0CF00BC055
:1075D000DEFF0CC0DEFF010EDE6EDE6A140EDE6E14
:1075E000000127EC76F0030EDE6EE2ECB0F088933B
:1075F000B7EF33F052EF46F0220E895DD8A484EF46
:107600003BF0BFEC84F0010E955DD8A412EF3BF087
:10761000D89688B3D886D8B610EF3BF065EF31F036
:107620003DEF3BF0020E955DD8A41EEF3BF036EC2B
:10763000BFF0888354EF96F03DEF3BF0030E955D6D
:10764000D8A42AEF3BF036ECBFF0888354EF96F0D5
:107650003DEF3BF0040E955DD8A43CEF3BF08881F4
:1076600004EE1AF0D89001012135E926000EEA2235
:10767000EECF86F0EFCF87F00001050E955DD8A420
:1076800051EF3BF0D89688B3D886D8B651EF3BF08F
:107690008AC02FFA89C08AF02FCA89F08883B7EF91
:1076A00033F0D89688A3D886D8B665EF3BF0CD0ED8
:1076B000DE6EDE6ADE6A34EC9CF0490EDE6E640E2D
:1076C000DE6E0E0EDE6E34EC9CF002EE1AF0D890F8
:1076D00001012135E926000EEA22EECF0BF0EFCFB3
:1076E0000CF00BC0DEFF0CC0DEFF010EDE6EDE6AAA
:1076F000140EDE6E000127EC76F059EC68F08893EA
:10770000B7EF33F052EF46F0230E895DD8A4E9EFCE
:107710003BF0BFEC84F0010E955DD8A498EF3BF0F0
:10772000D89688B3D886D8B698EF3BF065EF31F09D
:10773000050E955DD8A4ACEF3BF0D89688B3D886FB
:10774000D8B6ACEF3BF08AC02FFA89C08AF02FCAB6
:1077500089F08883B7EF33F0040E955DD8A4B3EFBA
:107760003BF088EC64F0D89688A3D886D8B6C8EFEA
:107770003BF0D10EDE6E050EDE6EDE6A34EC9CF060
:10778000D30EDE6E8E0EDE6E090EDE6E34EC9CF0D5
:1077900003EE1AF0D89001012135E926000EEA2205
:1077A000EECF0BF0EFCF0CF00BC0DEFF0CC0DEFF16
:1077B000010EDE6EDE6A140EDE6E000127EC76F03E
:1077C000010EDE6EE2ECB0F08893B7EF33F052EFCB
:1077D00046F0240E895DD8A44EEF3CF0BFEC84F057
:1077E000010E955DD8A4FDEF3BF0D89688B3D886FE
:1077F000D8B6FDEF3BF065EF31F0050E955DD8A4EE
:1078000011EF3CF0D89688B3D886D8B611EF3CF08B
:107810008AC02FFA89C08AF02FCA89F08883B7EF0F
:1078200033F0040E955DD8A418EF3CF088EC64F0BA
:10783000D89688A3D886D8B62DEF3CF0D10EDE6E50
:10784000050EDE6EDE6A34EC9CF03F0EDE6E860EB8
:10785000DE6E090EDE6E34EC9CF003EE1AF0D8906A
:1078600001012135E926000EEA22EECF0BF0EFCF21
:107870000CF00BC0DEFF0CC0DEFF010EDE6EDE6A18
:10788000140EDE6E000127EC76F0030EDE6EE2ECE5
:10789000B0F08893B7EF33F052EF46F0250E895DD4
:1078A000D8A4CBEF3CF0BFEC84F0010E955DD8A4DA
:1078B00064EF3CF0D89688B3D886D8B662EF3CF037
:1078C00065EF31F07AEF3CF0020E955DD8A470EFD1
:1078D0003CF036ECBFF0888354EF96F07AEF3CF042
:1078E000030E955DD8A47AEF3CF036ECBFF08883A8
:1078F00054EF96F0040E955DD8A481EF3CF088EC2F
:1079000064F0050E955DD8A495EF3CF0D89688B349
:10791000D886D8B695EF3CF08AC02FFA89C08AF095
:107920002FCA89F08883B7EF33F0D89688A3D8861A
:10793000D8B6AAEF3CF0D10EDE6E050EDE6EDE6A22
:1079400034EC9CF0CF0EDE6E900EDE6E080EDE6E16
:1079500034EC9CF003EE1AF0D89001012135E926B1
:10796000000EEA22EECF0BF0EFCF0CF00BC0DEFFE3
:107970000CC0DEFF010EDE6EDE6A140EDE6E00014C
:1079800027EC76F0020EDE6EE2ECB0F08893B7EFF3
:1079900033F052EF46F0260E895DD8A43AEF3DF061
:1079A000BFEC84F0010E955DD8A4DFEF3CF0D896D3
:1079B00088B3D886D8B6DFEF3CF065EF31F0040E1F
:1079C000955DD8A4F1EF3CF0888104EE1AF0D890D0
:1079D00001012135E926000EEA22EECF86F0EFCF35
:1079E00087F00001050E955DD8A406EF3DF0D8960E
:1079F00088B3D886D8B606EF3DF08AC02FFA89C082
:107A00008AF02FCA89F08883B7EF33F0D89688A31D
:107A1000D886D8B61BEF3DF0D10EDE6E050EDE6EB9
:107A2000DE6A34EC9CF0490EDE6E640EDE6E0E0EE5
:107A3000DE6E34EC9CF003EE1AF0D8900101213593
:107A4000E926000EEA22EECF0BF0EFCF0CF00BC0D0
:107A5000DEFF0CC0DEFF010EDE6EDE6A140EDE6E8F
:107A6000000127EC76F059EC68F08893B7EF33F01B
:107A700052EF46F0270E895DD8A4A0EF3DF0BFEC91
:107A800084F0010E955DD8A44EEF3DF0D89688B3F2
:107A9000D886D8B64EEF3DF065EF31F0050E955D16
:107AA000D8A462EF3DF0D89688B3D886D8B662EFF6
:107AB0003DF08AC02FFA89C08AF02FCA89F08883E6
:107AC000B7EF33F0040E955DD8A469EF3DF088EC74
:107AD00064F0D89688A3D886D8B67EEF3DF03D0EE8
:107AE000DE6E860EDE6EDE6A34EC9CF03F0EDE6EDD
:107AF000860EDE6E090EDE6E34EC9CF004EE1AF09B
:107B0000D89001012135E926000EEA22EECF0BF0D4
:107B1000EFCF0CF00BC0DEFF0CC0DEFF010EDE6EFF
:107B2000010EDE6E0A0EDE6E000127EC76F0030E0B
:107B3000DE6EE2ECB0F08893B7EF33F052EF46F030
:107B4000280E895DD8A406EF3EF0BFEC84F0010E4C
:107B5000955DD8A4B4EF3DF0D89688B3D886D8B652
:107B6000B4EF3DF065EF31F0050E955DD8A4C8EF98
:107B70003DF0D89688B3D886D8B6C8EF3DF08AC015
:107B80002FFA89C08AF02FCA89F08883B7EF33F0C3
:107B9000040E955DD8A4CFEF3DF088EC64F0D89644
:107BA00088A3D886D8B6E4EF3DF03D0EDE6E860E93
:107BB000DE6EDE6A34EC9CF0D30EDE6E8E0EDE6E70
:107BC000090EDE6E34EC9CF004EE1AF0D890010140
:107BD0002135E926000EEA22EECF0BF0EFCF0CF0B4
:107BE0000BC0DEFF0CC0DEFF010EDE6E010EDE6E8E
:107BF0000A0EDE6E000127EC76F0010EDE6EE2EC7E
:107C0000B0F08893B7EF33F052EF46F0290E895D5C
:107C1000D8A484EF3EF0BFEC84F0010E955DD8A4AB
:107C20001CEF3EF0D89688B3D886D8B61AEF3EF04F
:107C300065EF31F032EF3EF0020E955DD8A428EFEB
:107C40003EF036ECBFF0888354EF96F032EF3EF012
:107C5000030E955DD8A432EF3EF036ECBFF088837A
:107C600054EF96F0040E955DD8A439EF3EF088EC01
:107C700064F0050E955DD8A44DEF3EF0D89688B31C
:107C8000D886D8B64DEF3EF08AC02FFA89C08AF068
:107C90002FCA89F08883B7EF33F0D89688A3D886A7
:107CA000D8B662EF3EF03D0EDE6E860EDE6EDE6A08
:107CB00034EC9CF0CF0EDE6E900EDE6E080EDE6EA3
:107CC00034EC9CF004EE1AF0D89001012135E9263D
:107CD000000EEA22EECF0BF0EFCF0CF00BC0DEFF70
:107CE0000CC0DEFF010EDE6E010EDE6E0A0EDE6ED1
:107CF000000127EC76F0020EDE6EE2ECB0F0889325
:107D0000B7EF33F052EF46F02A0E895DD8A4F4EFB6
:107D10003EF0BFEC84F0010E955DD8A498EF3EF0E4
:107D2000D89688B3D886D8B698EF3EF065EF31F094
:107D3000040E955DD8A4AAEF3EF0888104EE1AF0F7
:107D4000D89001012135E926000EEA22EECF86F017
:107D5000EFCF87F00001050E955DD8A4BFEF3EF090
:107D6000D89688B3D886D8B6BFEF3EF08AC02FFA2F
:107D700089C08AF02FCA89F08883B7EF33F0D8968C
:107D800088A3D886D8B6D4EF3EF03D0EDE6E860EC0
:107D9000DE6EDE6A34EC9CF0490EDE6E640EDE6E42
:107DA0000E0EDE6E34EC9CF004EE1AF0D890010159
:107DB0002135E926000EEA22EECF0BF0EFCF0CF0D2
:107DC0000BC0DEFF0CC0DEFF010EDE6E010EDE6EAC
:107DD0000A0EDE6E000127EC76F059EC68F088930D
:107DE000B7EF33F052EF46F0330E895DD8A47CEF45
:107DF0003FF0BFEC84F0010E955DD8A40AEF3FF090
:107E0000D89688B3D886D8B608EF3FF065EF31F042
:107E100036EF3FF0020E955DD8A416EF3FF036EC3A
:107E2000BFF08883BDEF95F036EF3FF0030E955D10
:107E3000D8A422EF3FF036ECBFF08883BDEF95F079
:107E400036EF3FF0050E955DD8A436EF3FF0D8969B
:107E500088B3D886D8B636EF3FF08AC02FFA89C0EB
:107E60008AF02FCA89F08883B7EF33F0040E955D4E
:107E7000D8A43DEF3FF088EC64F0D89688A3D8866C
:107E8000D8B673EF3FF03D0EDE6E860EDE6EDE6A14
:107E900034EC9CF03D0EDE6E7D0EDE6E090EDE6E65
:107EA00034EC9CF0430EDE6E8B0EDE6E090EDE6E41
:107EB00034EC9CF0010E0101425D0001D8A46BEF8F
:107EC0003FF06D0EDE6E7D0EDE6E0B0EDE6E34EC60
:107ED0009CF073EF3FF06B0EDE6E7D0EDE6E0B0ED0
:107EE000DE6E34EC9CF0330EDE6E02EC6FF08893A5
:107EF000B7EF33F052EF46F0340E895DD8A403EFAC
:107F000040F0BFEC84F0010E955DD8A492EF3FF0F5
:107F1000D89688B3D886D8B690EF3FF065EF31F0A9
:107F2000BEEF3FF0020E955DD8A49EEF3FF036EC19
:107F3000BFF08883BDEF95F0BEEF3FF0030E955D77
:107F4000D8A4AAEF3FF036ECBFF08883BDEF95F0E0
:107F5000BEEF3FF0050E955DD8A4BEEF3FF0D8967A
:107F600088B3D886D8B6BEEF3FF08AC02FFA89C052
:107F70008AF02FCA89F08883B7EF33F0040E955D3D
:107F8000D8A4C5EF3FF088EC64F0D89688A3D886D3
:107F9000D8B6FAEF3FF03D0EDE6E7D0EDE6E090EB6
:107FA000DE6E34EC9CF0430EDE6E8B0EDE6E090E40
:107FB000DE6E34EC9CF0D10EDE6EDE6ADE6A34ECEE
:107FC0009CF0010E0101425D0001D8A4F2EF3FF0E8
:107FD0006D0EDE6E7D0EDE6E0B0EDE6E34EC9CF0F2
:107FE000FAEF3FF06B0EDE6E7D0EDE6E0B0EDE6E78
:107FF00034EC9CF0340EDE6E02EC6FF08893B7EF39
:1080000033F052EF46F0350E895DD8A48AEF40F088
:10801000BFEC84F0010E955DD8A419EF40F0D8961E
:1080200088B3D886D8B617EF40F065EF31F045EF4A
:1080300040F0020E955DD8A425EF40F036ECBFF07D
:108040008883BDEF95F045EF40F0030E955DD8A411
:1080500031EF40F036ECBFF08883BDEF95F045EF8F
:1080600040F0050E955DD8A445EF40F0D89688B352
:10807000D886D8B645EF40F08AC02FFA89C08AF07A
:108080002FCA89F08883B7EF33F0040E955DD8A42A
:108090004CEF40F088EC64F0D89688A3D886D8B628
:1080A00081EF40F03D0EDE6E7D0EDE6E090EDE6E5F
:1080B00034EC9CF0430EDE6E8B0EDE6E090EDE6E2F
:1080C00034EC9CF0CD0EDE6EDE6ADE6A34EC9CF0A1
:1080D000010E0101425D0001D8A479EF40F06D0E60
:1080E000DE6E7D0EDE6E0B0EDE6E34EC9CF081EFEC
:1080F00040F06B0EDE6E7D0EDE6E0B0EDE6E34EC2F
:108100009CF0350EDE6E02EC6FF08893B7EF33F023
:1081100052EF46F0360E895DD8A40BEF41F0BFEC6C
:1081200084F0010E955DD8A4A0EF40F0D89688B3F6
:10813000D886D8B69EEF40F065EF31F0CCEF40F036
:10814000020E955DD8A4ACEF40F036ECBFF088830A
:10815000BDEF95F0CCEF40F0030E955DD8A4B8EFDD
:1081600040F036ECBFF08883BDEF95F0CCEF40F0E7
:10817000050E955DD8A4CCEF40F0D89688B3D8868C
:10818000D8B6CCEF40F08AC02FFA89C08AF02FCA47
:1081900089F08883B7EF33F0040E955DD8A4D3EF50
:1081A00040F088EC64F0D89688A3D886D8B602EF61
:1081B00041F03D0EDE6E7D0EDE6E090EDE6E34EC9D
:1081C0009CF0430EDE6E8B0EDE6E090EDE6E34EC1E
:1081D0009CF0010E0101425D0001D8A4FAEF40F0CD
:1081E0006D0EDE6E7D0EDE6E0B0EDE6E34EC9CF0E0
:1081F00002EF41F06B0EDE6E7D0EDE6E0B0EDE6E5C
:1082000034EC9CF0360EDE6E02EC6FF08893B7EF24
:1082100033F052EF46F0370E895DD8A48CEF41F071
:10822000BFEC84F0010E955DD8A421EF41F0D89603
:1082300088B3D886D8B61FEF41F065EF31F04DEF27
:1082400041F0020E955DD8A42DEF41F036ECBFF061
:108250008883BDEF95F04DEF41F0030E955DD8A4F6
:1082600039EF41F036ECBFF08883BDEF95F04DEF6C
:1082700041F0050E955DD8A44DEF41F0D89688B336
:10828000D886D8B64DEF41F08AC02FFA89C08AF05F
:108290002FCA89F08883B7EF33F0040E955DD8A418
:1082A00054EF41F088EC64F0D89688A3D886D8B60D
:1082B00083EF41F03D0EDE6E7D0EDE6E090EDE6E4A
:1082C00034EC9CF0430EDE6E8B0EDE6E090EDE6E1D
:1082D00034EC9CF0010E0101425D0001D8A47BEF5B
:1082E00041F06D0EDE6E7D0EDE6E0B0EDE6E34EC3A
:1082F0009CF083EF41F06B0EDE6E7D0EDE6E0B0E9A
:10830000DE6E34EC9CF0370EDE6E02EC6FF088937C
:10831000B7EF33F052EF46F0380E895DD8A4E4EFA2
:1083200041F0BFEC84F0010E955DD8A4A2EF41F0BE
:10833000D89688B3D886D8B6A0EF41F065EF31F073
:10834000CEEF41F0020E955DD8A4AEEF41F036ECD1
:10835000BFF08883BDEF95F0CEEF41F0030E955D41
:10836000D8A4BAEF41F036ECBFF08883BDEF95F0AA
:10837000CEEF41F0050E955DD8A4CEEF41F0D89632
:1083800088B3D886D8B6CEEF41F08AC02FFA89C01C
:108390008AF02FCA89F08883B7EF33F0040E955D19
:1083A000D8A4D5EF41F088EC64F0D89688A3D8869D
:1083B000D8B6DBEF41F0380EDE6E02EC6FF088933A
:1083C000B7EF33F052EF46F0390E895DD8A453EF82
:1083D00042F0BFEC84F0010E955DD8A4FAEF41F0B5
:1083E000D89688B3D886D8B6F8EF41F065EF31F06B
:1083F00026EF42F0020E955DD8A406EF42F036EC6F
:10840000BFF08883BDEF95F026EF42F0030E955D37
:10841000D8A412EF42F036ECBFF08883BDEF95F0A0
:1084200026EF42F0050E955DD8A426EF42F0D896CF
:1084300088B3D886D8B626EF42F08AC02FFA89C012
:108440008AF02FCA89F08883B7EF33F0040E955D68
:10845000D8A42DEF42F088EC64F0D89688A3D88693
:10846000D8B64AEF42F03D0EDE6E860EDE6EDE6A54
:1084700034EC9CF0650EDE6E420EDE6E0E0EDE6E8D
:1084800034EC9CF0670EDE6E500EDE6E0E0EDE6E6D
:1084900034EC9CF0390EDE6E02EC6FF08893B7EF8F
:1084A00033F052EF46F03A0E895DD8A45CEF42F00B
:1084B000BAEF91F052EF46F03D0E895DD8A4E8EF97
:1084C00042F0BFEC84F0010E955DD8A472EF42F04B
:1084D000EAECC2F0D89688B3D886D8B672EF42F0EC
:1084E00065EF31F0020E955DD8A47EEF42F08883EF
:1084F000D3ECBEF02DEC8DF0D3ECBEF0030E955D09
:10850000D8A48AEF42F08883D3ECBEF02DEC8DF036
:10851000D3ECBEF0050E955DD8A49EEF42F0D89640
:1085200088B3D886D8B69EEF42F08AC02FFA89C0A9
:108530008AF02FCA89F08883B7EF33F0040E955D77
:10854000D8A4A5EF42F088EC64F0D89688A3D8862A
:10855000D8B6E1EF42F0D89688BBD886D8B6BBEF44
:1085600042F036ECBFF0A3EC68F0B36BB26BB56BC6
:10857000B46BE1EF42F0890EDE6EDE6ADE6A34EC47
:108580009CF08A0EDE6E0F0EDE6E030EDE6E34EC95
:108590009CF0D70EDE6E840EDE6E020EDE6E34ECC4
:1085A0009CF0D90EDE6E840EDE6E060EDE6E34ECAE
:1085B0009CF01A0EDE6E790EDE6E040EDE6E34EC6A
:1085C0009CF0E4EC6AF08893B7EF33F052EF46F09A
:1085D0003E0E895DD8A409EF43F0D89688A3D886CB
:1085E000D8B601EF43F0D89688BBD886D8B601EF4D
:1085F00043F036ECBFF0A3EC68F0B36BB26BB56B35
:10860000B46B010EDE6EECEC7EF081EF83F052EF86
:1086100046F03F0E895DD8A426EF43F0D89688A394
:10862000D886D8B622EF43F0D89688BBD886D8B67D
:1086300022EF43F036ECBFF0A3EC68F0B36BB26B03
:10864000B56BB46B0FEF82F052EF46F0400E895DD0
:10865000D8A447EF43F0D89688A3D886D8B63FEF82
:1086600043F0D89688BBD886D8B63FEF43F036ECB7
:10867000BFF0A3EC68F0B36BB26BB56BB46B010EDB
:10868000DE6EECEC7EF0D6EF80F052EF46F0470E57
:10869000895DD8A486EF43F0BFEC84F0180EDE6E3F
:1086A000DE6ADE6A34EC9CF0D70EDE6E840EDE6E7F
:1086B000030EDE6E34EC9CF0D90EDE6E840EDE6EA0
:1086C000070EDE6E34EC9CF01C0EDE6E7A0EDE6E53
:1086D000050EDE6E34EC9CF0010E955DD8A479EFAA
:1086E00043F0D89688B3D886D8B679EF43F065EFD3
:1086F00031F0D89688A3D886D8B682EF43F0DE6AE8
:10870000ECEC7EF087EF7FF052EF46F0480E895D8B
:10871000D8A49EEF43F0BFEC84F0010E955DD8A481
:108720009AEF43F0D89688B3D886D8B69AEF43F03C
:1087300065EF31F052EF98F052EF46F0490E895D47
:10874000D8A468EF44F0D89688A3D886D8B6B2EFFC
:1087500043F0010E0101446F680E436F010E466F36
:10876000680E456F0001BFEC84F0010E955DD8A442
:10877000C4EF43F0D89688B3D886D8B6C2EF43F09A
:1087800065EF31F040EF44F0020E955DD8A414EF90
:1087900044F004EE1AF0D89001012135E926000ECC
:1087A000EA22EECF43F1EFCF44F1000136ECBFF007
:1087B0005B0EDE6E360EDE6EDE6A34EC9CF05B0E17
:1087C000DE6E360EDE6E040EDE6E34EC9CF05B0E5A
:1087D000DE6E360EDE6E090EDE6E34EC9CF05B0E45
:1087E000DE6E360EDE6E0E0EDE6E34EC9CF00A018E
:1087F000336B0001150E0A01335D0001D8B010EF94
:1088000044F0DBECC2F0C80E51EC01F0EAECC2F02F
:10881000C80E51EC01F00A01332B0001D8A4E9D7AE
:1088200036ECBFF040EF44F0030E955DD8A434EF72
:1088300044F001014451010A680ED8B44319000103
:10884000D8B432EF44F004EE1AF0D890010121358B
:10885000E926000EEA22EECF45F1EFCF46F1000106
:1088600036ECBFF040EF44F0040E955DD8A43BEF2A
:1088700044F040EF44F0050E955DD8A440EF44F07D
:108880008CEC85F03F0EDE6E860EDE6E090EDE6E1F
:1088900034EC9CF0888304EE1AF0D8900101213565
:1088A000E926000EEA22EECF0BF0EFCF0CF00BC062
:1088B000DEFF0CC0DEFFDE6A010EDE6E0A0EDE6E2B
:1088C000000127EC76F08893B7EF33F052EF46F0D3
:1088D0004A0E895DD8A495EF44F08D53D8A47DEF5E
:1088E00044F0010E8D6FF50EDE6E3E0EDE6E060E4E
:1088F000DE6E34EC9CF086EF44F08D6BF70EDE6E8E
:108900003E0EDE6E060EDE6E34EC9CF08B6B8C6BD6
:10891000010E246E2C0E52EC01F036ECBFF00A0E64
:10892000896F65EF31F052EF46F04B0E895DD8A4A8
:108930000DEF45F0BFEC84F0010E955DD8A4A9EFD2
:1089400044F0D89688B3D886D8B6A9EF44F065EF3E
:1089500031F0040E955DD8A4B0EF44F088EC64F0DB
:10896000020E955DD8A407EF45F0AA6A4F0EA96ED6
:10897000000E43EC01F00A0E51EC01F0AA6A500E11
:10898000A96E000E43EC01F00A0E51EC01F0AA6A48
:10899000510EA96E000E43EC01F00A0E51EC01F0ED
:1089A000AA6A520EA96E000E43EC01F00A0E51ECB9
:1089B00001F0AA6A530EA96E000E43EC01F00A0EF4
:1089C00051EC01F0AA6A540EA96E000E43EC01F0BE
:1089D0000A0E51EC01F0AA6A550EA96E000E43EC86
:1089E00001F00A0E51EC01F0AA6A560EA96E000EB3
:1089F00043EC01F00A0E51EC01F00101276B266BEC
:108A0000296B286B08011B6B1A6B196B186B000123
:108A1000DCEC78F0889352EF46F04C0E895DD8A4D8
:108A2000A0EF45F0BFEC84F0010E955DD8A423EFD4
:108A300045F0D89688B3D886D8B621EF45F065EFD3
:108A400031F056EF45F0020E955DD8A42FEF45F0BA
:108A500036ECBFF0888354EF96F056EF45F0030EE6
:108A6000955DD8A43BEF45F036ECBFF0888354EF1A
:108A700096F056EF45F0040E955DD8A442EF45F010
:108A800056EF45F0050E955DD8A456EF45F0D89603
:108A900088B3D886D8B656EF45F08AC02FFA89C079
:108AA0008AF02FCA89F08883B7EF33F0D89688A36D
:108AB000D886D8B676EF45F0CD0EDE6EDE6ADE6A79
:108AC00034EC9CF03F0EDE6E860EDE6E090EDE6E1E
:108AD00034EC9CF03D0EDE6E900EDE6EDE6A34EC01
:108AE0009CF001012B6B2A6B2D6B2C6B00012AC1B2
:108AF000DEFF2BC1DEFF010EDE6E010EDE6E140EF8
:108B0000DE6E27EC76F004EE1AF0D89001012135E4
:108B1000E926000EEA22EECF0BF0EFCF0CF00BC0EF
:108B2000DEFF0CC0DEFFDE6A010EDE6E0A0EDE6EB8
:108B3000000127EC76F08893B7EF33F052EF46F060
:108B40004D0E895DD8A4A9EF45F0C8EF99F052EF1A
:108B500046F0510E895DD8A4B6EF45F036ECBFF073
:108B60009DEC8AF065EF31F052EF46F0520E895DD0
:108B7000D8A4C3EF45F036ECBFF0E0EC8BF065EF26
:108B800031F052EF46F0530E895DD8A4D0EF45F096
:108B900036ECBFF03CEC87F065EF31F052EF46F079
:108BA000540E895DD8A4F9EF45F0CB2B020ECB5DB6
:108BB000D8A4E6EF45F0CB6BF70EDE6E370EDE6E17
:108BC000060EDE6E34EC9CF0EEEF45F0F50EDE6E38
:108BD000370EDE6E060EDE6E34EC9CF0010E246E57
:108BE0002C0E52EC01F036ECBFF065EF31F052EF95
:108BF00046F0550E895DD8A422EF46F0832B020E75
:108C0000835DD8A40FEF46F0836BF70EDE6E390E4E
:108C1000DE6E060EDE6E34EC9CF017EF46F0F50EBD
:108C2000DE6E390EDE6E060EDE6E34EC9CF0010E4A
:108C3000246E2C0E52EC01F036ECBFF065EF31F0F3
:108C400052EF46F0560E895DD8A42FEF46F036EC71
:108C5000BFF0E3EC96F065EF31F052EF46F0570EBF
:108C6000895DD8A43CEF46F036ECBFF0BCEC88F050
:108C700065EF31F052EF46F0580E895DD8A449EF08
:108C800046F036ECBFF0A9EC89F065EF31F052EF19
:108C900046F05B0E895DD8A450EF46F052EF46F0E7
:108CA00065EF31F0B7EF33F0FF0EDB50DD520A0114
:108CB0003287E8A032970101212B800E215D00014F
:108CC000D8A465EF46F00101216B0001D8960A0196
:108CD00032A7D8860001D8B6E2EF52F00A013293EB
:108CE000346B0001D8960A0132B3D8860001D8B699
:108CF0008FEF46F000EE42F00A013451EB500B6E5C
:108D00002C0E0B5C0001D8A48BEF46F00A013283D5
:108D100000018DEF46F00A01342B0001E2D70A0171
:108D2000342900EE42F0EBCF0BF00BC038FA020E04
:108D3000342500EE42F0EBCF0BF00BC039FA030EF6
:108D4000342500EE42F0EBCF0BF00BC03AFA040EE4
:108D5000342500EE42F0EBCF0BF00BC03BFA050ED2
:108D6000342500EE42F0EBCF0BF00BC03CFA060EC0
:108D7000342500EE42F0EBCF0BF00BC03DFA070EAE
:108D8000342500EE42F0EBCF0BF00BC03EFA080E9C
:108D9000342500EE42F0EBCF0BF00BC03FFA090E8A
:108DA000342500EE42F0EBCF0BF00BC040FA0A0E78
:108DB000342500EE42F0EBCF0BF00BC041FA3293BA
:108DC000356B00010A0E0A01355D0001D8B013EFC2
:108DD00047F00AEE38F00A013551EB500B6E2C0EBD
:108DE0000B5C0001D8A4FDEF46F0F36A0AEE38F000
:108DF0000A013551F3CFEBFF32830001D8960A0107
:108E000032A3D8860001D8B60DEF47F0F36A0AEE18
:108E100038F00A013551F3CFEBFF00010A01352B81
:108E20000001D8A4CED70A013295366B0001D8963E
:108E30000A0132B5D8860001D8B663EF47F00AEED2
:108E400038F00A013651EB500B6E2E0E0B5C000110
:108E5000D8A45FEF47F0060E0A01365D0AEE38F03F
:108E6000EB5001014B6F050E0A01365D0AEE38F03A
:108E7000EB5001014C6F040E0A01365D0AEE38F02A
:108E8000EB5001014D6F030E0A01365D0AEE38F01A
:108E9000EB5001014E6F020E0A01365D0AEE38F00A
:108EA000EB5001014F6F0A0136050AEE38F0EB5026
:108EB0000101506F0A013285000161EF47F00A019C
:108EC000362B0001B3D70A013293342B0001D89618
:108ED0000A0132B3D8860001D8B684EF47F000EE1D
:108EE00042F00A013451EB500B6E2C0E0B5C00016A
:108EF000D8A480EF47F00A013283000182EF47F0E7
:108F00000A01342B0001E2D70A01342900EE42F0B5
:108F1000EB500B6E560E0B5C0001D8A492EF47F09D
:108F200009EFAEF00A01342900EE42F0EB500B6E6F
:108F3000410E0B5C0001D8B4A0EF47F009EFAEF092
:108F40000A01342B32930001D8960A0132B3D88635
:108F50000001D8B6C1EF47F000EE42F00A013451EB
:108F6000EB500B6E2C0E0B5C0001D8A4BDEF47F04C
:108F70000A0132830001BFEF47F00A01342B0001E0
:108F8000E2D70A01342900EE42F0EBCF0BF00BC020
:108F900042FA020E342500EE42F0EBCF0BF00BC08C
:108FA00043FA030E342500EE42F0EBCF0BF00BC07A
:108FB00044FA040E342500EE42F0EBCF0BF00BC068
:108FC00045FA050E342500EE42F0EBCF0BF00BC056
:108FD00046FA060E342500EE42F0EBCF0BF00BC044
:108FE00047FA070E342500EE42F0EBCF0BF00BC032
:108FF00048FA080E342500EE42F0EBCF0BF00BC020
:1090000049FA090E342500EE42F0EBCF0BF00BC00D
:109010004AFA0A0E342500EE42F0EBCF0BF00BC0FB
:109020004BFA0B0E342500EE42F0EBCF0BF00BC0E9
:109030004CFA3293356B00010B0E0A01355D0001CD
:10904000D8B04DEF48F00AEE42F00A013551EB502E
:109050000B6E2C0E0B5C0001D8A437EF48F0F36ABE
:109060000AEE42F00A013551F3CFEBFF32830001E3
:10907000D8960A0132A3D8860001D8B647EF48F047
:10908000F36A0AEE42F00A013551F3CFEBFF00011B
:109090000A01352B0001D8A4CED70A013295366BD0
:1090A0000001D8960A0132B5D8860001D8B6ACEFD7
:1090B00048F00AEE42F00A013651EB500B6E2E0ECC
:1090C0000B5C0001D8A4A8EF48F0040E0A01365D3D
:1090D0000AEE42F0EB500101526F030E0A01365DB9
:1090E0000AEE42F0EB500101536F020E0A01365DA9
:1090F0000AEE42F0EB500101546F0A0136050AEE08
:1091000042F0EB500101556F0A0136290AEE42F098
:10911000EB500101566F020E0A0136250AEE42F0AD
:10912000EB500101576F030E0A0136250AEE42F09B
:10913000EB500101586F040E0A0136250AEE42F089
:10914000EB500101596F0A0132850001AAEF48F086
:109150000A01362B0001A4D7226A216A206A54C171
:109160001FF02A6A010E296E860E286EA00E276E49
:10917000FFEC01F022C099F021C098F020C097F0D8
:109180001FC096F0226A216A206A55C11FF02A6A20
:10919000296A270E286E100E276EFFEC01F022C000
:1091A00034F021C033F020C032F01FC031F0315014
:1091B0009627325097233350982334509923226AAC
:1091C000216A206A56C11FF02A6A296A030E286E96
:1091D000E80E276EFFEC01F022C034F021C033F01E
:1091E00020C032F01FC031F0315096273250972303
:1091F0003350982334509923226A216A206A57C138
:109200001FF02A6A296A286A640E276EFFEC01F0B3
:1092100022C034F021C033F020C032F01FC031F042
:109220003150962732509723335098233450992346
:10923000226A216A206A58C11FF02A6A296A286AAC
:109240000A0E276EFFEC01F022C034F021C033F08B
:1092500020C032F01FC031F0315096273250972392
:109260003350982334509923010159510001962518
:10927000966F000E9721976F000E9821986F000E41
:109280009921996F010152510A0DF3CF31F0F4CFBA
:1092900032F0535131240001CC6F0A01342B329348
:1092A0000001D8960A0132B3D8860001D8B66EEF15
:1092B00049F000EE42F00A013451EB500B6E2C0ED7
:1092C0000B5C0001D8A46AEF49F00A013283000167
:1092D0006CEF49F00A01342B0001E2D70A0134296E
:1092E00000EE42F0EB5001015A6F0A01342B329329
:1092F0000001D8960A0132B3D8860001D8B696EF9D
:1093000049F000EE42F00A013451EB500B6E2C0E86
:109310000B5C0001D8A492EF49F00A0132830001EE
:1093200094EF49F00A01342B0001E2D70A013429F5
:1093300000EE42F0EBCF0BF00BC04DFA020E3425DD
:1093400000EE42F0EBCF0BF00BC04EFA030E3425CB
:1093500000EE42F0EBCF0BF00BC04FFA040E3425B9
:1093600000EE42F0EBCF0BF00BC050FA050E3425A7
:1093700000EE42F0EBCF0BF00BC051FA060E342595
:1093800000EE42F0EBCF0BF00BC052FA070E342583
:1093900000EE42F0EBCF0BF00BC053FA080E342571
:1093A00000EE42F0EBCF0BF00BC054FA090E34255F
:1093B00000EE42F0EBCF0BF00BC055FA0A0E34254D
:1093C00000EE42F0EBCF0BF00BC056FA0B0E34253B
:1093D00000EE42F0EBCF0BF00BC057FA0C0E342529
:1093E00000EE42F0EBCF0BF00BC058FA3293356B26
:1093F00000010B0E0A01355D0001D8B02AEF4AF0DA
:109400000AEE4DF00A013551EB500B6E2C0E0B5C41
:109410000001D8A414EF4AF0F36A0AEE4DF00A01F5
:109420003551F3CFEBFF32830001D8960A0132A306
:10943000D8860001D8B624EF4AF0F36A0AEE4DF060
:109440000A013551F3CFEBFF00010A01352B000172
:10945000D8A4CED70A013295366B0001D8960A01FE
:1094600032B5D8860001D8B691EF4AF00AEE4DF039
:109470000A013651EB500B6E2E0E0B5C0001D8A486
:109480008DEF4AF0050E0A01365D0AEE4DF0EB5005
:1094900001015B6F040E0A01365D0AEE4DF0EB50E0
:1094A00001015C6F030E0A01365D0AEE4DF0EB50D0
:1094B00001015D6F020E0A01365D0AEE4DF0EB50C0
:1094C00001015E6F0A0136050AEE4DF0EB50010115
:1094D0005F6F0A0136290AEE4DF0EB500101606F13
:1094E000020E0A0136250AEE4DF0EB500101616FC4
:1094F000030E0A0136250AEE4DF0EB500101626FB2
:10950000040E0A0136250AEE4DF0EB500101636F9F
:109510000A01328500018FEF4AF00A01362B000163
:109520009CD7226A216A206A5EC11FF02A6A010E56
:10953000296E860E286EA00E276EFFEC01F022C069
:109540009DF021C09CF020C09BF01FC09AF0226AC1
:10955000216A206A5FC11FF02A6A296A270E286ED5
:10956000100E276EFFEC01F022C034F021C033F062
:1095700020C032F01FC031F031509A2732509B2367
:1095800033509C2334509D23226A216A206A60C193
:109590001FF02A6A296A030E286EE80E276EFFEC78
:1095A00001F022C034F021C033F020C032F01FC0DF
:1095B00031F031509A2732509B2333509C23345042
:1095C0009D23226A216A206A61C11FF02A6A296AE2
:1095D000286A640E276EFFEC01F022C034F021C02F
:1095E00033F020C032F01FC031F031509A27325092
:1095F0009B2333509C2334509D23226A216A206A86
:1096000062C11FF02A6A296A286A0A0E276EFFECD7
:1096100001F022C034F021C033F020C032F01FC06E
:1096200031F031509A2732509B2333509C233450D1
:109630009D230101635100019A259A6F000E9B2121
:109640009B6F000E9C219C6F000E9D219D6F326AC6
:109650005BC131F03250640DF3CF32F03150640D04
:10966000F3CF31F0F4503226366A5CC135F0365013
:109670000A0DF3CF36F035500A0DF3CF35F0F45024
:109680003626355031263650322201015D513124C3
:109690000001CD6F0A01342B32930001D8960A01E4
:1096A00032B3D8860001D8B66BEF4BF000EE42F033
:1096B0000A013451EB500B6E2C0E0B5C0001D8A448
:1096C00067EF4BF00A013283000169EF4BF00A01AA
:1096D000342B0001E2D70A01342900EE42F0EB50AE
:1096E0000101646F0A01342B32930001D8960A01FC
:1096F00032B3D8860001D8B693EF4BF000EE42F0BB
:109700000A013451EB500B6E2C0E0B5C0001D8A4F7
:109710008FEF4BF00A013283000191EF4BF00A0109
:10972000342B0001E2D70A01342900EE42F0EBCFDE
:109730000BF00BC059FA020E342500EE42F0EBCFCD
:109740000BF00BC05AFA030E342500EE42F0EBCFBB
:109750000BF00BC05BFA040E342500EE42F0EBCFA9
:109760000BF00BC05CFA050E342500EE42F0EBCF97
:109770000BF00BC05DFA060E342500EE42F0EBCF85
:109780000BF00BC05EFA070E342500EE42F0EBCF73
:109790000BF00BC05FFA3293356B0001070E0A0124
:1097A000355D0001D8B0FFEF4BF00AEE59F00A0129
:1097B0003551EB500B6E2C0E0B5C0001D8A4E9EF79
:1097C0004BF0F36A0AEE59F00A013551F3CFEBFF83
:1097D00032830001D8960A0132A3D8860001D8B698
:1097E000F9EF4BF0F36A0AEE59F00A013551F3CF65
:1097F000EBFF00010A01352B0001D8A4CED70A01E6
:109800003295366B0001D8960A0132B5D886000130
:10981000D8B658EF4CF00AEE59F00A013651EB5029
:109820000B6E2E0E0B5C0001D8A454EF4CF0020E10
:109830000A01365D0001D8B023EF4CF00101656BE1
:1098400000012BEF4CF0020E0A01365D0AEE59F0D2
:10985000EB500101656F0001010E0A01365D000148
:10986000D8B038EF4CF00101666B00013FEF4CF0CF
:109870000A0136050AEE59F0EB500101666F00014E
:109880000A0136290AEE59F0EB500101676F020E0A
:109890000A0136250AEE59F0EB500101686F0A0102
:1098A0003285000156EF4CF00A01362B0001AAD791
:1098B0000A0E0101655D0001D8A061EF4CF00101C5
:1098C000656B00010A0E0101665D0001D8A06BEF17
:1098D0004CF00101666B00010A0E0101675D000199
:1098E000D8A075EF4CF00101676B00010A0E010171
:1098F000685D0001D8A07FEF4CF00101686B0001AA
:10990000326A65C131F032C02EF031502D6EE80D53
:10991000F3CF31F0F4CF32F02E50E80DF350322671
:109920002D50030DF3503226366A66C135F036509D
:10993000640DF3CF36F03550640DF3CF35F0F450AD
:1099400036263550312636503222366A67C135F018
:1099500036500A0DF3CF36F035500A0DF3CF35F0FF
:10996000F4503626355031263650322201016851E6
:109970003124696F000E32206A6F270E0A01376F9B
:1099800000010A0137290B6E01EE9EF0D8903735A1
:10999000E926000EEA22EECF0FF0EFCF10F001EE35
:1099A0009EF0D8900B34E926000EEA220FC0EEFF9D
:1099B00010C0EFFF010E375F0001D8B0E1D76AC1D8
:1099C0009FF169C19EF1C16BC06BBF6BBE6B0A0199
:1099D000696B00010A0169510101325D0001D8A0E3
:1099E0000BEF4DF001EE9EF0D8900A016935E926A3
:1099F000000EEA22EECF0BF0EFCF0CF00B5000017F
:109A0000BE270C50BF23000EC023C1230A01692BBF
:109A10000001D8A4DED7336A346A01013229316EDD
:109A2000000E326A3222C1C022F0C0C021F0BFC095
:109A300020F0BEC01FF034C02AF033C029F032C07D
:109A400028F031C027F088EC01F020C0C3F01FC01F
:109A5000C2F003EE1AF0D8902135E926000EEA2272
:109A6000C2C0EEFFC3C0EFFF03EE1AF0D89021355D
:109A7000E926000EEA22EECF0BF0EFCF0CF00B50F0
:109A8000265D0C5027590001D8B053EF4DF003EE7E
:109A90001AF0D89001012135E926000EEA22EECF16
:109AA00026F1EFCF27F10001C16BC06BBF6BBE6B1E
:109AB0000A01696B0001280E0A01695D0001D8B036
:109AC0007BEF4DF001EE9EF0D8900A016935E92652
:109AD000000EEA22EECF0BF0EFCF0CF00B5000019E
:109AE000BE270C50BF23000EC023C1230A01692BDF
:109AF0000001D8A4DFD7C1C022F0C0C021F0BFC090
:109B000020F0BEC01FF02A6A296A286A280E276E34
:109B100088EC01F020C036F51FC035F50501355140
:109B20000101285D05013651010129590001D8B014
:109B30009EEF4DF036C529F135C528F10A01342BC9
:109B400032930001D8960A0132B3D8860001D8B604
:109B5000BFEF4DF000EE42F00A013451EB500B6EB6
:109B60002C0E0B5C0001D8A4BBEF4DF00A01328330
:109B70000001BDEF4DF00A01342B0001E2D70A01CC
:109B8000342900EE42F0EBCF0BF00BC060FA020E6E
:109B9000342500EE42F0EBCF0BF00BC061FA030E60
:109BA000342500EE42F0EBCF0BF00BC062FA040E4E
:109BB000342500EE42F0EBCF0BF00BC063FA050E3C
:109BC000342500EE42F0EBCF0BF00BC064FA060E2A
:109BD000342500EE42F0EBCF0BF00BC065FA070E18
:109BE000342500EE42F0EBCF0BF00BC066FA329357
:109BF000356B0001070E0A01355D0001D8B02BEF6F
:109C00004EF00AEE60F00A013551EB500B6E2C0E4F
:109C10000B5C0001D8A415EF4EF0F36A0AEE60F079
:109C20000A013551F3CFEBFF32830001D8960A01C8
:109C300032A3D8860001D8B625EF4EF0F36A0AEEBB
:109C400060F00A013551F3CFEBFF00010A01352B1B
:109C50000001D8A4CED70A013295366B0001D89600
:109C60000A0132B5D8860001D8B68AEF4EF00AEE66
:109C700060F00A013651EB500B6E2E0E0B5C0001AA
:109C8000D8A486EF4EF0030E0A01365D0001D8B06D
:109C90004FEF4EF001016B6B000157EF4EF0030EDA
:109CA0000A01365D0AEE60F0EB5001016B6F0001B6
:109CB000020E0A01365D0001D8B064EF4EF00101DA
:109CC0006C6B00016CEF4EF0020E0A01365D0AEE7D
:109CD00060F0EB5001016C6F0001010E0A01365D6E
:109CE0000001D8B079EF4EF001016D6B000180EFFB
:109CF0004EF00A0136050AEE60F0EB5001016D6F7F
:109D000000010A013285000188EF4EF00A01362B6E
:109D10000001A4D7040E01016B5D0001D8A093EFF0
:109D20004EF001016B6B00010A0E01016C5D000138
:109D3000D8A09DEF4EF001016C6B00010A0E0101ED
:109D40006D5D0001D8A0A7EF4EF001016D6B000121
:109D5000326A6BC131F03250640DF3CF32F03150C2
:109D6000640DF3CF31F0F4503226366A6CC135F011
:109D700036500A0DF3CF36F035500A0DF3CF35F0DB
:109D8000F4503626355031263650322201016D51BD
:109D90003124406F000E3220416F2E530001D8A4B1
:109DA000F8EF4EF0010141530001D8A4DFEF4EF06F
:109DB00001012F51405D0001D8A0E7EF4EF00101F5
:109DC0002F51405F000E415B0001F5EF4EF00101A5
:109DD00040512F5D406F411DD8B0010F416F405180
:109DE0006808406F010E4155416F000113EF4FF0BD
:109DF00001012F514027000E4123010E415D00015A
:109E0000D8A012EF4FF0D8A40DEF4FF0680E01016B
:109E1000405D0001D8A012EF4FF0680E0101405FD5
:109E2000010E415B0001130E0A01376F00010A01A8
:109E300037290B6E01EEF0F0D8903735E926000E89
:109E4000EA22EECF0FF0EFCF10F001EEF0F0D89055
:109E50000B34E926000EEA220FC0EEFF10C0EFFF20
:109E6000010E375F0001D8B0E1D741C1F1F140C127
:109E7000F0F10A01946B956B696B00010A0169515D
:109E80000101325D0001D8A092EF4FF001EEF0F039
:109E9000D8900A016935E926000EEA22EECF0BF0D0
:109EA000EFCF0CF00AEE6AF0D8906935E926000E83
:109EB000EA220BC0EEFF0CC0EFFF0AEE6AF0D8906A
:109EC0006935E926000EEA22EECF1FF0EFCF20F031
:109ED000020E72EC01F00B6E030E0B5C0001D8A4B5
:109EE00074EF4FF00A01942B00010AEE6AF0D8904B
:109EF0000A016935E926000EEA22EECF1FF0EFCF06
:109F000020F0020E72EC01F00B6E0B520001D8A48F
:109F10008CEF4FF00A01952B00010A01692B00011B
:109F2000D8A4ABD70A0194530001D8B4F8EF4FF08E
:109F30000A0195530001D8B4F8EF4FF00A0194518B
:109F400095250B6E0C6A0C3601013229116E000E3C
:109F5000126A122212500C5C0001D8A4F8EF4FF0E4
:109F600011500B5CD8A4F8EF4FF00A01696B0001A7
:109F70000A0169510101325D0001D8A0F8EF4FF0EC
:109F80000AEE6AF0D8900A016935E926000EEA2245
:109F9000EECF1FF0EFCF20F0020E72EC01F00B6E4F
:109FA0000B520001D8A4F2EF4FF00AEE6AF0D890FD
:109FB0000A016935E926000EEA22EECF0FF0EFCF55
:109FC00010F0680E0F240B6E010E10200C6E0AEEBE
:109FD0006AF0D8906935E926000EEA220BC0EEFF40
:109FE0000CC0EFFF00010A01692B0001D8A4BFD704
:109FF000C16BC06BBF6BBE6B0A01696B00010A01CC
:10A0000069510101325D0001D8A020EF50F00AEE45
:10A010006AF0D8900A016935E926000EEA22EECFEF
:10A020000BF0EFCF0CF00B500001BE270C50BF23FC
:10A03000000EC023C1230A01692B0001D8A4DED77A
:10A04000336A346A01013229316E000E326A3222DB
:10A05000C1C022F0C0C021F0BFC020F0BEC01FF0C0
:10A0600034C02AF033C029F032C028F031C027F0C4
:10A0700088EC01F020C0C7F01FC0C6F0010E00013F
:10A08000C75DD8A050EF50F0D8A44CEF50F0680E48
:10A09000C65DD8A050EF50F0680EC65F010EC75BDA
:10A0A00004EE1AF0D89001012135E926000EEA22CB
:10A0B000C6C0EEFFC7C0EFFF0A01342B3293000188
:10A0C000D8960A0132B3D8860001D8B67DEF50F099
:10A0D00000EE42F00A013451EB500B6E2C0E0B5C7B
:10A0E0000001D8A479EF50F00A01328300017BEF20
:10A0F00050F00A01342B0001E2D70A01342900EEA6
:10A1000042F0EB5001016E6F020E0A01342500EEA1
:10A1100042F0EB5001016F6F030E0A01342500EE8F
:10A1200042F0EB500101706F040E0A01342500EE7D
:10A1300042F0EB500101716F050E0A01342500EE6B
:10A1400042F0EB500101726F060E0A01342500EE59
:10A1500042F0EB500101736F00019153D8B4BDEF91
:10A1600050F09351010A900ED8B49219D8A4BDEFC3
:10A1700050F041C193F040C192F09153D8B4CDEF6B
:10A1800050F092C0DEFF93C0DEFF3BEC0FF01AEE02
:10A1900067F058EC02F0D0EF50F00A01686B676B83
:10A1A0000001130E0A01376F00010A0137290B6EF7
:10A1B00001EE74F0D8903735E926000EEA22EECF92
:10A1C0000FF0EFCF10F001EE74F0D8900B34E926C9
:10A1D000000EEA220FC0EEFF10C0EFFF010E375F46
:10A1E0000001D8B0E1D768CA75F167CA74F1C16BD4
:10A1F000C06BBF6BBE6B0A01696B00010A0169513C
:10A200000101325D0001D8A01FEF51F001EE74F0A2
:10A21000D8900A016935E926000EEA22EECF0BF04C
:10A22000EFCF0CF00B500001BE270C50BF23000EE7
:10A23000C023C1230A01692B0001D8A4DED7336AE9
:10A24000346A01013229316E000E326A3222C1C0F5
:10A2500022F0C0C021F0BFC020F0BEC01FF034C04B
:10A260002AF033C029F032C028F031C027F088EC42
:10A2700001F020C0C5F01FC0C4F002EE1AF0D89063
:10A280002135E926000EEA22C4C0EEFFC5C0EFFF6B
:10A290000A01675101012C5D0A01685101012D5924
:10A2A0000001D8B05CEF51F068CA2DF167CA2CF1FB
:10A2B00041C12BF140C12AF168CA20F067CA1FF0E2
:10A2C000030E72EC01F005011A6F68CA20F067CA2C
:10A2D0001FF0020E72EC01F01B6F68CA20F067CA13
:10A2E0001FF0010E72EC01F01C6F68CA20F067CA03
:10A2F0001FF0000E72EC01F01D6F020E0001B65D42
:10A30000D8A492EF51F0D89688B3D886D8B692EFF9
:10A3100051F0C853D8A491EF51F043EC29F0C9C0D3
:10A32000C8F0C80703EE1AF0D89001012135E926DC
:10A33000000EEA22EECF0BF0EFCF0CF00C52000132
:10A34000D8A4A8EF51F01F0E0B5CD8A0E0EF52F09C
:10A350003D0E0501345D0001D8A0DDEF52F01A6A10
:10A360007C0E196E120E186E920E176E9AC013F0B4
:10A370009BC014F09CC015F09DC016F059EC09F07C
:10A380004DEC08F016C025F515C024F514C023F5D2
:10A3900013C022F5CD5155EC09F025C51AF024C59E
:10A3A00019F023C518F022C517F0B3EC07F016C05A
:10A3B00025F515C024F514C023F513C022F5570E5A
:10A3C0000101645D0001D8A4E9EF51F0800E0501A0
:10A3D000231B00011A6A7C0E196E120E186E920E63
:10A3E000176E96C013F097C014F098C015F099C07E
:10A3F00016F059EC09F04DEC08F016C021F515C027
:10A4000020F514C01FF513C01EF5CC5155EC09F012
:10A4100021C51AF020C519F01FC518F01EC517F088
:10A42000B3EC07F016C021F515C020F514C01FF5D8
:10A4300013C01EF5530E01015A5D0001D8A424EF8C
:10A4400052F0800E05011F1B00010501265300017B
:10A45000D8B4C8EF52F01EC5DEFF1FC5DEFF20C511
:10A46000DEFF21C5DEFF22C5DEFF23C5DEFF24C5DA
:10A47000DEFF25C5DEFF26C5DEFF27C5DEFF28C5BA
:10A48000DEFF29C5DEFF2AC5DEFF2BC5DEFF2CC59A
:10A49000DEFF2DC5DEFF73EC17F015EE30F047EC54
:10A4A00002F033C522F032C521F031C520F030C5AD
:10A4B0001FF02A6A0F0E296E420E286E400E276E7C
:10A4C00088EC01F020C02FF51FC02EF5226A216A0A
:10A4D0002FC520F02EC51FF02A6A0F0E296E420EDE
:10A4E000286E400E276EFFEC01F022C034F021C030
:10A4F00033F020C032F01FC031F031500501305F21
:10A500003250315B3350325B3450335BD89633BFBB
:10A51000D8860001D8B6C0EF52F005013151321192
:10A52000331106E1650E305D0001D8A0C0EF52F096
:10A53000050130510801182705013151080119237F
:10A540000501325108011A230501335108011B236B
:10A5500021C529F520C528F51FC527F51EC526F5F7
:10A5600025C52DF524C52CF523C52BF522C52AF5C7
:10A570000501336B326B316B306B0001C5EF52F06C
:10A580000501336B326B316B306B0001D8EF52F049
:10A5900021C529F520C528F51FC527F51EC526F5B7
:10A5A00025C52DF524C52CF523C52BF522C52AF587
:10A5B0000501346B0001DFEF52F00501342B00017F
:10A5C000B4EF5AF00A013293346B0001D8960A01B5
:10A5D00032B3D8860001D8B603EF53F000EE42F054
:10A5E0000A013451EB500B6E2C0E0B5C0001D8A409
:10A5F000FFEF52F00A013283000101EF53F00A012C
:10A60000342B0001E2D70A013293342B0001D89693
:10A610000A0132B3D8860001D8B624EF53F000EE19
:10A6200042F00A013451EB500B6E2C0E0B5C000112
:10A63000D8A420EF53F00A013283000122EF53F037
:10A640000A01342B0001E2D70A01342B32930001B6
:10A65000D8960A0132B3D8860001D8B645EF53F038
:10A6600000EE42F00A013451EB500B6E2C0E0B5CE5
:10A670000001D8A441EF53F00A013283000143EFF7
:10A6800053F00A01342B0001E2D70A01342900EE0D
:10A6900042F0EBCF0BF00BC042FA020E342500EE75
:10A6A00042F0EBCF0BF00BC043FA030E342500EE63
:10A6B00042F0EBCF0BF00BC044FA040E342500EE51
:10A6C00042F0EBCF0BF00BC045FA050E342500EE3F
:10A6D00042F0EBCF0BF00BC046FA060E342500EE2D
:10A6E00042F0EBCF0BF00BC047FA070E342500EE1B
:10A6F00042F0EBCF0BF00BC048FA080E342500EE09
:10A7000042F0EBCF0BF00BC049FA090E342500EEF6
:10A7100042F0EBCF0BF00BC04AFA0A0E342500EEE4
:10A7200042F0EBCF0BF00BC04BFA0B0E342500EED2
:10A7300042F0EBCF0BF00BC04CFA3293356B0001BB
:10A740000B0E0A01355D0001D8B0D1EF53F00AEECF
:10A7500042F00A013551EB500B6E2C0E0B5C0001E0
:10A76000D8A4BBEF53F0F36A0AEE42F00A01355168
:10A77000F3CFEBFF32830001D8960A0132A3D886CB
:10A780000001D8B6CBEF53F0F36A0AEE42F00A01AB
:10A790003551F3CFEBFF00010A01352B0001D8A49E
:10A7A000CED70A013295366B0001D8960A0132B530
:10A7B000D8860001D8B630EF54F00AEE42F00A0114
:10A7C0003651EB500B6E2E0E0B5C0001D8A42CEF13
:10A7D00054F0040E0A01365D0AEE42F0EB5001011E
:10A7E000526F030E0A01365D0AEE42F0EB50010192
:10A7F000536F020E0A01365D0AEE42F0EB50010182
:10A80000546F0A0136050AEE42F0EB500101556F14
:10A810000A0136290AEE42F0EB500101566F020E92
:10A820000A0136250AEE42F0EB500101576F030E84
:10A830000A0136250AEE42F0EB500101586F040E72
:10A840000A0136250AEE42F0EB500101596F0A0168
:10A85000328500012EEF54F00A01362B0001A4D7F7
:10A86000226A216A206A54C11FF02A6A010E296EE9
:10A87000860E286EA00E276EFFEC01F022C099F024
:10A8800021C098F020C097F01FC096F0226A216A7C
:10A89000206A55C11FF02A6A296A270E286E100EF9
:10A8A000276EFFEC01F022C034F021C033F020C04D
:10A8B00032F01FC031F03150962732509723335079
:10A8C000982334509923226A216A206A56C11FF0C6
:10A8D0002A6A296A030E286EE80E276EFFEC01F043
:10A8E00022C034F021C033F020C032F01FC031F05C
:10A8F0003150962732509723335098233450992360
:10A90000226A216A206A57C11FF02A6A296A286AC6
:10A91000640E276EFFEC01F022C034F021C033F04A
:10A9200020C032F01FC031F03150962732509723AB
:10A930003350982334509923226A216A206A58C1DF
:10A940001FF02A6A296A286A0A0E276EFFEC01F0B6
:10A9500022C034F021C033F020C032F01FC031F0EB
:10A9600031509627325097233350982334509923EF
:10A970000101595100019625966F000E9721976F9E
:10A98000000E9821986F000E9921996F0101525184
:10A990000A0DF3CF31F0F4CF32F0535131240001DE
:10A9A000CC6F0A01342B32930001D8960A0132B3DE
:10A9B000D8860001D8B6F2EF54F000EE42F00A015A
:10A9C0003451EB500B6E2C0E0B5C0001D8A4EEEF53
:10A9D00054F00A0132830001F0EF54F00A01342BE5
:10A9E0000001E2D70A01342900EE42F0EB500101E8
:10A9F0005A6F0A01342B32930001D8960A0132B300
:10AA0000D8860001D8B61AEF55F000EE42F00A01E0
:10AA10003451EB500B6E2C0E0B5C0001D8A416EFDA
:10AA200055F00A013283000118EF55F00A01342B6A
:10AA30000001E2D70A01342900EE42F0EBCF0BF01F
:10AA40000BC04DFA020E342500EE42F0EBCF0BF0B6
:10AA50000BC04EFA030E342500EE42F0EBCF0BF0A4
:10AA60000BC04FFA040E342500EE42F0EBCF0BF092
:10AA70000BC050FA050E342500EE42F0EBCF0BF080
:10AA80000BC051FA060E342500EE42F0EBCF0BF06E
:10AA90000BC052FA070E342500EE42F0EBCF0BF05C
:10AAA0000BC053FA080E342500EE42F0EBCF0BF04A
:10AAB0000BC054FA090E342500EE42F0EBCF0BF038
:10AAC0000BC055FA0A0E342500EE42F0EBCF0BF026
:10AAD0000BC056FA0B0E342500EE42F0EBCF0BF014
:10AAE0000BC057FA0C0E342500EE42F0EBCF0BF002
:10AAF0000BC058FA3293356B00010B0E0A01355D1D
:10AB00000001D8B0AEEF55F00AEE4DF00A01355114
:10AB1000EB500B6E2C0E0B5C0001D8A498EF55F097
:10AB2000F36A0AEE4DF00A013551F3CFEBFF3283A1
:10AB30000001D8960A0132A3D8860001D8B6A8EF42
:10AB400055F0F36A0AEE4DF00A013551F3CFEBFFF1
:10AB500000010A01352B0001D8A4CED70A01329595
:10AB6000366B0001D8960A0132B5D8860001D8B6F6
:10AB700015EF56F00AEE4DF00A013651EB500B6E10
:10AB80002E0E0B5C0001D8A411EF56F0050E0A0141
:10AB9000365D0AEE4DF0EB5001015B6F040E0A01C9
:10ABA000365D0AEE4DF0EB5001015C6F030E0A01B9
:10ABB000365D0AEE4DF0EB5001015D6F020E0A01A9
:10ABC000365D0AEE4DF0EB5001015E6F0A0136056D
:10ABD0000AEE4DF0EB5001015F6F0A0136290AEED3
:10ABE0004DF0EB500101606F020E0A0136250AEEAE
:10ABF0004DF0EB500101616F030E0A0136250AEE9C
:10AC00004DF0EB500101626F040E0A0136250AEE89
:10AC10004DF0EB500101636F0A013285000113EF23
:10AC200056F00A01362B00019CD7226A216A206A5D
:10AC30005EC11FF02A6A010E296E860E286EA00ED4
:10AC4000276EFFEC01F022C09DF021C09CF020C0D7
:10AC50009BF01FC09AF0226A216A206A5FC11FF030
:10AC60002A6A296A270E286E100E276EFFEC01F063
:10AC700022C034F021C033F020C032F01FC031F0C8
:10AC800031509A2732509B2333509C2334509D23BC
:10AC9000226A216A206A60C11FF02A6A296A030EAB
:10ACA000286EE80E276EFFEC01F022C034F021C0C0
:10ACB00033F020C032F01FC031F031509A273250AB
:10ACC0009B2333509C2334509D23226A216A206A9F
:10ACD00061C11FF02A6A296A286A640E276EFFEC98
:10ACE00001F022C034F021C033F020C032F01FC088
:10ACF00031F031509A2732509B2333509C233450EB
:10AD00009D23226A216A206A62C11FF02A6A296A89
:10AD1000286A0A0E276EFFEC01F022C034F021C031
:10AD200033F020C032F01FC031F031509A2732503A
:10AD30009B2333509C2334509D2301016351000118
:10AD40009A259A6F000E9B219B6F000E9C219C6F91
:10AD5000000E9D219D6F326A5BC131F03250640D4F
:10AD6000F3CF32F03150640DF3CF31F0F45032268E
:10AD7000366A5CC135F036500A0DF3CF36F03550E7
:10AD80000A0DF3CF35F0F4503626355031263650C3
:10AD9000322201015D5131240001CD6F0A01342BB3
:10ADA00032930001D8960A0132B3D8860001D8B692
:10ADB000EFEF56F000EE42F00A013451EB500B6E0B
:10ADC0002C0E0B5C0001D8A4EBEF56F00A01328385
:10ADD0000001EDEF56F00A01342B0001E2D70A0121
:10ADE000342900EE42F0EB500101646F0A01342B6C
:10ADF00032930001D8960A0132B3D8860001D8B642
:10AE000017EF57F000EE42F00A013451EB500B6E91
:10AE10002C0E0B5C0001D8A413EF57F00A0132830B
:10AE2000000115EF57F00A01342B0001E2D70A01A7
:10AE3000342900EE42F0EBCF0BF00BC059FA020EB2
:10AE4000342500EE42F0EBCF0BF00BC05AFA030EA4
:10AE5000342500EE42F0EBCF0BF00BC05BFA040E92
:10AE6000342500EE42F0EBCF0BF00BC05CFA050E80
:10AE7000342500EE42F0EBCF0BF00BC05DFA060E6E
:10AE8000342500EE42F0EBCF0BF00BC05EFA070E5C
:10AE9000342500EE42F0EBCF0BF00BC05FFA32939B
:10AEA000356B0001070E0A01355D0001D8B083EF54
:10AEB00057F00AEE59F00A013551EB500B6E2C0E8B
:10AEC0000B5C0001D8A46DEF57F0F36A0AEE59F05D
:10AED0000A013551F3CFEBFF32830001D8960A0106
:10AEE00032A3D8860001D8B67DEF57F0F36A0AEE98
:10AEF00059F00A013551F3CFEBFF00010A01352B60
:10AF00000001D8A4CED70A013295366B0001D8963D
:10AF10000A0132B5D8860001D8B6DCEF57F00AEE48
:10AF200059F00A013651EB500B6E2E0E0B5C0001EE
:10AF3000D8A4D8EF57F0020E0A01365D0001D8B050
:10AF4000A7EF57F00101656B0001AFEF57F0020E5C
:10AF50000A01365D0AEE59F0EB500101656F000100
:10AF6000010E0A01365D0001D8B0BCEF57F00101B7
:10AF7000666B0001C3EF57F00A0136050AEE59F07F
:10AF8000EB500101666F00010A0136290AEE59F003
:10AF9000EB500101676F020E0A0136250AEE59F0E7
:10AFA000EB500101686F0A0132850001DAEF57F0BA
:10AFB0000A01362B0001AAD70A0E0101655D0001C6
:10AFC000D8A0E5EF57F00101656B00010A0E010101
:10AFD000665D0001D8A0EFEF57F00101666B00013C
:10AFE0000A0E0101675D0001D8A0F9EF57F00101D9
:10AFF000676B00010A0E0101685D0001D8A003EF34
:10B0000058F00101686B0001326A65C131F032C04D
:10B010002EF031502D6EE80DF3CF31F0F4CF32F039
:10B020002E50E80DF35032262D50030DF3503226EA
:10B03000366A66C135F03650640DF3CF36F03550C0
:10B04000640DF3CF35F0F4503626355031263650A6
:10B050003222366A67C135F036500A0DF3CF36F02A
:10B0600035500A0DF3CF35F0F450362635503126E1
:10B0700036503222010168513124696F000E3220AE
:10B080006A6F270E0A01376F00010A0137290B6E1C
:10B0900001EE9EF0D8903735E926000EEA22EECF79
:10B0A0000FF0EFCF10F001EE9EF0D8900B34E926B0
:10B0B000000EEA220FC0EEFF10C0EFFF010E375F57
:10B0C0000001D8B0E1D76AC19FF169C19EF1C16B9F
:10B0D000C06BBF6BBE6B0A01696B00010A0169514D
:10B0E0000101325D0001D8A08FEF58F001EE9EF013
:10B0F000D8900A016935E926000EEA22EECF0BF05E
:10B10000EFCF0CF00B500001BE270C50BF23000EF8
:10B11000C023C1230A01692B0001D8A4DED7336AFA
:10B12000346A01013229316E000E326A3222C1C006
:10B1300022F0C0C021F0BFC020F0BEC01FF034C05C
:10B140002AF033C029F032C028F031C027F088EC53
:10B1500001F020C0C3F01FC0C2F003EE1AF0D89077
:10B160002135E926000EEA22C2C0EEFFC3C0EFFF80
:10B1700003EE1AF0D8902135E926000EEA22EECF30
:10B180000BF0EFCF0CF00B50265D0C50275900014F
:10B19000D8B0D7EF58F003EE1AF0D890010121355E
:10B1A000E926000EEA22EECF26F1EFCF27F10001CB
:10B1B000C16BC06BBF6BBE6B0A01696B0001280ECF
:10B1C0000A01695D0001D8B0FFEF58F001EE9EF072
:10B1D000D8900A016935E926000EEA22EECF0BF07D
:10B1E000EFCF0CF00B500001BE270C50BF23000E18
:10B1F000C023C1230A01692B0001D8A4DFD7C1C035
:10B2000022F0C0C021F0BFC020F0BEC01FF02A6AEB
:10B21000296A286A280E276E88EC01F020C029F1DF
:10B220001FC028F10A01342B32930001D8960A017D
:10B2300032B3D8860001D8B633EF59F000EE42F0B1
:10B240000A013451EB500B6E2C0E0B5C0001D8A49C
:10B250002FEF59F00A013283000131EF59F00A0152
:10B26000342B0001E2D70A01342900EE42F0EBCF83
:10B270000BF00BC060FA020E342500EE42F0EBCF6B
:10B280000BF00BC061FA030E342500EE42F0EBCF59
:10B290000BF00BC062FA040E342500EE42F0EBCF47
:10B2A0000BF00BC063FA050E342500EE42F0EBCF35
:10B2B0000BF00BC064FA060E342500EE42F0EBCF23
:10B2C0000BF00BC065FA070E342500EE42F0EBCF11
:10B2D0000BF00BC066FA3293356B0001070E0A01C2
:10B2E000355D0001D8B09FEF59F00AEE60F00A0119
:10B2F0003551EB500B6E2C0E0B5C0001D8A489EF7E
:10B3000059F0F36A0AEE60F00A013551F3CFEBFF12
:10B3100032830001D8960A0132A3D8860001D8B63C
:10B3200099EF59F0F36A0AEE60F00A013551F3CF54
:10B33000EBFF00010A01352B0001D8A4CED70A018A
:10B340003295366B0001D8960A0132B5D8860001D5
:10B35000D8B6FEEF59F00AEE60F00A013651EB5014
:10B360000B6E2E0E0B5C0001D8A4FAEF59F0030E01
:10B370000A01365D0001D8B0C3EF59F001016B6BD3
:10B380000001CBEF59F0030E0A01365D0AEE60F0C2
:10B39000EB5001016B6F0001020E0A01365D0001E6
:10B3A000D8B0D8EF59F001016C6B0001E0EF59F013
:10B3B000020E0A01365D0AEE60F0EB5001016C6F7F
:10B3C0000001010E0A01365D0001D8B0EDEF59F021
:10B3D00001016D6B0001F4EF59F00A0136050AEE28
:10B3E00060F0EB5001016D6F00010A013285000130
:10B3F000FCEF59F00A01362B0001A4D7040E01011D
:10B400006B5D0001D8A007EF5AF001016B6B0001E2
:10B410000A0E01016C5D0001D8A011EF5AF0010184
:10B420006C6B00010A0E01016D5D0001D8A01BEFDD
:10B430005AF001016D6B0001326A6BC131F032507C
:10B44000640DF3CF32F03150640DF3CF31F0F4508E
:10B450003226366A6CC135F036500A0DF3CF36F01D
:10B4600035500A0DF3CF35F0F450362635503126DD
:10B470003650322201016D513124406F000E3220CE
:10B48000416F2E530001D8A46CEF5AF001014153D3
:10B490000001D8A453EF5AF001012F51405D000183
:10B4A000D8A05BEF5AF001012F51405F000E415BC5
:10B4B000000169EF5AF0010140512F5D406F411DBD
:10B4C000D8B0010F416F40516808406F010E4155DF
:10B4D000416F000187EF5AF001012F514027000E04
:10B4E0004123010E415D0001D8A086EF5AF0D8A497
:10B4F00081EF5AF0680E0101405D0001D8A086EF8F
:10B500005AF0680E0101405F010E415B000104EE3C
:10B510001AF0D89001012135E926000EEA2240C137
:10B52000EEFF41C1EFFF0A01342B32930001D896A0
:10B530000A0132B3D8860001D8B6B4EF5AF000EE53
:10B5400042F00A013451EB500B6E2C0E0B5C0001E3
:10B55000D8A4B0EF5AF00A0132830001B2EF5AF0DA
:10B560000A01342B0001E2D7120036ECBFF0820E44
:10B57000026E800E096E306A540E2F6E06680568E2
:10B580004BEC00F0D8A0F3D70A01966F640E965DDD
:10B590000001D8A41AEF5BF00A019A6B986B976BC5
:10B5A00000010A0198530001D8A408EF5BF0640E73
:10B5B0000A01975D0001D8B008EF5BF00101475127
:10B5C000FCEC00F00A019851100DF3CF32F09751C6
:10B5D000100DF3CF31F0F4503226314A322A325076
:10B5E000FCEC00F03150FCEC00F0E1EC00F0996F65
:10B5F000DE0E995D0001D8A400EF5BF00A019A2BE2
:10B6000000010A01972BD8B4982B0001D8A4C8D701
:10B61000820E026E400E096E306A540E2F6E066A5C
:10B62000056A200E016E0A019A518DEC00F00001AE
:10B63000D7EF5EF0650E0A01965D0001D8A499EF80
:10B640005BF00A019A6B986B976B00010A019853A3
:10B650000001D8A45DEF5BF0640E0A01975D000164
:10B66000D8B05DEF5BF001014751FCEC00F00A013E
:10B670009851100DF3CF32F09751100DF3CF31F0F8
:10B68000F4503226314A322A3250FCEC00F031506C
:10B69000FCEC00F0E1EC00F0996FDE0E995D00012A
:10B6A000D8A455EF5BF00A019A2B00010A01972BF1
:10B6B000D8B4982B0001D8A4C8D70A019A51100D0C
:10B6C000F3CF31F0F4CF32F031040B6E000E32586C
:10B6D0000C6E986B976B00010A0197510B5C9851A7
:10B6E0000C580001D8A097EF5BF001014751FCEC2A
:10B6F00000F00A019851FCEC00F09751FCEC00F0CE
:10B70000E1EC00F0996F820E026E400E096E306A15
:10B71000540E2F6E066A056A200E016E99518DEC4B
:10B7200000F0972BD8B4982B0001D8A4D4D7D7EF2A
:10B730005EF0660E0A01965D0001D8A4A8EF5BF0EA
:10B7400036ECBFF00A0E896F65EF31F0D7EF5EF08F
:10B75000670E0A01965D0001D8A4F1EF5BF00A01C3
:10B76000986B976B00010A01974B982B9853000137
:10B77000D8A4C2EF5BF00B0E0A01975D0001D8A0C0
:10B78000C3EF5BF0F4D6820E026E800E096E306A53
:10B79000540E2F6E130E066E880E056E4BEC00F0E5
:10B7A000D8A0E0D70A01966F96CADEFF000128EC08
:10B7B00063F0FF0EDB50DD520A013289E8A03299B6
:10B7C000820E026E400E096E306A540E2F6E066AAB
:10B7D000056A200E016E7B0E8DEC00F00001D7EFA4
:10B7E0005EF0680E0A01965D0001D8A417EF5DF0C7
:10B7F000820E026E800E096E306A540E2F6E130E8A
:10B80000066E880E056E4BEC00F0D8A0B0D6010194
:10B810002F6F820E026E800E096E306A540E2F6EEC
:10B82000130E066E880E056E4BEC00F00001D8A0DA
:10B830009ED601012E6F820E026E800E096E306A56
:10B84000540E2F6E130E066E880E056E4BEC00F034
:10B850000001D8A08CD60101306F820E026E800EDE
:10B86000096E306A540E2F6E130E066E880E056E2A
:10B870004BEC00F00001D8A07AD60101316F820EA6
:10B88000026E800E096E306A540E2F6E130E066E15
:10B89000880E056E4BEC00F00001D8A068D60101BF
:10B8A000326F820E026E800E096E306A540E2F6E59
:10B8B000130E066E880E056E4BEC00F00001D8A04A
:10B8C00056D60101376F820E026E800E096E306A05
:10B8D000540E2F6E130E066E880E056E4BEC00F0A4
:10B8E0000001D8A044D60101366F820E026E800E90
:10B8F000096E306A540E2F6E130E066E880E056E9A
:10B900004BEC00F00001D8A032D60101356F820E59
:10B91000026E800E096E306A540E2F6E130E066E84
:10B92000880E056E4BEC00F00001D8A020D6010176
:10B93000426FAA6A460EA96E2F5143EC01F00A0E1F
:10B9400051EC01F0AA6A4C0EA96E2E5143EC01F0A5
:10B950000A0E51EC01F0AA6A470EA96E305143EC71
:10B9600001F00A0E51EC01F0AA6A480EA96E31519D
:10B9700043EC01F00A0E51EC01F0AA6A490EA96EDF
:10B98000325143EC01F00A0E51EC01F0AA6A4D0E5F
:10B99000A96E375143EC01F00A0E51EC01F0AA6A8E
:10B9A0004E0EA96E365143EC01F00A0E51EC01F037
:10B9B000AA6A4B0EA96E355143EC01F00A0E51EC08
:10B9C00001F0AA6A4A0EA96E425143EC01F00A0E38
:10B9D00051EC01F0820E026E400E096E306A540E78
:10B9E0002F6E066A056A200E016EFF0E8DEC00F0C8
:10B9F000010E315D0001D8A408EF5DF00101305166
:10BA0000020DF3CFC9F0F4CFCAF0000115EF5DF0DD
:10BA1000010130513C0DF3CF31F0F4CF32F0D8902A
:10BA200031340001C96F3234CA6FD7EF5EF0690E4E
:10BA30000A01965D0001D8A44CEF5DF0820E026E03
:10BA4000400E096E306A540E2F6E066A056A200E8B
:10BA5000016E010123518DEC00F0820E026E400E4A
:10BA6000096E306A540E2F6E066A056A200E016E4A
:10BA700024518DEC00F0820E026E400E096E306A89
:10BA8000540E2F6E066A056A200E016E22518DEC4F
:10BA900000F00001D7EF5EF06A0E0A01965D00012A
:10BAA000D8A4F9EF5DF0460E3AEC01F001012F6FDA
:10BAB000820E026E400E096E306A540E2F6E066AB8
:10BAC000056A200E016E2F518DEC00F04C0E3AEC01
:10BAD00001F02E6F820E026E400E096E306A540E17
:10BAE0002F6E066A056A200E016E2E518DEC00F055
:10BAF000470E3AEC01F0306F820E026E400E096E76
:10BB0000306A540E2F6E066A056A200E016E30519F
:10BB10008DEC00F0480E3AEC01F0316F820E026EAF
:10BB2000400E096E306A540E2F6E066A056A200EAA
:10BB3000016E31518DEC00F0490E3AEC01F0326F9C
:10BB4000820E026E400E096E306A540E2F6E066A27
:10BB5000056A200E016E32518DEC00F04D0E3AEC6C
:10BB600001F0376F820E026E400E096E306A540E7D
:10BB70002F6E066A056A200E016E37518DEC00F0BB
:10BB80004E0E3AEC01F0366F820E026E400E096ED8
:10BB9000306A540E2F6E066A056A200E016E365109
:10BBA0008DEC00F04B0E3AEC01F0356F820E026E18
:10BBB000400E096E306A540E2F6E066A056A200E1A
:10BBC000016E35518DEC00F04A0E3AEC01F0426FF7
:10BBD000820E026E400E096E306A540E2F6E066A97
:10BBE000056A200E016E42518DEC00F00001D7EF86
:10BBF0005EF06B0E0A01965D0001D8A412EF5EF0B4
:10BC000079EC62F0820E026E400E096E306A540EBC
:10BC10002F6E066A056A200E016EFF0E8DEC00F095
:10BC2000D7EF5EF06C0E0A01965D0001D8A431EFEB
:10BC30005EF0FA0EDE6E160EDE6E060EDE6E34EC72
:10BC40009CF0820E026E400E096E306A540E2F6E0A
:10BC5000066A056A200E016ECC0E8DEC00F0D7EF5F
:10BC60005EF06D0E0A01965D0001D8A43CEF5EF017
:10BC7000D1EC62F0D7EF5EF06E0E0A01965D000126
:10BC8000D8A469EF5EF0640E0A019B6F0001D20E2A
:10BC90000A019B5D0001D8B067EF5EF0AA6A9BCAFB
:10BCA000A9FF3CEC01F00A019C6F820E026E400E6F
:10BCB000096E306A540E2F6E066A056A200E016EF8
:10BCC0009C518DEC00F09B2B0001D8A4DFD7D7EF5F
:10BCD0005EF06F0E0A01965D0001D8A4D7EF5EF00A
:10BCE0000A019D6B00010A019D2B0B0E9D5D000159
:10BCF000D8A489EF5EF0820E026E400E096E306AA3
:10BD0000540E2F6E066A056A200E016ED20E8DEC5F
:10BD100000F00B0E0A019D5D0001D8B0D7EF5EF078
:10BD2000640E0A019B6F0001D20E0A019B5D0001A7
:10BD3000D8B0C9EF5EF0820E026E400E096E306A16
:10BD4000540E2F6E066A056A200E016E0A019B5181
:10BD50008DEC00F0820E026E800E096E306A540E79
:10BD60002F6E070E066ED00E056E4BEC00F0000134
:10BD7000D8A0B8D70A019C6FAA6A9BCAA9FF9C5198
:10BD800043EC01F00A0E51EC01F09B2B0001D8A40A
:10BD9000CAD7820E026E400E096E306A540E2F6EA4
:10BDA000066A056A200E016EDE0E8DEC00F0B7EF1C
:10BDB0005AF012000A01AB6BAA6BA06B9F6B0001DB
:10BDC000060E0A01A05D0001D8A0F1EF5EF0D8A434
:10BDD00010EF5FF0400E0A019F5D0001D8B010EF38
:10BDE0005FF001014751FCEC00F00A01A051FCECAE
:10BDF00000F09F51FCEC00F0E1EC00F09E6FDE0ED5
:10BE00009E5D0001D8A409EF5FF0A0CAABFA9FCAFB
:10BE1000AAFA0A019F2BD8B4A02B0001D8A4CFD72F
:10BE20000A01AB51AA110001D8A41BEF5FF0FCEC92
:10BE300060F0FAEF60F001014751FCEC00F00A01FC
:10BE4000AA05316E000EAB59326E3250FCEC00F098
:10BE50003150FCEC00F0E1EC00F09E6F9E2B0101F4
:10BE60004851FCEC00F00F0E0A01AA25316E000EBD
:10BE7000AB21326E3250FCEC00F03150FCEC00F0A3
:10BE80009E51FAEC00F0050E51EC01F00101485111
:10BE9000FCEC00F0100E0A01AA25316E000EAB2159
:10BEA000326E3250FCEC00F03150FCEC00F0DE0E53
:10BEB000FAEC00F0050E51EC01F001014B510A0DB6
:10BEC000F3CF31F0F4CF32F04C5131240A01B16F8D
:10BED00001014851FCEC00F0110E0A01AA25316E57
:10BEE000000EAB21326E3250FCEC00F03150FCEC15
:10BEF00000F0B151FAEC00F0050E51EC01F0010137
:10BF00004D510A0DF3CF31F0F4CF32F04E513124C0
:10BF10000A01B16F01014851FCEC00F0120E0A0158
:10BF2000AA25316E000EAB21326E3250FCEC00F0CF
:10BF30003150FCEC00F0B151FAEC00F0050E51EC80
:10BF400001F001014F510A0DF3CF31F0F4CF32F07F
:10BF5000505131240A01B16F01014851FCEC00F04D
:10BF6000130E0A01AA25316E000EAB21326E32503B
:10BF7000FCEC00F03150FCEC00F0B151FAEC00F0B8
:10BF8000050E51EC01F001016E510A0DF3CF31F0B5
:10BF9000F4CF32F06F5131240A01B16F01014851E1
:10BFA000FCEC00F0140E0A01AA25316E000EAB2144
:10BFB000326E3250FCEC00F03150FCEC00F0B1512C
:10BFC000FAEC00F0050E51EC01F0010170510A0D80
:10BFD000F3CF31F0F4CF32F0715131240A01B16F57
:10BFE00001014851FCEC00F0150E0A01AA25316E42
:10BFF000000EAB21326E3250FCEC00F03150FCEC04
:10C0000000F0B151FAEC00F0050E51EC01F0010125
:10C0100072510A0DF3CF31F0F4CF32F07351312465
:10C020000A01B16F01014851FCEC00F0160E0A0143
:10C03000AA25316E000EAB21326E3250FCEC00F0BE
:10C040003150FCEC00F0B151FAEC00F0050E51EC6F
:10C0500001F001014751FCEC00F00B0E0A01AA258A
:10C06000316E000EAB21326E3250FCEC00F03150DC
:10C07000FCEC00F0E1EC00F0AD6FADCABBF00101EB
:10C080004751FCEC00F00C0E0A01AA25316E000E9F
:10C09000AB21326E3250FCEC00F03150FCEC00F081
:10C0A000E1EC00F0AE6FAECABAF001014751FCEC12
:10C0B00000F00D0E0A01AA25316E000EAB21326E82
:10C0C0003250FCEC00F03150FCEC00F0E1EC00F000
:10C0D000AF6FAFCAB9F001014751FCEC00F00E0E92
:10C0E0000A01AA25316E000EAB21326E3250FCECF3
:10C0F00000F03150FCEC00F0E1EC00F0B06FB0CAA1
:10C10000B8F00001B82B000EB923BA23BB23BBC083
:10C11000ADFABAC0AEFAB9C0AFFAB8C0B0FAB80753
:10C12000000EB95BBA5BBB5B1B0E0A01AA250001BE
:10C13000BC6F000E0A01AB210001BD6F0101485127
:10C14000FCEC00F0170E0A01AA25316E000EAB219F
:10C15000326E3250FCEC00F03150FCEC00F0AD518E
:10C16000FAEC00F0050E51EC01F001014851FCEC35
:10C1700000F0180E0A01AA25316E000EAB21326EB6
:10C180003250FCEC00F03150FCEC00F0AE51FAEC17
:10C1900000F0050E51EC01F001014851FCEC00F0FB
:10C1A000190E0A01AA25316E000EAB21326E3250F3
:10C1B000FCEC00F03150FCEC00F0AF51FAEC00F078
:10C1C000050E51EC01F001014851FCEC00F01A0E93
:10C1D0000A01AA25316E000EAB21326E3250FCEC02
:10C1E00000F03150FCEC00F0B051FAEC00F0050E1C
:10C1F00051EC01F000011200A30E0A01B36FA20E70
:10C20000B46FB66BB56BB451FCEC00F0B651FCECFE
:10C2100000F0B551FCEC00F0010EFAEC00F0050E58
:10C2200051EC01F0B351FCEC00F0B651FCEC00F025
:10C23000B551FCEC00F0E1EC00F0B76FB451FCEC50
:10C2400000F0010EB525316E000EB621326E32506F
:10C25000FCEC00F03150FCEC00F0DE0EFAEC00F0EB
:10C26000050E51EC01F0B351FCEC00F0010EB525C8
:10C27000316E000EB621326E3250FCEC00F03150BF
:10C28000FCEC00F0E1EC00F0B76F01014B510A0D3E
:10C29000F3CF31F0F4CF32F04C5131240A01B86FB2
:10C2A000B451FCEC00F0020EB525316E000EB62143
:10C2B000326E3250FCEC00F03150FCEC00F0B85122
:10C2C000FAEC00F0050E51EC01F001014D510A0DA0
:10C2D000F3CF31F0F4CF32F04E5131240A01B86F70
:10C2E000B451FCEC00F0030EB525316E000EB62102
:10C2F000326E3250FCEC00F03150FCEC00F0B851E2
:10C30000FAEC00F0050E51EC01F001014F510A0D5D
:10C31000F3CF31F0F4CF32F0505131240A01B86F2D
:10C32000B451FCEC00F0040EB525316E000EB621C0
:10C33000326E3250FCEC00F03150FCEC00F0B851A1
:10C34000FAEC00F0050E51EC01F001016E510A0DFE
:10C35000F3CF31F0F4CF32F06F5131240A01B86FCE
:10C36000B451FCEC00F0050EB525316E000EB6217F
:10C37000326E3250FCEC00F03150FCEC00F0B85161
:10C38000FAEC00F0050E51EC01F0010170510A0DBC
:10C39000F3CF31F0F4CF32F0715131240A01B86F8C
:10C3A000B451FCEC00F0060EB525316E000EB6213E
:10C3B000326E3250FCEC00F03150FCEC00F0B85121
:10C3C000FAEC00F0050E51EC01F0010172510A0D7A
:10C3D000F3CF31F0F4CF32F0735131240A01B86F4A
:10C3E000B451FCEC00F0070EB525316E000EB621FD
:10C3F000326E3250FCEC00F03150FCEC00F0B851E1
:10C40000FAEC00F0050E51EC01F0A56BA46B060EE2
:10C41000A36F400EA26FA5CAB8FAB451FCEC00F0AD
:10C42000080EB525316E000EB621326E3250FCEC8E
:10C4300000F03150FCEC00F0B851FAEC00F0050EC1
:10C4400051EC01F0A4CAB8FAB451FCEC00F0090EAA
:10C45000B525316E000EB621326E3250FCEC00F084
:10C460003150FCEC00F0B851FAEC00F0050E51EC44
:10C4700001F0A3CAB8FAB451FCEC00F00A0EB525DD
:10C48000316E000EB621326E3250FCEC00F03150AD
:10C49000FCEC00F0B851FAEC00F0050E51EC01F0A4
:10C4A000A2CAB8FAB451FCEC00F00B0EB525316EFF
:10C4B000000EB621326E3250FCEC00F03150FCEC34
:10C4C00000F0B851FAEC00F0050E51EC01F000015B
:10C4D000BB6BBA6B060EB96F3F0EB86F0C0E0A013C
:10C4E000B5250001BC6F000E0A01B6210001BD6F29
:10C4F00012000A01BA6BB96B0001060E0A01BA5D9F
:10C500000001D8A08EEF62F0D8A4A4EF62F0410E33
:10C510000A01B95D0001D8B0A4EF62F0A20EFCECF4
:10C5200000F00A01BA51FCEC00F0B951FCEC00F04B
:10C53000000EFAEC00F0050E51EC01F0B92BD8B466
:10C54000BA2B0001D8A4D8D712000A01BC6BBB6B70
:10C550000001FF0E0A01BC5D0001D8A0BAEF62F035
:10C56000D8A4D0EF62F0FF0E0A01BB5D0001D8B085
:10C57000D0EF62F0A20EFCEC00F00A01BC51FCEC22
:10C5800000F0BB51FCEC00F0000EFAEC00F0050EE0
:10C5900051EC01F0BB2BD8B4BC2B0001D8A4D8D7E8
:10C5A00012000A01BF6BBE6B00017F0E0A01BF5D66
:10C5B0000001D8A0E6EF62F0D8A427EF63F0F00EF8
:10C5C0000A01BE5D0001D8B027EF63F0820E026E53
:10C5D000800E096E306A540E2F6E130E066E880E92
:10C5E000056E4BEC00F0D8A0B7EF5AF00A01BD6F12
:10C5F000A00EFCEC00F0BF51FCEC00F0BE51FCECD6
:10C6000000F0BD51FAEC00F00A0E51EC01F0A10E61
:10C61000FCEC00F0BF51FCEC00F0BE51FCEC00F073
:10C62000E1EC00F0C06F820E026E400E096E306ABF
:10C63000540E2F6E066A056A200E016EC0518DECF5
:10C6400000F0BE2BD8B4BF2B0001D8A4ADD7120088
:10C65000A30E0A01CA6FA20ECB6FAB0ECC6FAA0E4F
:10C66000CD6FFF0EDBCFC1FADD52329BC151100DF1
:10C67000F3CF31F0F4CF32F0080E315CDF6F000EF3
:10C680003258E06FCA51FCEC00F0E051FCEC00F0D5
:10C69000DF51FCEC00F0E1EC00F0D76FC151100D60
:10C6A000F3CF31F0F4CF32F0070E315CDF6F000EC4
:10C6B0003258E06FCA51FCEC00F0E051FCEC00F0A5
:10C6C000DF51FCEC00F0E1EC00F0D86FC151100D2F
:10C6D000F3CF31F0F4CF32F0060E315CDF6F000E95
:10C6E0003258E06FCA51FCEC00F0E051FCEC00F075
:10C6F000DF51FCEC00F0E1EC00F0D96FC151100DFE
:10C70000F3CF31F0F4CF32F0050E315CDF6F000E65
:10C710003258E06FCA51FCEC00F0E051FCEC00F044
:10C72000DF51FCEC00F0E1EC00F0DA6FD7CAC5FA9B
:10C73000D8CAC4FAD9CAC3FADACAC2FAC151100DAA
:10C74000F3CF31F0F4CF32F0040E315CDF6F000E26
:10C750003258E06FCA51FCEC00F0E051FCEC00F004
:10C76000DF51FCEC00F0E1EC00F0D76FC151100D8F
:10C77000F3CF31F0F4CF32F0030E315CDF6F000EF7
:10C780003258E06FCA51FCEC00F0E051FCEC00F0D4
:10C79000DF51FCEC00F0E1EC00F0D86FC151100D5E
:10C7A000F3CF31F0F4CF32F0020E315CDF6F000EC8
:10C7B0003258E06FCA51FCEC00F0E051FCEC00F0A4
:10C7C000DF51FCEC00F0E1EC00F0D96FC151100D2D
:10C7D000F3CF31F0F4CF32F03104DF6F000E325876
:10C7E000E06FCA51FCEC00F0E051FCEC00F0DF51CE
:10C7F000FCEC00F0E1EC00F0DA6FD7CAC9FAD8CA55
:10C80000C8FAD9CAC7FADACAC6FAC5CAD6FAC4CAB1
:10C81000D5FAC3CAD4FAC2CAD3FA00010A01D35165
:10C82000C65DD451C759D551C859D651C959D651E9
:10C83000C919D8B0800A0001D8A880EF64F0D89652
:10C840000A01D6BFD8860001D8B657EF64F00A01B6
:10C85000D6530AE1D55108E1FF0ED35DFF0ED4593E
:10C860000001D8A057EF64F00A01D329DF6F000E52
:10C87000D421E06FCC51FCEC00F0E051FCEC00F076
:10C88000DF51FCEC00F0E1EC00F0D26F820E026EA2
:10C89000400E096E306A540E2F6E066A056A200E2D
:10C8A000016ED2518DEC00F0000176EF64F0D4CA35
:10C8B000E0FAD3CADFFA0A01CA51FCEC00F0E051F9
:10C8C000FCEC00F0DF51FCEC00F0E1EC00F0D26F8A
:10C8D000820E026E400E096E306A540E2F6E066A8A
:10C8E000056A200E016ED2518DEC00F000010A01A4
:10C8F000D32B000ED423D523D6230001D8A08DD767
:10C900000A01328BE86A32BB010EDE6E00011200B2
:10C9100036ECBFF00A01E56B640EE76F0001C80E4C
:10C920000A01E75D0001D8B0AAEF64F0AA6AE7CA7D
:10C93000A9FF3CEC01F00A01F56FF5290001D8A42C
:10C94000A4EF64F0E7CAE5FA0B0E0A01E72700013D
:10C95000D8A0E4D70A01E5530001D8B448EF68F045
:10C96000206AE5CA1FF0000E72EC01F00A01E66FC2
:10C97000030EDE6E110EDE6E070EDE6E000134EC6D
:10C980009CF0E6CADEFF4D0EDE6E060EDE6E14EC87
:10C99000BDF0710EDE6E630EDE6E070EDE6E34ECE1
:10C9A0009CF09DC022F09CC021F09BC020F09AC05A
:10C9B0001FF02A6A296A286A0A0E276EFFEC01F026
:10C9C00022C034F021C033F020C032F01FC031F05B
:10C9D00034C022F033C021F032C020F031C01FF04B
:10C9E0002A6A296A286A060E276E88EC01F022C09E
:10C9F000F2FA21C0F1FA20C0F0FA1FC0EFFA226A61
:10CA0000216A206ACDC01FF02A6A0F0E296E420EDD
:10CA1000286E400E276EFFEC01F022C034F021C0DA
:10CA200033F020C032F01FC031F031500A01EF273F
:10CA30003250F0233350F1233450F22399C022F0C6
:10CA400098C021F097C020F096C01FF02A6A296A8A
:10CA5000286A0A0E276EFFEC01F022C034F021C0D4
:10CA600033F020C032F01FC031F034C022F033C0A8
:10CA700021F032C020F031C01FF02A6A296A286AEA
:10CA8000060E276E88EC01F022C0EBFA21C0EAFA0C
:10CA900020C0E9FA1FC0E8FA226A216A206ACCC0E5
:10CAA0001FF02A6A0F0E296E420E286E400E276E66
:10CAB000FFEC01F022C034F021C033F020C032F08E
:10CAC0001FC031F03150E8273250E9233350EA23B8
:10CAD0003450EB23F36BF46BF2CA22F0F1CA21F06D
:10CAE000F0CA20F0EFCA1FF0010E7CEC01F0F36FEA
:10CAF000F2CA22F0F1CA21F0F0CA20F0EFCA1FF00A
:10CB0000000E7CEC01F0F46FF3510A0DF3CF31F01D
:10CB1000F4CF32F0F4513124F56F040EE525AA6A02
:10CB2000A96EAA36F55143EC01F00A0E51EC01F062
:10CB3000040EE525AA6AA96EAA363CEC01F0F56F51
:10CB4000F2CA22F0F1CA21F0F0CA20F0EFCA1FF0B9
:10CB50002A6A296A286A640E276E88EC01F022C0CE
:10CB6000F2FA21C0F1FA20C0F0FA1FC0EFFAF36B1D
:10CB7000F46BF2CA22F0F1CA21F0F0CA20F0EFCA39
:10CB80001FF0010E7CEC01F0F36FF2CA22F0F1CA43
:10CB900021F0F0CA20F0EFCA1FF0000E7CEC01F08B
:10CBA000F46FF3510A0DF3CF31F0F4CF32F0F451BA
:10CBB0003124F56F030EE525AA6AA96EAA36F55150
:10CBC00043EC01F00A0E51EC01F0030EE525AA6AD0
:10CBD000A96EAA363CEC01F0F56FF2CA22F0F1CA58
:10CBE00021F0F0CA20F0EFCA1FF02A6A296A286AE9
:10CBF000640E276E88EC01F022C0F2FA21C0F1FA2F
:10CC000020C0F0FA1FC0EFFAF36BF46BF2CA22F007
:10CC1000F1CA21F0F0CA20F0EFCA1FF0010E7CEC3F
:10CC200001F0F36FF2CA22F0F1CA21F0F0CA20F04D
:10CC3000EFCA1FF0000E7CEC01F0F46FF3510A0D07
:10CC4000F3CF31F0F4CF32F0F4513124F56F020E0E
:10CC5000E525AA6AA96EAA36F55143EC01F00A0E41
:10CC600051EC01F0020EE525AA6AA96EAA363CEC49
:10CC700001F0F56FF2CA22F0F1CA21F0F0CA20F0FB
:10CC8000EFCA1FF02A6A296A286A640E276E88ECA8
:10CC900001F022C0F2FA21C0F1FA20C0F0FA1FC060
:10CCA000EFFAF36BF46BF2CA22F0F1CA21F0F0CA8A
:10CCB00020F0EFCA1FF0010E7CEC01F0F36FF2CA16
:10CCC00022F0F1CA21F0F0CA20F0EFCA1FF0000EE6
:10CCD0007CEC01F0F46FF3510A0DF3CF31F0F4CF97
:10CCE00032F0F4513124F56FE529A96E000EAA6ADD
:10CCF000AA22F55143EC01F00A0E51EC01F0E529AE
:10CD0000A96E000EAA6AAA223CEC01F0F56FF2CAE5
:10CD100022F0F1CA21F0F0CA20F0EFCA1FF02A6A0F
:10CD2000296A286A640E276E88EC01F022C0F2FAA4
:10CD300021C0F1FA20C0F0FA1FC0EFFAF46BF2CA7A
:10CD400022F0F1CA21F0F0CA20F0EFCA1FF0000E65
:10CD50007CEC01F0F46FF4CAF5FAAA6AE5CAA9FFFF
:10CD6000F55143EC01F00A0E51EC01F0AA6AE5CA54
:10CD7000A9FF3CEC01F0F56FF36BF46BEBCA22F00A
:10CD8000EACA21F0E9CA20F0E8CA1FF0010E7CECE3
:10CD900001F0F36FEBCA22F0EACA21F0E9CA20F0F1
:10CDA000E8CA1FF0000E7CEC01F0F46FF3510A0D9D
:10CDB000F3CF31F0F4CF32F0F4513124F56F080E97
:10CDC000E525AA6AA96EAA36F55143EC01F00A0ED0
:10CDD00051EC01F0080EE525AA6AA96EAA363CECD2
:10CDE00001F0F56FEBCA22F0EACA21F0E9CA20F09F
:10CDF000E8CA1FF02A6A296A286A640E276E88EC3E
:10CE000001F022C0EBFA21C0EAFA20C0E9FA1FC003
:10CE1000E8FAF36BF46BEBCA22F0EACA21F0E9CA34
:10CE200020F0E8CA1FF0010E7CEC01F0F36FEBCAB2
:10CE300022F0EACA21F0E9CA20F0E8CA1FF0000E89
:10CE40007CEC01F0F46FF3510A0DF3CF31F0F4CF25
:10CE500032F0F4513124F56F070EE525AA6AA96E68
:10CE6000AA36F55143EC01F00A0E51EC01F0070E21
:10CE7000E525AA6AA96EAA363CEC01F0F56FEBCA6B
:10CE800022F0EACA21F0E9CA20F0E8CA1FF02A6AB3
:10CE9000296A286A640E276E88EC01F022C0EBFA3A
:10CEA00021C0EAFA20C0E9FA1FC0E8FAF36BF46B7C
:10CEB000EBCA22F0EACA21F0E9CA20F0E8CA1FF062
:10CEC000010E7CEC01F0F36FEBCA22F0EACA21F00C
:10CED000E9CA20F0E8CA1FF0000E7CEC01F0F46F04
:10CEE000F3510A0DF3CF31F0F4CF32F0F451312485
:10CEF000F56F060EE525AA6AA96EAA36F55143EC30
:10CF000001F00A0E51EC01F0060EE525AA6AA96EA1
:10CF1000AA363CEC01F0F56FEBCA22F0EACA21F028
:10CF2000E9CA20F0E8CA1FF02A6A296A286A640E52
:10CF3000276E88EC01F022C0EBFA21C0EAFA20C08B
:10CF4000E9FA1FC0E8FAF36BF46BEBCA22F0EACA05
:10CF500021F0E9CA20F0E8CA1FF0010E7CEC01F0D4
:10CF6000F36FEBCA22F0EACA21F0E9CA20F0E8CA5E
:10CF70001FF0000E7CEC01F0F46FF3510A0DF3CFBB
:10CF800031F0F4CF32F0F4513124F56F050EE52580
:10CF9000AA6AA96EAA36F55143EC01F0050EE52503
:10CFA000AA6AA96EAA363CEC01F0F56F0A0E51ECA4
:10CFB00001F0570E0101645D0001D8A4F7EF67F09E
:10CFC000090E0A01E525AA6AA96EAA36010E43ECEC
:10CFD00001F00A0E51EC01F0090EE525AA6AA96ECE
:10CFE000AA363CEC01F0F56F00010BEF68F0090E7A
:10CFF0000A01E525AA6AA96EAA36000E43EC01F0E3
:10D000000A0E51EC01F0090EE525AA6AA96EAA36AE
:10D010003CEC01F0F56F0001530E01015A5D000177
:10D02000D8A42AEF68F00A0E0A01E525AA6AA96EBB
:10D03000AA36010E43EC01F00A0E51EC01F0090E84
:10D04000E525AA6AA96EAA363CEC01F0F56F00014D
:10D050003EEF68F00A0E0A01E525AA6AA96EAA3613
:10D06000000E43EC01F00A0E51EC01F0090EE5252B
:10D07000AA6AA96EAA363CEC01F0F56F00010F0E0A
:10D08000246EA00E52EC01F036ECBFF057EF68F0C2
:10D090000B0EDE6E4A0EDE6E010EDE6E14ECBDF07F
:10D0A000070E246ED00E52EC01F036ECBFF08883F0
:10D0B0001200D89688A3D886D8B660EF68F0888D1D
:10D0C000D89688A1D886D8B6A0EF68F004EE1AF0FA
:10D0D000D89001012135E926000EEA22EECF0BF0AF
:10D0E000EFCF0CF00BC0DEFF0CC0DEFF86C0DEFF12
:10D0F00087C0DEFF010EDE6E0001ACEC0EF01AEE12
:10D10000F7F058EC02F00A01F8530001D8A490EFB0
:10D1100068F01F0E0A01F75D0001D8A096EF68F0D5
:10D120008891888DFFECAFF09EEF68F0FFECAFF0D8
:10D13000F7CADEFFF8CADEFF6FECB0F0A2EF68F0CE
:10D14000C6EC0FF01200890EDE6E200EDE6EDE6A77
:10D1500034EC9CF08A0EDE6E2F0EDE6E030EDE6E59
:10D1600034EC9CF01C0EDE6E060EDE6E080EDE6EDB
:10D1700034EC9CF0D70EDE6E870EDE6E080EDE6E8F
:10D1800034EC9CF0040EDE6E350EDE6E080EDE6EA4
:10D1900034EC9CF0BFEC84F0010E955DD8A4D3EF85
:10D1A00068F065EF31F0020E955DD8B4D9EF68F004
:10D1B000F1D736ECBFF09CEC0AF0010EDE6E54ECB9
:10D1C00046F041C1D2F040C1D1F0CCC0AEF01A6AF5
:10D1D0007C0E196E120E186E920E176E96C013F01A
:10D1E00097C014F098C015F099C016F059EC09F0EA
:10D1F0004DEC08F016C0A1F015C0A0F014C09FF0CF
:10D2000013C09EF0CC5155EC09F0A1C01AF0A0C09B
:10D2100019F09FC018F09EC017F0B3EC07F016C0CD
:10D22000A1F015C0A0F014C09FF013C09EF0530EE3
:10D2300001015A5D0001D8A420EF69F0800E9F1B08
:10D24000CDC0B0F01A6A7C0E196E120E186E920ED6
:10D25000176E9AC013F09BC014F09CC015F09DC0CF
:10D2600016F059EC09F04DEC08F016C0A5F015C009
:10D27000A4F014C0A3F013C0A2F0CD5155EC09F0F6
:10D28000A5C01AF0A4C019F0A3C018F0A2C017F0EE
:10D29000B3EC07F016C0A5F015C0A4F014C0A3F0BD
:10D2A00013C0A2F0570E0101645D0001D8A45BEF2A
:10D2B00069F0800EA31B890EDE6E200EDE6EDE6A24
:10D2C00034EC9CF08A0EDE6E2F0EDE6E030EDE6EE8
:10D2D00034EC9CF01C0EDE6E060EDE6E080EDE6E6A
:10D2E00034EC9CF0D90EDE6E870EDE6E080EDE6E1C
:10D2F00034EC9CF0060EDE6E350EDE6E080EDE6E31
:10D3000034EC9CF0BFEC84F0010E955DD8A48BEF5B
:10D3100069F065EF31F0030E955DD8B491EF69F0D7
:10D32000F1D736ECBFF09CEC0AF0010EDE6E54EC47
:10D3300046F0CCC0AFF01A6A7C0E196E120E186E51
:10D34000920E176E96C013F097C014F098C015F0A7
:10D3500099C016F059EC09F04DEC08F016C0A9F090
:10D3600015C0A8F014C0A7F013C0A6F0CC5155EC1E
:10D3700009F0A9C01AF0A8C019F0A7C018F0A6C0FB
:10D3800017F0B3EC07F016C0A9F015C0A8F014C050
:10D39000A7F013C0A6F0530E01015A5D0001D8A4F6
:10D3A000D4EF69F0800EA71BCDC0B1F01A6A7C0ED5
:10D3B000196E120E186E920E176E9AC013F09BC063
:10D3C00014F09CC015F09DC016F059EC09F04DEC1E
:10D3D00008F016C0ADF015C0ACF014C0ABF013C02F
:10D3E000AAF0CD5155EC09F0ADC01AF0ACC019F05F
:10D3F000ABC018F0AAC017F0B3EC07F016C0ADF040
:10D4000015C0ACF014C0ABF013C0AAF0570E010168
:10D41000645D0001D8A40FEF6AF0800EAB1B9EC0C4
:10D42000DEFF9FC0DEFFA0C0DEFFA1C0DEFFA2C006
:10D43000DEFFA3C0DEFFA4C0DEFFA5C0DEFFA6C0E6
:10D44000DEFFA7C0DEFFA8C0DEFFA9C0DEFFAAC0C6
:10D45000DEFFABC0DEFFACC0DEFFADC0DEFF73ECB5
:10D4600017F01AEEF9F047EC02F0FCCA22F0FBCA02
:10D4700021F0FACA20F0F9CA1FF02A6A0F0E296EAD
:10D48000420E286E400E276E88EC01F020C039F164
:10D490001FC038F1226A216A39C120F038C11FF05B
:10D4A0002A6A0F0E296E420E286E400E276EFFEC80
:10D4B00001F022C034F021C033F020C032F01FC090
:10D4C00031F031500A01F95D01013C6F32500A011F
:10D4D000FA5901013D6F33500A01FB5901013E6FBA
:10D4E00034500A01FC5901013F6F3FC122F03EC197
:10D4F00021F03DC120F03CC11FF02A6A296A286A48
:10D50000640E276EFFEC01F022C03FF121C03EF116
:10D5100020C03DF11FC03CF139530001D8A498EF61
:10D520006AF0B40E0101385D0001D8A0A2EF6AF0E4
:10D53000B40E0101385D3A6F000E39593B6F00019E
:10D54000A9EF6AF0B40E010138253A6F000E3921B7
:10D550003B6F0001010E0101355D0001D8A4DFEF32
:10D560006AF03FC122F03EC121F03DC120F03CC134
:10D570001FF02A6A296A286A210E276EFFEC01F043
:10D5800022C034F021C033F020C032F01FC031F08F
:10D5900034C022F033C021F032C020F031C01FF07F
:10D5A0002A6A296A286A0A0E276E88EC01F022C0CE
:10D5B0003FF121C03EF120C03DF11FC03CF1888306
:10D5C000888BB7EF33F01200BFEC84F0010E955D4D
:10D5D000D8A4F7EF6AF0EAECC2F0D89688B3D88600
:10D5E000D8B6F5EF6AF065EF31F030EF6BF0020E70
:10D5F000955DD8A405EF6BF08883D3ECBEF02DECDD
:10D600008DF0D3ECBEF030EF6BF0030E955DD8A437
:10D6100013EF6BF08883D3ECBEF02DEC8DF0D3ECE0
:10D62000BEF030EF6BF0040E955DD8A41AEF6BF0EE
:10D6300030EF6BF0050E955DD8A430EF6BF0D89607
:10D6400088B3D886D8B62EEF6BF08AC02FFA89C07F
:10D650008AF02FCA89F08883B7EF33F030EF6BF090
:10D660009CEC0AF0DE6A54EC46F068EC6CF01BEEC1
:10D6700006F047EC02F0D8960B0109BFD8860001EE
:10D68000D8B658EF6BF03D0E0B01065D860E0759BC
:10D69000010E0859000E09590001D8A058EF6BF08F
:10D6A0000B01096B010E086F860E076F3C0E066FAB
:10D6B00000010B01006B026B036B046B056B09CB64
:10D6C00022F008CB21F007CB20F006CB1FF0040E90
:10D6D0007CEC01F0006F09CB22F008CB21F007CBE6
:10D6E00020F006CB1FF0030E7CEC01F0026F09CB9B
:10D6F00022F008CB21F007CB20F006CB1FF0020E62
:10D700007CEC01F0036F09CB22F008CB21F007CBB2
:10D7100020F006CB1FF0010E7CEC01F0046F09CB6A
:10D7200022F008CB21F007CB20F006CB1FF0000E33
:10D730007CEC01F0056F00530001D8B4DCEF6BF016
:10D740000B0101530001D8A4A9EF6BF0D3ECBEF09C
:10D750008883326A00CB31F03250640DF3CF32F05F
:10D760003150640DF3CF31F0F4503226366A02CBDB
:10D7700035F036500A0DF3CF36F035500A0DF3CFA1
:10D7800035F0F450362635503126365032220B0112
:10D79000035131240A01FE6F000E3220FF6FFECAD2
:10D7A000DEFFFFCADEFFDE6A010EDE6EDE6A00010A
:10D7B00027EC76F02DEF6CF00B0101530001D8B48B
:10D7C000E5EF6BF0D3ECBEF08883326A02CB31F028
:10D7D00032C02EF031502D6EE80DF3CF31F0F4CF82
:10D7E00032F02E50E80DF35032262D50030DF35039
:10D7F0003226366A03CB35F03650640DF3CF36F05F
:10D800003550640DF3CF35F0F450362635503126BF
:10D8100036503222366A04CB35F036500A0DF3CF3B
:10D8200036F035500A0DF3CF35F0F450362635502A
:10D830003126365032220B01055131240A01FE6F88
:10D84000000E3220FF6FFECADEFFFFCADEFFDE6A77
:10D85000DE6ADE6A000127EC76F000CB01FBD89689
:10D8600088A3D886D8B665EF6CF001013553000166
:10D87000D8A445EF6CF00C0EDE6E820EDE6E0D0E3F
:10D88000DE6E34EC9CF04DEF6CF00A0EDE6E820E14
:10D89000DE6E0D0EDE6E34EC9CF00101375300019C
:10D8A000D8A45DEF6CF06F0EDE6E820EDE6E090E98
:10D8B000DE6E34EC9CF065EF6CF06B0EDE6E820E6B
:10D8C000DE6E090EDE6E34EC9CF088937DD612007D
:10D8D0007EEC10F01BEE12F047EC02F0010E01019D
:10D8E000355D0001D8A4A3EF6CF015CB22F014CB6A
:10D8F00021F013CB20F012CB1FF02A6A296A286A84
:10D90000210E276EFFEC01F022C034F021C033F06D
:10D9100020C032F01FC031F034C022F033C021F0FB
:10D9200032C020F031C01FF02A6A296A286A0A0E24
:10D93000276E88EC01F022C015FB21C014FB20C02B
:10D9400013FB1FC012FBD651D511D411D311D8B47B
:10D95000C2EF6CF00B0112510001D35D0B010A6F95
:10D9600013510001D4590B010B6F14510001D5590B
:10D970000B010C6F15510001D6590B010D6F000101
:10D98000C7EF6CF00B010D6B0C6B0B6B0A6B00019E
:10D9900015CBD6F014CBD5F013CBD4F012CBD3F0FB
:10D9A00004EE1AF0D89001012135E926000EEA2292
:10D9B000EECF0BF0EFCF0CF00BC0DEFF0CC0DEFFA4
:10D9C000D1C0DEFFD2C0DEFFDE6A0001ACEC0EF09B
:10D9D0001BEE16F058EC02F0B351640DF3CF19FBB7
:10D9E000B251640DF3CF18FBF4500B01192700015D
:10D9F000B551640DF3CF1BFBB451640DF3CF1AFB8B
:10DA0000F4500B011B271D6B36C11CFB0101355364
:10DA10000001D8A426EF6DF00B011D510A0DF3CFC4
:10DA200032F01C510A0DF3CF31F0F450322632C0DF
:10DA300020F031C01FF0246A210E236EE8EC01F0C3
:10DA40001C6F20C01DFB000147EF6DF0010E0101AE
:10DA5000355D0001D8A42FEF6DF046EF6DF00B019E
:10DA60001D510A0DF3CF32F01C510A0DF3CF31F0E6
:10DA7000F450322632C020F031C01FF0246A210E4B
:10DA8000236EE8EC01F01C6F20C01DFB00010101BA
:10DA90003491D8960B010DAFD8860001D8B6F1EFBE
:10DAA0006DF00B0117530001D8A4AFEF6DF05B0EC2
:10DAB0000B01165D0001D8B0AFEF6DF00B0115BF83
:10DAC00014D015530001D8A477EF6DF00B01145159
:10DAD0000001D8A477EF6DF0E80E0B01125D030E84
:10DAE00013590001D8B077EF6DF0010134810001C6
:10DAF0000B011C5112250E6F1D5113210F6F000ECB
:10DB00001421106F000E1521116F18510E5F19515D
:10DB10000F5B000E105B000E115B1A510E271B519C
:10DB20000F23000E102311230A510E5F0B510F5BC0
:10DB30000C51105B0D51115B11CB22F010CB21F079
:10DB40000FCB20F00E512FEC02F00E6F20C00FFB18
:10DB500021C010FB22C011FB0001F1EF6DF00B01A1
:10DB600017530001D8A4BCEF6DF05B0E0B01165DDE
:10DB70000001D8A0F0EF6DF00B011C5112250E6FC3
:10DB80001D5113210F6F000E1421106F000E15216F
:10DB9000116F18510E2719510F23000E1023112356
:10DBA0001A510E5F1B510F5B000E105B000E115BD4
:10DBB0000A510E5F0B510F5B0C51105B0D51115B45
:10DBC00011CB22F010CB21F00FCB20F00E512FEC17
:10DBD00002F00E6F20C00FFB21C010FB22C011FB12
:10DBE0000001D8960B010DBFD8860001D8B6B5EF5D
:10DBF0006EF00B010A510B110C110D110001D8B47C
:10DC0000B5EF6EF0D8960B010DBFD8860001D8B6DF
:10DC1000B5EF6EF00B010B510C110D1106E1010E69
:10DC20000A5D0001D8A0B5EF6EF00B01175300019B
:10DC3000D8A459EF6EF05B0E0B01165D0001D8B051
:10DC400059EF6EF00B011C51125D0E6F1D511359EF
:10DC50000F6F000E1459106F000E1559116F1851E7
:10DC60000E2719510F23000E102311231A510E5F96
:10DC70001B510F5B000E105B000E115B0A510E5F13
:10DC80000B510F5B0C51105B0D51115B11CB22F04E
:10DC900010CB21F00FCB20F00E512FEC02F00E6FC5
:10DCA00020C00FFB21C010FB22C011FB0001B5EF0B
:10DCB0006EF00B0117530001D8A466EF6EF05B0EF7
:10DCC0000B01165D0001D8A0B4EF6EF00B0115BF7B
:10DCD00014D015530001D8A47FEF6EF00B0114513E
:10DCE0000001D8A47FEF6EF0E80E0B01125D030E69
:10DCF00013590001D8B07FEF6EF0010134810001AB
:10DD00000B011C51125D0E6F1D5113590F6F000E48
:10DD10001459106F000E1559116F18510E5F1951DB
:10DD20000F5B000E105B000E115B1A510E271B518A
:10DD30000F23000E102311230A510E5F0B510F5BAE
:10DD40000C51105B0D51115B11CB22F010CB21F067
:10DD50000FCB20F00E512FEC02F00E6F20C00FFB06
:10DD600021C010FB22C011FB0001010E0101375D33
:10DD70000001D8A4F9EF6EF001013C510B010E5DDA
:10DD800001013D510B010F5901013E510B01105989
:10DD900001013F510B01115901013F510B011119B3
:10DDA000D8B0800A0001D8B8F9EF6EF038C1DEFFB4
:10DDB00039C1DEFF0ECBDEFF0FCBDEFF10CBDEFF67
:10DDC00011CBDEFF04EE1AF0D89001012135E926CF
:10DDD000000EEA22EECF0BF0EFCF0CF00BC0DEFF0F
:10DDE0000CC0DEFF00018EEC15F01BEE0EF047ECD0
:10DDF00002F00ECBDEFF0FCBDEFF10CBDEFF11CB30
:10DE0000DEFF1200FF0EDBCF43FBDD5294510B0D02
:10DE1000F3CF31F0F4CF32F0640E31240B01586FA0
:10DE2000AA6A58CBA9FF3CEC01F0346F5829A96EBF
:10DE3000000EAA6AAA223CEC01F0356F020E5825AA
:10DE4000AA6AA96EAA363CEC01F0366F030E58257B
:10DE5000AA6AA96EAA363CEC01F0376F040E582569
:10DE6000AA6AA96EAA363CEC01F0386F050E582557
:10DE7000AA6AA96EAA363CEC01F0396F060E582545
:10DE8000AA6AA96EAA363CEC01F03A6F070E582533
:10DE9000AA6AA96EAA363CEC01F03B6F080E582521
:10DEA000AA6AA96EAA363CEC01F03C6F090E58250F
:10DEB000AA6AA96EAA363CEC01F03D6F0A0E5825FD
:10DEC000AA6AA96EAA363CEC01F03E6F3429000123
:10DED000D8A479EF6FF00B01606B5F6B5E695D69D1
:10DEE000646B636B696B6A6B6B6B6C6B0001D8EF77
:10DEF00071F0226A216A206A34CB1FF0050E2A6E67
:10DF0000F50E296EE10E286E276AFFEC01F022C0A3
:10DF10004FFB21C04EFB20C04DFB1FC04CFB226AB3
:10DF2000216A206A35CB1FF02A6A0F0E296E420E35
:10DF3000286E400E276EFFEC01F022C034F021C0A5
:10DF400033F020C032F01FC031F031500B014C27AC
:10DF500032504D2333504E2334504F23226A216ACE
:10DF6000206A36CB1FF02A6A296A270E286E100E07
:10DF7000276EFFEC01F022C034F021C033F020C046
:10DF800032F01FC031F031504C2732504D23335006
:10DF90004E2334504F23226A216A206A37CB1FF068
:10DFA0002A6A296A286A640E276EFFEC01F022C0F3
:10DFB00034F021C033F020C032F01FC031F03150B6
:10DFC0004C2732504D2333504E2334504F23385179
:10DFD0004C254C6F000E4D214D6F000E4E214E6FA3
:10DFE000000E4F214F6F010E3D5D0001D8A400EFE0
:10DFF00070F0D880000E0B014C574D574E574F57BD
:10E000000001226A216A206A39CB1FF02A6A0F0EAA
:10E01000296E420E286E400E276EFFEC01F022C0E2
:10E020004BFB21C04AFB20C049FB1FC048FB226AB2
:10E03000216A206A3ACB1FF02A6A296A270E286EC5
:10E04000100E276EFFEC01F022C034F021C033F037
:10E0500020C032F01FC031F031500B014827325040
:10E06000492333504A2334504B23226A216A206AC1
:10E070003BCB1FF02A6A296A286A640E276EFFECE0
:10E0800001F022C034F021C033F020C032F01FC0B4
:10E0900031F0315048273250492333504A2334500D
:10E0A0004B233C514825486F000E4921496F000E13
:10E0B0004A214A6F000E4B214B6F010E3E5D00015D
:10E0C000D8A46AEF70F0D880000E0B01485749576A
:10E0D0004A574B5700011A6A240E196E740E186EB7
:10E0E000920E176E48CB13F049CB14F04ACB15F0C3
:10E0F0004BCB16F059EC09F04DEC08F016C053FB71
:10E1000015C052FB14C051FB13C050FB1A6A240EF9
:10E11000196E740E186E920E176E4CCB13F04DCB19
:10E1200014F04ECB15F04FCB16F059EC09F04DEC36
:10E1300008F016C057FB15C056FB14C055FB13C0A2
:10E1400054FB1A6A7C0E196E120E186E920E176E20
:10E150009AC013F09BC014F09CC015F09DC016F03F
:10E1600059EC09F04DEC08F016C047FB15C046FB12
:10E1700014C045FB13C044FBCD5155EC09F047CB0F
:10E180001AF046CB19F045CB18F044CB17F0B3EC9E
:10E1900007F016C047FB15C046FB14C045FB13C073
:10E1A00044FB570E0101645D0001D8A4DBEF70F061
:10E1B000800E0B01451B00011A6A7C0E196E120EAF
:10E1C000186E920E176E96C013F097C014F098C098
:10E1D00015F099C016F059EC09F04DEC08F016C096
:10E1E00042FB15C041FB14C040FB13C03FFBCC51A8
:10E1F00055EC09F042CB1AF041CB19F040CB18F0A6
:10E200003FCB17F0B3EC07F016C042FB15C041FB43
:10E2100014C040FB13C03FFB530E01015A5D0001C7
:10E22000D8A416EF71F0800E0B01401B00013FCB0C
:10E23000DEFF40CBDEFF41CBDEFF42CBDEFF44CB37
:10E24000DEFF45CBDEFF46CBDEFF47CBDEFF50CB0C
:10E25000DEFF51CBDEFF52CBDEFF53CBDEFF54CBD4
:10E26000DEFF55CBDEFF56CBDEFF57CBDEFF73EC78
:10E2700017F01BEE59F047EC02F05CCB22F05BCBC1
:10E2800021F05ACB20F059CB1FF02A6A0F0E296ECD
:10E29000420E286E400E276E88EC01F020C064FB11
:10E2A0001FC063FB226A216A64CB20F063CB1FF09E
:10E2B0002A6A0F0E296E420E286E400E276EFFEC62
:10E2C00001F022C034F021C033F020C032F01FC072
:10E2D00031F031500B01595D5D6F32505A595E6F0C
:10E2E00033505B595F6F34505C59606F370E435D3C
:10E2F000010ED8A4000E3B6E380E435D010ED8A46B
:10E30000000E3B100001D8B4D7EF71F003EE1AF005
:10E31000D89001012135E926000EEA22EECF0BF05C
:10E32000EFCF0CF00BC0DEFF0CC0DEFF5DCBDEFFDD
:10E330005ECBDEFF5FCBDEFF60CBDEFF0001CAEC11
:10E3400016F01BEE6EF058EC02F06FCB20F06ECBA7
:10E350001FF0246A3C0E236EE8EC01F00B016D6F98
:10E36000206A6DCB1FF0010E72EC01F0696F206A1C
:10E370006DCB1FF0000E72EC01F06A6F6FCB20F0D6
:10E380006ECB1FF0246A3C0E236EE8EC01F027C030
:10E390006DFB206A6DCB1FF0010E72EC01F06B6F0C
:10E3A000206A6DCB1FF0000E72EC01F06C6F000163
:10E3B000010E0101355D0001D8A474EF72F00A016D
:10E3C000329F0B0160BF0CD0A00E5D5D860E5E59C2
:10E3D000010E5F59000E60590001D8B06CEF72F069
:10E3E00060CB22F05FCB21F05ECB20F05DCB1FF045
:10E3F0002A6A296A286A210E276EFFEC01F022C0E2
:10E4000034F021C033F020C032F01FC031F034C0EE
:10E4100022F033C021F032C020F031C01FF02A6A50
:10E42000296A286A0A0E276E88EC01F022C060FB78
:10E4300021C05FFB20C05EFB1FC05DFBD8960B01B7
:10E4400060BFD8860001D8B665EF72F00B0160534B
:10E450000AE15F5108E1E80E5D5D030E5E590001BF
:10E46000D8A065EF72F060CB22F05FCB21F05ECBDD
:10E4700020F05DCB1FF02A6A296A030E286EE80E91
:10E48000276EFFEC01F022C034F021C033F020C031
:10E4900032F01FC031F034C022F033C021F032C05E
:10E4A00020F031C01FF02A6A296A170E286EBC0EB0
:10E4B000276E88EC01F022C060FB21C05FFB20C00A
:10E4C0005EFB1FC05DFB0A01328F00015ECB62FB69
:10E4D0005DCB61FB71EF72F0030E0B01626FE70E13
:10E4E000616F000195EF72F0D8960B0160BFD8867E
:10E4F0000001D8B690EF72F00B0160530AE15F5152
:10E5000008E1FF0E5D5DFF0E5E590001D8A090EF9F
:10E5100072F00B01606B5F6B030E5E6FE70E5D6F59
:10E5200000015ECB62FB5DCB61FB010E0101425D30
:10E530000001D8A4B7EF72F004EE1AF0D8900101F0
:10E540002135E926000EEA22EECF0BF0EFCF0CF0DA
:10E550000BC0DEFF0CC0DEFF63CBDEFF64CBDEFF53
:10E5600000016EEC0EF01BEE63F058EC02F0330E7F
:10E570000B01435D0001D8A4E3EF72F063CBDEFF33
:10E5800064CBDEFFDE6A010EDE6EDE6A27EC76F01B
:10E5900004EE1AF0D89001012135E926000EEA2296
:10E5A000EECF0BF0EFCF0CF00BC0DEFF0CC0DEFFA8
:10E5B000010EDE6E010EDE6E0A0EDE6E000127EC2D
:10E5C00076F0F0EF74F0340E0B01435D0001D8A437
:10E5D0000EEF73F063CBDEFF64CBDEFFDE6A010E6D
:10E5E000DE6EDE6A27EC76F003EE1AF0D8900101B9
:10E5F0002135E926000EEA22EECF0BF0EFCF0CF02A
:10E600000BC0DEFF0CC0DEFF010EDE6EDE6A140EF4
:10E61000DE6E000127EC76F0F0EF74F0350E0B01A2
:10E62000435D0001D8A436EF73F063CBDEFF64CB0B
:10E63000DEFF3BEC0FF01BEE70F058EC02F063CB0A
:10E64000DEFF64CBDEFFDE6A010EDE6EDE6A27ECE3
:10E6500076F070CBDEFF71CBDEFF010EDE6EDE6A80
:10E66000140EDE6E27EC76F0F0EF74F0360E0B0130
:10E67000435D0001D8A4D9EF73F063CBDEFF64CB18
:10E68000DEFFDE6A010EDE6EDE6A27EC76F062CB1C
:10E6900020F061CB1FF0030E246EE80E07EC00F0B3
:10E6A0003B6E010E0A0132BFE86A3B140001D8B488
:10E6B00093EF73F0D8960A0132ADD8860001D8B630
:10E6C00065EF73F004ECBFF0888361CBDEFF62CBB3
:10E6D000DEFF010EDE6E010EDE6EDE6A27EC76F0E6
:10E6E0000A01329DD896000188A3D886D8B691EF4A
:10E6F00073F0010135530001D8A489EF73F00C0EBB
:10E70000DE6E820EDE6E040EDE6E34EC9CF091EF57
:10E7100073F00A0EDE6E820EDE6E040EDE6E34ECD8
:10E720009CF0D7EF73F0D8960A0132BDD88600016D
:10E73000D8B69EEF73F004ECBFF0888362CB20F074
:10E7400061CB1FF0246A0A0E236EE8EC01F00B0186
:10E75000616F20C062FB61CBDEFF62CBDEFF010E8A
:10E76000DE6EDE6ADE6A000127EC76F00A01328D89
:10E77000D896000188A3D886D8B6D7EF73F00101E8
:10E7800035530001D8A4CFEF73F0370EDE6E820E42
:10E79000DE6E040EDE6E34EC9CF0D7EF73F0390EB3
:10E7A000DE6E820EDE6E040EDE6E34EC9CF0F0EF58
:10E7B00074F0370E0B01435D0001D8A4F7EF73F03E
:10E7C00063CBDEFF64CBDEFFDE6A010EDE6EDE6A47
:10E7D00027EC76F0DE6A69CBDEFF6ACBDEFF6BCB1F
:10E7E000DEFF6CCBDEFFA1EC7DF0F0EF74F0380EB5
:10E7F0000B01435D0001D8A499EF74F062CB20F0C7
:10E8000061CB1FF0030E246EE80E04EC00F03B6EAB
:10E81000010E0A0132BFE86A3B140001D8B449EF87
:10E8200074F0D8960A0132ADD8860001D8B61CEF34
:10E8300074F0D3ECBEF0888361CBDEFF62CBDEFFE9
:10E84000DE6A010EDE6EDE6A27EC76F00A01329D8A
:10E85000D896000188A3D886D8B647EF74F0010196
:10E8600035530001D8A43FEF74F00C0EDE6E820E1B
:10E87000DE6E0D0EDE6E34EC9CF047EF74F00A0E87
:10E88000DE6E820EDE6E0D0EDE6E34EC9CF08CEFD2
:10E8900074F0D8960A0132BDD8860001D8B654EF7C
:10E8A00074F0D3ECBEF0888362CB20F061CB1FF014
:10E8B000246A0A0E236EE8EC01F00B01616F20C0A0
:10E8C00062FB61CBDEFF62CBDEFFDE6ADE6ADE6A00
:10E8D000000127EC76F00A01328DD896000188A35A
:10E8E000D886D8B68CEF74F0010135530001D8A456
:10E8F00084EF74F0370EDE6E820EDE6E0D0EDE6E6D
:10E9000034EC9CF08CEF74F0390EDE6E820EDE6E0D
:10E910000D0EDE6E34EC9CF0DE6A69CBDEFF6ACB56
:10E92000DEFF6BCBDEFF6CCBDEFFA1EC7DF0F0EF0A
:10E9300074F0390E0B01435D0001D8A4EEEF74F0C2
:10E9400004EE1AF0D89001012135E926000EEA22E2
:10E95000EECF0BF0EFCF0CF00BC0DEFF0CC0DEFFF4
:10E96000010EDE6E010EDE6E0A0EDE6E000127EC79
:10E9700076F0FFECAFF0010142530001D8A4E6EFBE
:10E9800074F004EE1AF0D89001012135E926000E4A
:10E99000EA22EECF0BF0EFCF0CF00BC0DEFF0CC085
:10E9A000DEFF63CBDEFF64CBDEFF010EDE6E000117
:10E9B000ACEC0EF01BEE72F058EC02F072CBDEFF06
:10E9C00073CBDEFF6FECB0F0ECEF74F063CBDEFFE7
:10E9D00064CBDEFF6FECB0F0F0EF74F065EF31F078
:10E9E00012001BEE7AF058EC02F0D89688A3D88675
:10E9F000D8B602EF75F0380E0B01776F380E786FCE
:10EA0000380E796F00017BCB20F07ACB1FF0030E1C
:10EA1000246EE80E236EE8EC01F00B01746F7BCBE3
:10EA200032F07ACB31F0366A74CB35F036C02EF046
:10EA300035502D6EE80DF3CF35F0F4CF36F02E5073
:10EA4000E80DF35036262D50030DF3503626355081
:10EA5000315E3650325A32C020F031C01FF0246A85
:10EA6000640E236EE8EC01F0756F7BCB32F07ACB4D
:10EA700031F0366A74CB35F036C02EF035502D6E3D
:10EA8000E80DF3CF35F0F4CF36F02E50E80DF3500B
:10EA900036262D50030DF35036263550315E365054
:10EAA000325A366A75CB35F03650640DF3CF36F0F6
:10EAB0003550640DF3CF35F0F45036263550315EC5
:10EAC0003650325A32C020F031C01FF0246A0A0E8C
:10EAD000236EE8EC01F0766FDE6A570EDE6E000101
:10EAE0005EECAEF0170E0B017D6F7551785D000185
:10EAF000D8B481EF75F075CBDEFF7DCBDEFF36EC51
:10EB0000B5F075CB78FB620E0B017D6F7651795DA8
:10EB10000001D8B492EF75F076CBDEFF7DCBDEFF3F
:10EB200036ECB5F076CB79FB0B017C917453000188
:10EB3000D8B4AFEF75F0010E0B017E6F7D6B745191
:10EB4000775D0001D8B4ADEF75F074CBDEFF7DCBFF
:10EB5000DEFF7ECBDEFF14ECBDF00B017C810001FB
:10EB6000E86A0B017CB1010EDE6E000112001BEEA3
:10EB70007FF058EC02F01BEE81F058EC02F00B0134
:10EB800081517F5D825180590001D8B0D0EF75F07E
:10EB9000050EDE6EDE6ADE6A34EC9CF0EEEF75F098
:10EBA0000B018051825D0001D8A4E7EF75F00B01E5
:10EBB0007F51815D0001D8A4E7EF75F0070EDE6E8E
:10EBC000DE6A070EDE6E34EC9CF0EEEF75F0090E97
:10EBD000DE6EDE6A0A0EDE6E34EC9CF012001BEE76
:10EBE00083F058EC02F01BEE85F058EC02F00B01BC
:10EBF0008551835D865184590001D8B008EF76F0C5
:10EC0000AF0EDE6EDE6ADE6A34EC9CF026EF76F044
:10EC10000B018451865D0001D8A41FEF76F00B0133
:10EC20008351855D0001D8A41FEF76F0B10EDE6E32
:10EC3000DE6A030EDE6E34EC9CF026EF76F0B30E47
:10EC4000DE6EDE6A040EDE6E34EC9CF01200FF0E07
:10EC5000DBCF97FBDD52FF0EDB50DD520B017C85D5
:10EC6000E8A07C95FF0EDB50DD527C83E8A07C930E
:10EC70001BEE91F058EC02F0D896000188A3D886DC
:10EC8000D8B650EF76F0430E0B018E6F430E8F6FA8
:10EC9000430E906F430E8B6F430E8C6F430E8D6F40
:10ECA00000010B01876B886B896B8A6BD8967CA3FC
:10ECB000D8860001D8B694EF77F00A0E0B01956F55
:10ECC0000D0E0001895DD8A469EF76F0040E0B01EA
:10ECD000956F0001D8960B017CA5D8860001D8B6A7
:10ECE000C8EF76F092CB20F091CB1FF0020E72ECC1
:10ECF00001F00B01876F92CB20F091CB1FF0010E3A
:10ED000072EC01F0886F92CB20F091CB1FF0000ED7
:10ED100072EC01F0896F8A6B97CB96FB87518B5D04
:10ED20000001D8B49CEF76F095CBDEFF96CBDEFFEA
:10ED300087CBDEFF20ECB5F087CB8BFB290E0B01D8
:10ED40009725966F88518C5D0001D8B4B0EF76F0AE
:10ED500095CBDEFF96CBDEFF88CBDEFF20ECB5F057
:10ED600088CB8CFB520E0B019725966F89518D5DD8
:10ED70000001D8B4C4EF76F095CBDEFF96CBDEFF72
:10ED800089CBDEFF20ECB5F089CB8DFB92EF77F0DD
:10ED900092CB20F091CB1FF0030E72EC01F00B012F
:10EDA000876F92CB20F091CB1FF0020E72EC01F036
:10EDB000886F92CB20F091CB1FF0010E72EC01F026
:10EDC000896F92CB20F091CB1FF0000E72EC01F016
:10EDD0008A6F87530001D8A441EF77F097CB96FB59
:10EDE0000B0188518B5D0001D8B4FFEF76F095CB15
:10EDF000DEFF96CBDEFF88CBDEFF20ECB5F088CBC4
:10EE00008BFB2D0E0B019725966F89518C5D0001B0
:10EE1000D8B413EF77F095CBDEFF96CBDEFF89CB2E
:10EE2000DEFF20ECB5F089CB8CFB5A0E0B01972549
:10EE3000966F8A518D5D0001D8B427EF77F095CB9E
:10EE4000DEFF96CBDEFF8ACBDEFF20ECB5F08ACB6F
:10EE50008DFB5B0E0B019725986F050EDE6E98CB30
:10EE6000DEFF00010FECAFF02E0E0B019725986F1F
:10EE7000050EDE6E98CBDEFF0001EBECAEF092EFFC
:10EE800077F097CB96FB0B0187518B5D0001D8B4CF
:10EE900052EF77F095CBDEFF96CBDEFF87CBDEFF20
:10EEA00020ECB5F087CB8BFB2D0E0B019725966FD1
:10EEB00088518C5D0001D8B466EF77F095CBDEFF0A
:10EEC00096CBDEFF88CBDEFF20ECB5F088CB8CFB49
:10EED0005A0E0B019725966F89518D5D0001D8B4AC
:10EEE0007AEF77F095CBDEFF96CBDEFF89CBDEFFA6
:10EEF00020ECB5F089CB8DFB2E0E0B019725986F7A
:10EF0000050EDE6E98CBDEFF00010FECAFF05B0E5E
:10EF10000B019725986F050EDE6E98CBDEFF000182
:10EF2000EBECAEF0DBEF78F0206A89C01FF0010E49
:10EF300072EC01F00B6E080E0B5CD8A4A5EF77F015
:10EF40000B01956B0001B4EF77F00D0E895DD8A42D
:10EF5000B0EF77F0040E0B01956F0001B3EF77F07F
:10EF6000010E0B01956F0001D8960B017CA5D88688
:10EF70000001D8B611EF78F092CB20F091CB1FF0C2
:10EF8000020E72EC01F00B01876F92CB20F091CB57
:10EF90001FF0010E72EC01F0886F92CB20F091CB44
:10EFA0001FF0000E72EC01F0896F97CB96FB875132
:10EFB0008E5D0001D8B4E5EF77F095CBDEFF96CB00
:10EFC000DEFF87CBDEFF20ECB5F087CB8EFB290E72
:10EFD0000B019725966F88518F5D0001D8B4F9EF2A
:10EFE00077F095CBDEFF96CBDEFF88CBDEFF20EC03
:10EFF000B5F088CB8FFB520E0B019725966F895188
:10F00000905D0001D8B40DEF78F095CBDEFF96CB84
:10F01000DEFF89CBDEFF20ECB5F089CB90FBDBEF88
:10F0200078F092CB20F091CB1FF0030E72EC01F040
:10F030000B01876F92CB20F091CB1FF0020E72EC88
:10F0400001F0886F92CB20F091CB1FF0010E72EC93
:10F0500001F0896F92CB20F091CB1FF0000E72EC83
:10F0600001F08A6F87530001D8A48AEF78F097CB1C
:10F0700096FB0B0188518E5D0001D8B448EF78F003
:10F0800095CBDEFF96CBDEFF88CBDEFF20ECB5F024
:10F0900088CB8EFB2D0E0B019725966F89518F5DC6
:10F0A0000001D8B45CEF78F095CBDEFF96CBDEFFA5
:10F0B00089CBDEFF20ECB5F089CB8FFB5A0E0B011C
:10F0C0009725966F8A51905D0001D8B470EF78F063
:10F0D00095CBDEFF96CBDEFF8ACBDEFF20ECB5F0D2
:10F0E0008ACB90FB530E0B019725986F010EDE6EB5
:10F0F00098CBDEFF000156ECAFF0260E0B019725F2
:10F10000986F010EDE6E98CBDEFF000132ECAFF09F
:10F11000DBEF78F097CB96FB0B0187518E5D0001FA
:10F12000D8B49BEF78F095CBDEFF96CBDEFF87CB94
:10F13000DEFF20ECB5F087CB8EFB2D0E0B01972563
:10F14000966F88518F5D0001D8B4AFEF78F095CB02
:10F15000DEFF96CBDEFF88CBDEFF20ECB5F088CB60
:10F160008FFB5A0E0B019725966F8951905D000118
:10F17000D8B4C3EF78F095CBDEFF96CBDEFF89CB1A
:10F18000DEFF20ECB5F089CB90FB260E0B01972516
:10F19000986F010EDE6E98CBDEFF000156ECAFF0EB
:10F1A000530E0B019725986F010EDE6E98CBDEFF94
:10F1B000000132ECAFF01200D89688A3D886D8B6FA
:10F1C00017EF79F01F0EDE6EDE6A010EDE6E34EC94
:10F1D0009CF0210EDE6EDE6A050EDE6E34EC9CF0D5
:10F1E000010E0101355D0001D8A400EF79F0390E60
:10F1F000DE6EDE6A090EDE6E34EC9CF007EF79F00D
:10F20000370EDE6EDE6A090EDE6E34EC9CF0150EF3
:10F21000DE6E070EDE6E0C0EDE6E34EC9CF0130E0E
:10F22000DE6E5A0EDE6E0C0EDE6E34EC9CF00B01C0
:10F230009A6B27C120F026C11FF0000E72EC01F07E
:10F240009A6F920E996F9ACBDEFF99CBDEFF010E7B
:10F25000DE6E000182ECBAF00B019A6B27C120F040
:10F2600026C11FF0010E72EC01F09A6F840E996FA7
:10F270009ACBDEFF99CBDEFF010EDE6E000182EC41
:10F28000BAF0010EDE6E17ECC2F0800E0B019A6F21
:10F290009ACBDEFF000133ECC2F0030EDE6EA3EC6E
:10F2A000C2F0030EDE6EA3ECC2F00B019A6B27C115
:10F2B00020F026C11FF0020E72EC01F09A6F720E60
:10F2C000996F9ACBDEFF99CBDEFF010EDE6E000157
:10F2D00082ECBAF00B019A6B27C120F026C11FF017
:10F2E000030E72EC01F09A6F640E996F9ACBDEFFF9
:10F2F00099CBDEFF010EDE6E000182ECBAF00B014D
:10F300009A6B29C120F028C11FF0000E72EC01F0A9
:10F310009A6F3E0E996F9ACBDEFF99CBDEFF010EFE
:10F32000DE6E000182ECBAF00B019A6B29C120F06D
:10F3300028C11FF0010E72EC01F09A6F300E996F28
:10F340009ACBDEFF99CBDEFF010EDE6E000182EC70
:10F35000BAF0010EDE6E17ECC2F02C0E0B019A6FA4
:10F360009ACBDEFF000133ECC2F0030EDE6EA3EC9D
:10F37000C2F0030EDE6EA3ECC2F00B019A6B29C142
:10F3800020F028C11FF0020E72EC01F09A6F1E0EE1
:10F39000996F9ACBDEFF99CBDEFF010EDE6E000186
:10F3A00082ECBAF00B019A6B29C120F028C11FF042
:10F3B000030E72EC01F09A6F100E996F9ACBDEFF7C
:10F3C00099CBDEFF010EDE6E000182ECBAF0010186
:10F3D00035530001D8A4F7EF79F01BC8A2FB1AC877
:10F3E000A1FB19C8A0FB18C89FFB27EF7AF01BC828
:10F3F00022F01AC821F019C820F018C81FF02A6A94
:10F40000296A030E286EE80E276EFFEC01F022C079
:10F4100034F021C033F020C032F01FC031F034C0CE
:10F4200022F033C021F032C020F031C01FF02A6A30
:10F43000296A070E286E3C0E276E88EC01F022C068
:10F44000A2FB21C0A1FB20C0A0FB1FC09FFB0B01A2
:10F450009A6BA2CB22F0A1CB21F0A0CB20F09FCBC6
:10F460001FF0010E7CEC01F09A6F920E996F9ACB0F
:10F47000DEFF99CBDEFF050EDE6E000182ECBAF0F6
:10F480000B019A6BA2CB22F0A1CB21F0A0CB20F0F4
:10F490009FCB1FF0020E7CEC01F09A6F840E996FE7
:10F4A0009ACBDEFF99CBDEFF050EDE6E000182EC0B
:10F4B000BAF0050EDE6E17ECC2F0800E0B019A6FEB
:10F4C0009ACBDEFF000133ECC2F0030EDE6EA3EC3C
:10F4D000C2F0030EDE6EA3ECC2F00B019A6BA2CB5E
:10F4E00022F0A1CB21F0A0CB20F09FCB1FF0030E88
:10F4F0007CEC01F09A6F720E996F9ACBDEFF99CB7C
:10F50000DEFF050EDE6E000182ECBAF00B019A6B95
:10F51000A2CB22F0A1CB21F0A0CB20F09FCB1FF0FB
:10F52000040E7CEC01F09A6F640E996F9ACBDEFFAB
:10F5300099CBDEFF050EDE6E000182ECBAF00B0106
:10F540009A6BA2CB22F0A1CB21F0A0CB20F09FCBD5
:10F550001FF0050E7CEC01F09A6F560E996F9ACB56
:10F56000DEFF99CBDEFF050EDE6E000182ECBAF005
:10F570000B019A6BA2CB22F0A1CB21F0A0CB20F003
:10F580009FCB1FF0060E7CEC01F09A6F480E996F2E
:10F590009ACBDEFF99CBDEFF050EDE6E000182EC1A
:10F5A000BAF099C022F098C021F097C020F096C020
:10F5B0001FF02A6A296A286A0A0E276EFFEC01F0FA
:10F5C00022C034F021C033F020C032F01FC031F02F
:10F5D00034C022F033C021F032C020F031C01FF01F
:10F5E0002A6A296A286A060E276E88EC01F022C072
:10F5F0009EFB21C09DFB20C09CFB1FC09BFB226A81
:10F60000216A206ACCC01FF02A6A0F0E296E420EB2
:10F61000286E400E276EFFEC01F022C034F021C0AE
:10F6200033F020C032F01FC031F031500B019B2766
:10F6300032509C2333509D2334509E23530E01019E
:10F640005A5D0001D8A44BEF7BF0010EDE6E25EC75
:10F65000C2F0380E0B019A6F9ACBDEFF00015DEC11
:10F66000C2F00C0EDE6EB1ECC2F00C0EDE6EB1EC30
:10F67000C2F00C0EDE6EB1ECC2F00C0EDE6EB1EC20
:10F68000C2F00C0EDE6EB1ECC2F00C0EDE6EB1EC10
:10F69000C2F069EF7BF0010EDE6E25ECC2F0380E91
:10F6A0000B019A6F9ACBDEFF00015DECC2F0DE6ABF
:10F6B000B1ECC2F0DE6AB1ECC2F0DE6AB1ECC2F0CD
:10F6C000DE6AB1ECC2F0DE6AB1ECC2F0DE6AB1EC27
:10F6D000C2F00B019A6B9ECB22F09DCB21F09CCB0C
:10F6E00020F09BCB1FF0010E7CEC01F09A6F920E84
:10F6F000996F9ACBDEFF99CBDEFF0D0EDE6E000117
:10F7000082ECBAF00B019A6B9ECB22F09DCB21F0DC
:10F710009CCB20F09BCB1FF0020E7CEC01F09A6F8B
:10F72000840E996F9ACBDEFF99CBDEFF0D0EDE6E55
:10F73000000182ECBAF00B019A6B9ECB22F09DCBBC
:10F7400021F09CCB20F09BCB1FF0030E7CEC01F052
:10F750009A6F760E996F9ACBDEFF99CBDEFF0D0E76
:10F76000DE6E000182ECBAF00B019A6B9ECB22F0A8
:10F770009DCB21F09CCB20F09BCB1FF0040E7CECAA
:10F7800001F09A6F680E996F9ACBDEFF99CBDEFF7E
:10F790000D0EDE6E000182ECBAF00B019A6B9ECB6F
:10F7A00022F09DCB21F09CCB20F09BCB1FF0050ECF
:10F7B0007CEC01F09A6F5A0E996F9ACBDEFF99CBD1
:10F7C000DEFF0D0EDE6E000182ECBAF0020EDE6E80
:10F7D00025ECC2F05E0E0B019A6F9ACBDEFF0001A2
:10F7E0005DECC2F0C00EDE6EB1ECC2F0C00EDE6E9B
:10F7F000B1ECC2F00B019A6B9ECB22F09DCB21F0B5
:10F800009CCB20F09BCB1FF0060E7CEC01F09A6F96
:10F81000480E996F9ACBDEFF99CBDEFF0D0EDE6EA0
:10F82000000182ECBAF00B019A6B9ECB22F09DCBCB
:10F8300021F09CCB20F09BCB1FF0070E7CEC01F05D
:10F840009A6F3A0E996F9ACBDEFF99CBDEFF0D0EC1
:10F85000DE6E000182ECBAF09DC022F09CC021F067
:10F860009BC020F09AC01FF02A6A296A286A0A0EF3
:10F87000276EFFEC01F022C034F021C033F020C02D
:10F8800032F01FC031F034C022F033C021F032C05A
:10F8900020F031C01FF02A6A296A286A060E276EF6
:10F8A00088EC01F022C09EFB21C09DFB20C09CFB88
:10F8B0001FC09BFB226A216A206ACDC01FF02A6A02
:10F8C0000F0E296E420E286E400E276EFFEC01F0DF
:10F8D00022C034F021C033F020C032F01FC031F01C
:10F8E00031500B019B2732509C2333509D233450C1
:10F8F0009E23570E0101645D0001D8A4A6EF7CF0A1
:10F90000050EDE6E25ECC2F02A0E0B019A6F9ACB23
:10F91000DEFF00015DECC2F00C0EDE6EB1ECC2F059
:10F920000C0EDE6EB1ECC2F00C0EDE6EB1ECC2F06D
:10F930000C0EDE6EB1ECC2F00C0EDE6EB1ECC2F05D
:10F940000C0EDE6EB1ECC2F0C4EF7CF0050EDE6E84
:10F9500025ECC2F02A0E0B019A6F9ACBDEFF000154
:10F960005DECC2F0DE6AB1ECC2F0DE6AB1ECC2F06E
:10F97000DE6AB1ECC2F0DE6AB1ECC2F0DE6AB1EC74
:10F98000C2F0DE6AB1ECC2F00B019A6B9ECB22F0A2
:10F990009DCB21F09CCB20F09BCB1FF0010E7CEC8B
:10F9A00001F09A6F920E996F9ACBDEFF99CBDEFF32
:10F9B000090EDE6E000182ECBAF00B019A6B9ECB51
:10F9C00022F09DCB21F09CCB20F09BCB1FF0020EB0
:10F9D0007CEC01F09A6F840E996F9ACBDEFF99CB85
:10F9E000DEFF090EDE6E000182ECBAF00B019A6BAD
:10F9F0009ECB22F09DCB21F09CCB20F09BCB1FF027
:10FA0000030E7CEC01F09A6F760E996F9ACBDEFFB5
:10FA100099CBDEFF090EDE6E000182ECBAF00B011D
:10FA20009A6B9ECB22F09DCB21F09CCB20F09BCB00
:10FA30001FF0040E7CEC01F09A6F680E996F9ACB60
:10FA4000DEFF99CBDEFF090EDE6E000182ECBAF01C
:10FA50000B019A6B9ECB22F09DCB21F09CCB20F02A
:10FA60009BCB1FF0050E7CEC01F09A6F5A0E996F3C
:10FA70009ACBDEFF99CBDEFF090EDE6E000182EC31
:10FA8000BAF0060EDE6E25ECC2F05E0E0B019A6F28
:10FA90009ACBDEFF00015DECC2F0C00EDE6EB1EC71
:10FAA000C2F0C00EDE6EB1ECC2F00B019A6B9ECBC1
:10FAB00022F09DCB21F09CCB20F09BCB1FF0060EBB
:10FAC0007CEC01F09A6F480E996F9ACBDEFF99CBD0
:10FAD000DEFF090EDE6E000182ECBAF00B019A6BBC
:10FAE0009ECB22F09DCB21F09CCB20F09BCB1FF036
:10FAF000070E7CEC01F09A6F3A0E996F9ACBDEFFFD
:10FB000099CBDEFF090EDE6E000182ECBAF00B012C
:10FB10009A6B9ECB22F09DCB21F09CCB20F09BCB0F
:10FB20001FF0080E7CEC01F09A6F2C0E996F9ACBA7
:10FB3000DEFF99CBDEFF090EDE6E000182ECBAF02B
:10FB40001200FF0EDBCFA6FBDD52FF0EDBCFA5FBC5
:10FB5000DD52FF0EDBCFA4FBDD52FF0EDBCFA3FB9C
:10FB6000DD52FF0EDB50DD520B017C87E8A07C9755
:10FB7000D896000188A3D886D8B6D0EF7DF0630E62
:10FB80000B01AA6F630EA96F630EA86F630EA76FB8
:10FB9000630EAE6F630EAD6F630EAC6F630EAB6F33
:10FBA0000001D8960B017CB7D8860001D8B611EFBA
:10FBB0007EF0020EDE6E25ECC2F0560EDE6E5DECBF
:10FBC000C2F00B01B16B0001040E0B01B15D00012D
:10FBD000D8B0F4EF7DF03F0EDE6EB1ECC2F00B0159
:10FBE000B12B0001D8A4EFD7050EDE6E25ECC2F0D4
:10FBF000560EDE6E5DECC2F00B01B16B0001040E1F
:10FC00000B01B15D0001D8B00FEF7EF0FC0EDE6E8F
:10FC1000B1ECC2F00B01B12B0001D8A4EFD747EF34
:10FC20007EF0020EDE6E17ECC2F04E0EDE6E33EC8E
:10FC3000C2F00B01B16B0001040E0B01B15D0001BC
:10FC4000D8B02CEF7EF03F0EDE6EA3ECC2F00B01BD
:10FC5000B12B0001D8A4EFD7050EDE6E17ECC2F071
:10FC60004E0EDE6E33ECC2F00B01B16B0001040EE0
:10FC70000B01B15D0001D8B047EF7EF0FC0EDE6EE7
:10FC8000A3ECC2F00B01B12B0001D8A4EFD7D8969A
:10FC90000B017CB7D8860001D8B69EEF7EF0090E26
:10FCA0000B01B06FAF6BA351A75D0001D8B461EF3A
:10FCB0007EF0B0CBDEFFAFCBDEFFA3CBDEFF20ECD0
:10FCC000B5F0A3CBA7FB280E0B01AF6FA451A85D25
:10FCD0000001D8B474EF7EF0B0CBDEFFAFCBDEFF17
:10FCE000A4CBDEFF20ECB5F0A4CBA8FB540E0B0197
:10FCF000AF6FA551A95D0001D8B487EF7EF0B0CBFE
:10FD0000DEFFAFCBDEFFA5CBDEFF20ECB5F0A5CB51
:10FD1000A9FB7C0E0B01AF6FA651AA5D0001D8B400
:10FD20009AEF7EF0B0CBDEFFAFCBDEFFA6CBDEFFDF
:10FD300020ECB5F0A6CBAAFBEBEF7EF0010E0B0199
:10FD4000B06FAF6BA351AB5D0001D8B4B0EF7EF0E4
:10FD5000B0CBDEFFAFCBDEFFA3CBDEFF20ECB5F0F8
:10FD6000A3CBABFB280E0B01AF6FA451AC5D000120
:10FD7000D8B4C3EF7EF0B0CBDEFFAFCBDEFFA4CBB9
:10FD8000DEFF20ECB5F0A4CBACFB540E0B01AF6F43
:10FD9000A551AD5D0001D8B4D6EF7EF0B0CBDEFF4B
:10FDA000AFCBDEFFA5CBDEFF20ECB5F0A5CBADFBE6
:10FDB0007C0E0B01AF6FA651AE5D0001D8B4E9EF28
:10FDC0007EF0B0CBDEFFAFCBDEFFA6CBDEFF20ECBC
:10FDD000B5F0A6CBAEFB1200FF0EDB50DD520B01DF
:10FDE0007C89E8A07C99030E0001CF6F840ECE6F52
:10FDF000CFC020F0CEC01FF0246A3C0E236EE8EC8A
:10FE000001F00B01B66F206AB6CB1FF0010E72EC49
:10FE100001F0B26F206AB6CB1FF0000E72EC01F059
:10FE2000B36FB46BB56B010EDE6EB2CBDEFFB3CB3E
:10FE3000DEFFB4CBDEFFB5CBDEFF000182DED8965D
:10FE400088A3D886D8B62BEF7FF0010E246EF40E6F
:10FE500052EC01F08893BFEC84F0010E955DD8A4BC
:10FE600054EF7FF0D8960B017CB9D8860001D8B644
:10FE70003EEF7FF087EF7FF052EF7FF03E0E895D1F
:10FE8000D8A447EF7FF081EF83F052EF7FF0400E70
:10FE9000895DD8A450EF7FF0D6EF80F052EF7FF06D
:10FEA000B7EF33F082EF7FF0020E955DD8A470EFCC
:10FEB0007FF02C0ECE27010ECF23030ECF5DD8A0EE
:10FEC0006EEF7FF0D8A46AEF7FF0850ECE5DD8A0EC
:10FED0006EEF7FF0010ECF6F2C0ECE6F82EF7FF0B2
:10FEE000030E955DD8A482EF7FF02C0ECE5F010E3D
:10FEF000CF5BCF51CE11D8A482EF7FF0030ECF6F2E
:10FF0000840ECE6FC80E51EC01F072D712001A0E9B
:10FF1000DE6E790EDE6E050EDE6E34EC9CF0C80EE1
:10FF200051EC01F00B01BC6B0001F2A456EF80F024
:10FF30000B01BC2B030EBC5D0001D8A4A2EF7FF027
:10FF40000B01BC6B0001C20ED76EF70ED66EF29499
:10FF5000CE07000ECF5BCFC020F0CEC01FF0246ACA
:10FF60003C0E236EE8EC01F00B01B76F206AB7CBB3
:10FF70001FF0010E72EC01F0B86F206AB7CB1FF0D2
:10FF8000000E72EC01F0B96FCFC020F0CEC01FF0B0
:10FF9000246A3C0E236EE8EC01F027C0B7FB206A10
:10FFA000B7CB1FF0010E72EC01F0BA6F206AB7CB2D
:10FFB0001FF0000E72EC01F0BB6F010EDE6EB8CBCD
:10FFC000DEFFB9CBDEFFBACBDEFFBBCBDEFF00012D
:10FFD000A1EC7DF0CF51CE11D8A4F1EF7FF059EF15
:10FFE00080F0BFEC84F0010E955DD8A403EF80F0A3
:10FFF000020E0B01BC5D0001D8A401EF80F065EF9B
:020000040001F9
:1000000031F054EF80F0020E955DD8A422EF80F01D
:10001000030ECF5D480ED8B4CE5DD8B020EF80F08F
:100020003C0ECE27000ECF23010EDE6EB8CBDEFFD6
:10003000B9CBDEFFBACBDEFFBBCBDEFFA1EC7DF0A0
:1000400054EF80F0030E955DD8A448EF80F0CF53B5
:10005000D8A430EF80F03D0ECE5DD8A042EF80F006
:100060003C0ECE5F000ECF5B010EDE6EB8CBDEFF26
:10007000B9CBDEFFBACBDEFFBBCBDEFFA1EC7DF060
:1000800046EF80F00A0E896F65EF31F054EF80F093
:10009000040E955DD8A44FEF80F054EF80F0050E6C
:1000A000955DD8A454EF80F057EF80F03DD73CD752
:1000B00012000B01BD6B00011A0E0B01BD5D0001AA
:1000C000D8B072EF80F0DBECC2F0C80E51EC01F05A
:1000D000EAECC2F0C80E51EC01F00B01BD2B00019F
:1000E000D8A4E9D7010EB75DD8A482EF80F0030E43
:1000F000B65DD8A482EF80F0020EB66FDAEC5EF047
:10010000020EB76F8AC089F08883B7EF33F0120010
:10011000C20ED76EF70ED66EF294CE07000ECF5BEE
:10012000CFC020F0CEC01FF0246A3C0E236EE8EC56
:1001300001F00B01BE6F206ABECB1FF0010E72EC06
:1001400001F0BF6F206ABECB1FF0000E72EC01F011
:10015000C06FCFC020F0CEC01FF0246A3C0E236ECB
:10016000E8EC01F027C0BEFB206ABECB1FF0010EF9
:1001700072EC01F0C16F206ABECB1FF0000E72EC72
:1001800001F0C26F010EDE6EBFCBDEFFC0CBDEFF23
:10019000C1CBDEFFC2CBDEFF0001A1EC7DF0CF5171
:1001A000CE11D8A4D5EF80F084D712000B017C9D2E
:1001B0000001F2A4DFEF80F0ABDFE0EF80F0F8D7D2
:1001C000CFC020F0CEC01FF0000E72EC01F00B6E1D
:1001D0000B52D8A410EF81F0CF53D8A4F5EF80F0E4
:1001E0003D0ECE5DD8A010EF81F0BFEC84F0F2A4FC
:1001F000FBEF80F08DDF010E955DD8A40FEF81F04D
:10020000D89688B3D886D8B60FEF81F036ECBFF019
:10021000010E246EF40E52EC01F065EF31F0C8D7F8
:10022000D8960B017CBDD8860001D8B623EF81F0AB
:100230009CEC0AF0F2A41EEF81F06ADF0B017C8DCA
:1002400000010BEF82F0DE6A54EC46F0F2A42AEFD4
:1002500081F05EDF68EC6CF01BEEC7F047EC02F05B
:10026000F2A434EF81F054DFCACB22F0C9CB21F0E5
:10027000C8CB20F0C7CB1FF02A6A296A286A640E0F
:10028000276E88EC01F022C0CAFB21C0C9FB20C048
:10029000C8FB1FC0C7FBF2A44FEF81F039DF01019B
:1002A00037530001D8A494EF81F001013C510B01B8
:1002B0000E5D01013D510B010F5901013E510B0132
:1002C000105901013F510B01115901013F510B011F
:1002D0001119D8B0800A0001D8B892EF81F038C166
:1002E000DEFF39C1DEFFC7CBDEFFC8CBDEFFC9CBE7
:1002F000DEFFCACBDEFF04EE1AF0D89001012135F3
:10030000E926000EEA22EECF0BF0EFCF0CF00BC087
:10031000DEFF0CC0DEFF00018EEC15F01BEEC3F01B
:1003200047EC02F09CEF81F0CACBC6FBC9CBC5FB02
:10033000C8CBC4FBC7CBC3FBF2A4A0EF81F0E8DEBF
:1003400003EE1AF0D89001012135E926000EEA22C9
:10035000EECF0BF0EFCF0CF00BC0DEFF0CC0DEFFDA
:10036000C3CBDEFFC4CBDEFFC5CBDEFFC6CBDEFFDB
:100370000001CAEC16F01BEED3F058EC02F0F2A428
:10038000C3EF81F0C5DED4CB20F0D3CB1FF0246ABD
:100390003C0E236EE8EC01F00B01D56F206AD5CB43
:1003A0001FF0010E72EC01F0D66F206AD5CB1FF062
:1003B000000E72EC01F0D76FD4CB20F0D3CB1FF03E
:1003C000246A3C0E236EE8EC01F027C0D5FB206ABE
:1003D000D5CB1FF0010E72EC01F0D86F206AD5CB9F
:1003E0001FF0000E72EC01F0D96F0001F2A4FAEFD9
:1003F00081F08EDEDE6AD6CBDEFFD7CBDEFFD8CB38
:10040000DEFFD9CBDEFFA1EC7DF0F2A409EF82F094
:100410007FDE0B017C9D00018893CAD61200D8961E
:1004200088B3D886D8B624EF82F0BFEC84F0010EF2
:10043000955DD8A424EF82F0D89688B3D886D8B634
:1004400024EF82F065EF31F09CEC0AF0DE6A54ECA8
:1004500046F068EC6CF01BEEDEF047EC02F0E1CB0E
:1004600022F0E0CB21F0DFCB20F0DECB1FF02A6AB8
:10047000296A286A640E276E88EC01F022C0E1FB2D
:1004800021C0E0FB20C0DFFB1FC0DEFB01013753B2
:100490000001D8A48BEF82F001013C510B010E5DED
:1004A00001013D510B010F5901013E510B01105942
:1004B00001013F510B01115901013F510B0111196C
:1004C000D8B0800A0001D8B889EF82F038C1DEFFC9
:1004D00039C1DEFFDECBDEFFDFCBDEFFE0CBDEFFB0
:1004E000E1CBDEFF04EE1AF0D89001012135E926B8
:1004F000000EEA22EECF0BF0EFCF0CF00BC0DEFFC8
:100500000CC0DEFF00018EEC15F01BEEDAF047ECBC
:1005100002F093EF82F0E1CBDDFBE0CBDCFBDFCB45
:10052000DBFBDECBDAFB03EE1AF0D89001012135BC
:10053000E926000EEA22EECF0BF0EFCF0CF00BC055
:10054000DEFF0CC0DEFFDACBDEFFDBCBDEFFDCCB79
:10055000DEFFDDCBDEFF0001CAEC16F01BEEEAF099
:1005600058EC02F0EBCB20F0EACB1FF0246A3C0EF3
:10057000236EE8EC01F00B01EC6F206AECCB1FF06E
:10058000010E72EC01F0ED6F206AECCB1FF0000E53
:1005900072EC01F0EE6FEBCB20F0EACB1FF0246A97
:1005A0003C0E236EE8EC01F027C0ECFB206AECCB9C
:1005B0001FF0010E72EC01F0EF6F206AECCB1FF020
:1005C000000E72EC01F0F06FE46BE66BE76BE86B2A
:1005D000DDCB22F0DCCB21F0DBCB20F0DACB1FF03F
:1005E000020E7CEC01F0E46FDDCB22F0DCCB21F0DD
:1005F000DBCB20F0DACB1FF0010E7CEC01F0E66FD4
:10060000DDCB22F0DCCB21F0DBCB20F0DACB1FF00E
:10061000000E7CEC01F0E76F326AE4CB31F032502F
:10062000640DF3CF32F03150640DF3CF31F0F4505C
:100630003226366AE6CB35F036500A0DF3CF36F067
:1006400035500A0DF3CF35F0F450362635503126AB
:1006500036503222E7513124E26F000E3220E36F30
:10066000E2CBDEFFE3CBDEFFDE6A010EDE6EDE6A8A
:10067000000127EC76F0E4CBE5FBD89688A3D8867A
:10068000D8B673EF83F0010135530001D8A453EFBE
:1006900083F00C0EDE6E820EDE6E0D0EDE6E34EC1E
:1006A0009CF05BEF83F00A0EDE6E820EDE6E0D0EA6
:1006B000DE6E34EC9CF0010137530001D8A46BEFDF
:1006C00083F06F0EDE6E820EDE6E090EDE6E34EC8F
:1006D0009CF073EF83F06B0EDE6E820EDE6E090E01
:1006E000DE6E34EC9CF0DE6AEDCBDEFFEECBDEFF9F
:1006F000EFCBDEFFF0CBDEFFA1EC7DF088938FD651
:100700001200010135530001D8A491EF83F00C0EC3
:10071000DE6E820EDE6E040EDE6E34EC9CF099EF1F
:1007200083F00A0EDE6E820EDE6E040EDE6E34EC98
:100730009CF0010137530001D8A4A9EF83F06F0E9C
:10074000DE6E820EDE6E010EDE6E34EC9CF0B1EFDA
:1007500083F06B0EDE6E820EDE6E010EDE6E34EC0A
:100760009CF00B017C9F0001F2A4BBEF83F088ECAE
:1007700080F0BCEF83F0F7D7CFC020F0CEC01FF0E1
:10078000000E72EC01F00B6E0B52D8A4EDEF83F06B
:10079000CF53D8A4D1EF83F03D0ECE5DD8A0EDEFBE
:1007A00083F0BFEC84F0F2A4D8EF83F088EC80F003
:1007B000010E955DD8A4ECEF83F0D89688B3D88667
:1007C000D8B6ECEF83F036ECBFF0010E246EF40ED9
:1007D00052EC01F065EF31F0C6D7D8960B017CBF23
:1007E000D8860001D8B601EF84F09CEC0AF0F2A4A0
:1007F000FCEF83F088EC80F00B017C8F0001BBEFF5
:1008000084F0DE6A54EC46F0F2A409EF84F088EC40
:1008100080F068EC6CF01BEEF1F047EC02F0F2A413
:1008200014EF84F088EC80F0D8960B01F4BFD886E2
:100830000001D8B631EF84F03D0E0B01F15D860E5C
:10084000F259010EF359000EF4590001D8A031EF0E
:1008500084F00B01F46B010EF36F860EF26F3C0E09
:10086000F16F0001F4CB22F0F3CB21F0F2CB20F0BA
:10087000F1CB1FF02A6A296A286A640E276E88EC79
:1008800001F022C0F4FB21C0F3FB20C0F2FB1FC02B
:10089000F1FBF2A44EEF84F088EC80F00B01F76BD3
:1008A000F86BF96BF4CB22F0F3CB21F0F2CB20F014
:1008B000F1CB1FF0020E7CEC01F0F76FF4CB22F0CD
:1008C000F3CB21F0F2CB20F0F1CB1FF0010E7CEC4A
:1008D00001F0F86FF4CB22F0F3CB21F0F2CB20F053
:1008E000F1CB1FF0000E7CEC01F0F96F0001F2A4D7
:1008F0007CEF84F088EC80F0326AF7CB31F0325034
:10090000640DF3CF32F03150640DF3CF31F0F45079
:100910003226366AF8CB35F036500A0DF3CF36F072
:1009200035500A0DF3CF35F0F450362635503126C8
:10093000365032220B01F9513124F56F000E32206E
:10094000F66FF5CBDEFFF6CBDEFF010EDE6E010E9D
:10095000DE6EDE6A000127EC76F0F2A4B2EF84F0DE
:1009600088EC80F0F7CBFCFBF2A4B9EF84F088ECC4
:1009700080F00B017C9F00018893F5D6120080B6B1
:10098000C3EF84F08887D89688A7D886D8B6D0EFEA
:1009900084F03B0EDE6E980EDE6EDE6A34EC9CF068
:1009A00080B2DCEF84F0050E51EC01F080B2DCEF98
:1009B00084F08889ADEF97F0956B0C010D930001E1
:1009C00080A0E8EF84F00C010D83030E0001956F09
:1009D00081A2F0EF84F00C010D83040E0001956FED
:1009E00080AAF8EF84F00C010D83010E0001956FD1
:1009F00082A200EF85F00C010D83020E0001956FBD
:100A000082A008EF85F00C010D83050E0001956FA3
:100A1000D8960C010DB3D8860001D8B68BEF85F0BF
:100A2000810E026E010E096E400E306E200E2F6E8A
:100A3000066A640E056E0B6AD8804BEC00F0D8A0F5
:100A40008BEF85F00BEEFDF00B5023C0EBFF0B2A74
:100A50000B501008F1E10C010E6B0001100E0C019F
:100A60000E5D0001D8B08BEF85F00BEEFDF00C01B0
:100A70000E51EB500B6E030E0B5C0001D8A486EFF9
:100A800085F0030E0C010E250BEEFDF0EB50106F00
:100A9000206A10CC1FF0080E21EC02F00F6F800EC0
:100AA0000F5D0001D8A459EF85F0010E956F86EF18
:100AB00085F0400E0C010F5D0001D8A464EF85F0B5
:100AC000020E956F86EF85F0200E0C010F5D000180
:100AD000D8A46FEF85F0030E956F86EF85F0100EAA
:100AE0000C010F5D0001D8A47AEF85F0040E956F1C
:100AF00086EF85F0080E0C010F5D0001D8A485EF8C
:100B000085F0050E956F86EF85F0956B0C010E2B29
:100B10000001D8A4A2D71200D89688A3D886D8B648
:100B200097EF85F0010E0C01136F680E126F000134
:100B300001014451010A680ED8B443190001D8A438
:100B4000FBEF85F0E0EC0CF011EE43F058EC02F016
:100B500001014451010A680ED8B443190001D8B408
:100B6000FBEF85F004EE1AF0D89001012135E9265B
:100B7000000EEA22EECF43F1EFCF44F1000136EC54
:100B8000BFF05B0EDE6E360EDE6EDE6A34EC9CF07D
:100B90005B0EDE6E360EDE6E040EDE6E34EC9CF006
:100BA0005B0EDE6E360EDE6E090EDE6E34EC9CF0F1
:100BB0005B0EDE6E360EDE6E0E0EDE6E34EC9CF0DC
:100BC0000C01116B0001150E0C01115D0001D8B074
:100BD000F9EF85F0DBECC2F0C80E51EC01F0EAEC65
:100BE000C2F0C80E51EC01F00C01112B0001D8A489
:100BF000E9D736ECBFF001014451010A680ED8B4C0
:100C000043190001D8B4A3EF86F001014651010A4F
:100C1000680ED8B445190001D8A4A3EF86F0E0EC23
:100C20000CF011EE45F058EC02F001014651010ABA
:100C3000680ED8B445190001D8B4A3EF86F004EECD
:100C40001AF0D89001012135E926000EEA22EECFF4
:100C500045F1EFCF46F144C120F043C11FF0020E31
:100C600072EC01F00B6E030E0B5C0001D8A44BEF8D
:100C700086F046C120F045C11FF0020E72EC01F073
:100C80000B6E0B52D8A44AEF86F0680E010145277F
:100C9000010E4623000144C120F043C11FF0020EA3
:100CA00072EC01F00B6E0B52D8A46AEF86F046C1CD
:100CB00020F045C11FF0020E72EC01F00B6E030E26
:100CC0000B5CD8A469EF86F0680E01014327010E82
:100CD0004423000101014551435D4651445900013F
:100CE000D8A08CEF86F001014551435D0B6E465153
:100CF00044590C6E0C520001D8A489EF86F0190EED
:100D00000B5CD8B089EF86F0010E0101466F680ECA
:100D1000456F0001A3EF86F001014351455D0B6E65
:100D2000445146590C6E0C520001D8A4A2EF86F033
:100D3000190E0B5CD8B0A2EF86F0010E0101466FD0
:100D4000680E456F000101014451010A680ED8B4D4
:100D500043190001D8B418EF87F001014651010A88
:100D6000680ED8B445190001D8B418EF87F0010116
:100D70004351455D445146590001D8B0EDEF86F02E
:100D800001014551435D0C01126F01014651445967
:100D90000C01136FD89013331233010145510C012C
:100DA0001227010146510C011323010E135D0001AE
:100DB000D8A0EAEF86F0D8A4E5EF86F0680E0C0123
:100DC000125D0001D8A0EAEF86F0680E0C01125FF8
:100DD000010E135B000118EF87F001014351455DDF
:100DE0000C01126F0101445146590C01136FD89048
:100DF00013331233010143510C01122701014451F5
:100E00000C011323010E135D0001D8A017EF87F02A
:100E1000D8A412EF87F0680E0C01125D0001D8A073
:100E200017EF87F0680E0C01125F010E135B0001D3
:100E30000C011351010A680ED8B412190001D8B47C
:100E40003BEF87F0D50EDE6E860EDE6EDE6A34EC8A
:100E50009CF0888312CCDEFF13CCDEFF010EDE6E29
:100E6000010EDE6E0A0EDE6E27EC76F0889313CC50
:100E700093F012CC92F01200D89688A3D886D8B6F8
:100E8000D3EF87F0890EDE6E1F0EDE6E010EDE6E72
:100E900034EC9CF0D70EDE6E860EDE6E090EDE6E32
:100EA00034EC9CF0450EDE6E860EDE6E0B0EDE6EB2
:100EB00034EC9CF0D90EDE6E860EDE6E0E0EDE6E0B
:100EC00034EC9CF0DB0EDE6E310EDE6E070EDE6E55
:100ED00034EC9CF0DF0EDE6E680EDE6E070EDE6E0A
:100EE00034EC9CF0E30EDE6E3A0EDE6E040EDE6E27
:100EF00034EC9CF0DD0EDE6E580EDE6E040EDE6EFF
:100F000034EC9CF04E0E3AEC01F00101366F0C010E
:100F1000176B36C116FC16CCDEFF17CCDEFFDE6A7F
:100F2000010EDE6E0A0EDE6E000127EC76F00A0E70
:100F300051EC01F04D0E3AEC01F00101376F3753DF
:100F40000001D8A4B1EF87F05F0EDE6E3C0EDE6EBE
:100F5000070EDE6E34EC9CF0C80E51EC01F0D0EFC1
:100F600087F0010E0101375D0001D8A4C5EF87F0BD
:100F70005D0EDE6E3C0EDE6E070EDE6E34EC9CF017
:100F8000C80E51EC01F0D0EF87F05F0EDE6E3C0E24
:100F9000DE6E070EDE6E34EC9CF0C80E51EC01F0F4
:100FA000C80E51EC01F0010136510C01145D000135
:100FB000D8B4EEEF87F00C01176B36C116FC16CCD7
:100FC000DEFF17CCDEFFDE6A010EDE6E0A0EDE6E7D
:100FD000000127EC76F00A0E51EC01F001013751C7
:100FE0000C010DB501080001D8B429EF88F001010A
:100FF00037530001D8A40AEF88F05F0EDE6E3C0E76
:10100000DE6E070EDE6E34EC9CF0C80E51EC01F083
:1010100029EF88F0010E0101375D0001D8A41EEF11
:1010200088F05D0EDE6E3C0EDE6E070EDE6E34EC7A
:101030009CF0C80E51EC01F029EF88F05F0EDE6ED7
:101040003C0EDE6E070EDE6E34EC9CF0C80E51ECEA
:1010500001F0D8960C010DA7D8860001D8B638EF5C
:1010600088F0010E246E2C0E52EC01F00C010D974D
:101070000001BFEC84F0010E955DD8A45CEF88F010
:10108000AA6A4D0EA96E0101375143EC01F0050E1D
:1010900051EC01F0AA6A4E0EA96E365143EC01F0F4
:1010A000050E51EC01F0D896000188B3D886D8B669
:1010B0005CEF88F065EF31F0020E955DD8A46FEF1C
:1010C00088F036C114FC0101362B36290001D8A462
:1010D0006CEF88F00101366B00010C010D870001F7
:1010E000030E955DD8A484EF88F036C114FC01018D
:1010F00036530001D8A47FEF88F001013669000162
:10110000010136070C010D870001040E955DD8A47E
:101110009EEF88F0010137310C01D8B00D85D8A0C1
:101120000D950101372B020E375D0001D8A49BEF0E
:1011300088F00101376B00010C010D870001050EDD
:10114000955DD8A4B8EF88F0010137310C01D8B013
:101150000D85D8A00D950101372B020E375D0001DA
:10116000D8A4B5EF88F00101376B00010C010D87A1
:101170000001889381D61200D89688A3D886D8B665
:1011800023EF89F0470EDE6E240EDE6E010EDE6E5A
:1011900034EC9CF0DB0EDE6E3B0EDE6E090EDE6E76
:1011A00034EC9CF0DF0EDE6E5D0EDE6E090EDE6E40
:1011B00034EC9CF0E30EDE6E3A0EDE6E050EDE6E53
:1011C00034EC9CF0DD0EDE6E580EDE6E050EDE6E2B
:1011D00034EC9CF04B0E3AEC01F00101356F3553C5
:1011E0000001D8A401EF89F00C0EDE6E490EDE6E10
:1011F000090EDE6E34EC9CF0C80E51EC01F020EFCD
:1012000089F0010E0101355D0001D8A415EF89F0C8
:101210000A0EDE6E490EDE6E090EDE6E34EC9CF0B8
:10122000C80E51EC01F020EF89F00C0EDE6E490E75
:10123000DE6E090EDE6E34EC9CF0C80E51EC01F04F
:10124000C80E51EC01F0010135510C010DB9010836
:101250000001D8B45EEF89F0010135530001D8A434
:101260003FEF89F00C0EDE6E490EDE6E090EDE6E6B
:1012700034EC9CF0C80E51EC01F05EEF89F0010EE9
:101280000101355D0001D8A453EF89F00A0EDE6E2E
:10129000490EDE6E090EDE6E34EC9CF0C80E51EC89
:1012A00001F05EEF89F00C0EDE6E490EDE6E090E67
:1012B000DE6E34EC9CF0C80E51EC01F0BFEC84F013
:1012C000010E955DD8A478EF89F0AA6A4B0EA96E3D
:1012D0000101355143EC01F0050E51EC01F0D896B7
:1012E000000188B3D886D8B678EF89F065EF31F081
:1012F000040E955DD8A48FEF89F0010135310C0102
:10130000D8B00D89D8A00D990101352B020E355D9D
:101310000001D8A48EEF89F00101356B0001050EA4
:10132000955DD8A4A6EF89F0010135310C01D8B044
:101330000D89D8A00D990101352B020E355D0001F4
:10134000D8A4A5EF89F00101356B0001889314D76B
:101350001200D89688A3D886D8B617EF8AF0030E65
:10136000DE6E340EDE6EDE6A34EC9CF0290EDE6E2C
:10137000280EDE6E030EDE6E34EC9CF0DB0EDE6EAD
:10138000310EDE6E0A0EDE6E34EC9CF0DF0EDE6E89
:10139000680EDE6E0A0EDE6E34EC9CF0E30EDE6E3E
:1013A0003A0EDE6E070EDE6E34EC9CF0DD0EDE6E65
:1013B000580EDE6E070EDE6E34EC9CF04A0E3AECF0
:1013C00001F00101426F42530001D8A4F5EF89F00A
:1013D0005D0EDE6E3C0EDE6E0A0EDE6E34EC9CF0B0
:1013E000C80E51EC01F014EF8AF0010E0101425DCC
:1013F0000001D8A409EF8AF0610EDE6E3C0EDE6EAD
:101400000A0EDE6E34EC9CF0C80E51EC01F014EFC5
:101410008AF05D0EDE6E3C0EDE6E0A0EDE6E34EC81
:101420009CF0C80E51EC01F0C80E51EC01F0010126
:1014300042510C010DBB01080001D8B452EF8AF0F3
:10144000010142530001D8A433EF8AF05D0EDE6E35
:101450003C0EDE6E0A0EDE6E34EC9CF0C80E51ECD3
:1014600001F052EF8AF0010E0101425D0001D8A4A3
:1014700047EF8AF0610EDE6E3C0EDE6E0A0EDE6E07
:1014800034EC9CF0C80E51EC01F052EF8AF05D0E86
:10149000DE6E3C0EDE6E0A0EDE6E34EC9CF0C80E84
:1014A00051EC01F0BFEC84F0010E955DD8A46CEF17
:1014B0008AF0AA6A4A0EA96E0101425143EC01F07A
:1014C000050E51EC01F0D896000188B3D886D8B645
:1014D0006CEF8AF065EF31F0040E955DD8A483EFD0
:1014E0008AF0010142310C01D8B00D8BD8A00D9BC0
:1014F0000101422B020E425D0001D8A482EF8AF066
:101500000101426B0001050E955DD8A49AEF8AF0A7
:10151000010142310C01D8B00D8BD8A00D9B010107
:10152000422B020E425D0001D8A499EF8AF001011E
:10153000426B000188930DD71200D89688A3D886F5
:10154000D8B616EF8BF0E90EDE6E1C0EDE6EDE6A8C
:1015500034EC9CF0D70EDE6E860EDE6E0A0EDE6E6A
:1015600034EC9CF03F0EDE6E890EDE6E0C0EDE6EED
:1015700034EC9CF0D90EDE6E860EDE6E0E0EDE6E44
:1015800034EC9CF0DB0EDE6E1B0EDE6E070EDE6EA4
:1015900034EC9CF0DF0EDE6E740EDE6E070EDE6E37
:1015A00034EC9CF0E30EDE6E3A0EDE6E040EDE6E60
:1015B00034EC9CF0DD0EDE6E580EDE6E040EDE6E38
:1015C00034EC9CF0460E3AEC01F001012F6F0C0157
:1015D0001A6B2FC119FC19CCDEFF1ACCDEFFDE6AB4
:1015E000010EDE6E0A0EDE6E000127EC76F00A0EAA
:1015F00051EC01F04C0E3AEC01F001012E6F2E532C
:101600000001D8A40EEF8BF0E50EDE6E2F0EDE6E1D
:10161000060EDE6E34EC9CF016EF8BF0E70EDE6EFD
:101620002F0EDE6E060EDE6E34EC9CF001012F51A3
:101630000C01185D0001D8B431EF8BF00C011A6B6E
:101640002FC119FC19CCDEFF1ACCDEFFDE6A010EB9
:10165000DE6E0A0EDE6E000127EC76F00A0E51EC0B
:1016600001F00C011B5101012E5D0001D8B457EFB0
:101670008BF001012E530001D8A44CEF8BF0E50E46
:10168000DE6E2F0EDE6E060EDE6E34EC9CF0640E07
:1016900051EC01F057EF8BF0E70EDE6E2F0EDE6E91
:1016A000060EDE6E34EC9CF0640E51EC01F0D89620
:1016B0000C010DADD8860001D8B666EF8BF0010E97
:1016C000246E2C0E52EC01F00C010D9D0001BFECBC
:1016D00084F0010E955DD8A48AEF8BF0AA6A460EBD
:1016E000A96E01012F5143EC01F0050E51EC01F000
:1016F000AA6A4C0EA96E2E5143EC01F0050E51EC76
:1017000001F0D896000188B3D886D8B68AEF8BF05E
:1017100065EF31F0020E955DD8A49DEF8BF02FC1DF
:1017200018FC01012F2B2F290001D8A49AEF8BF070
:1017300001012F6B00010C010D8D0001030E955D61
:10174000D8A4B2EF8BF02FC118FC01012F53000178
:10175000D8A4ADEF8BF001012F69000101012F0723
:101760000C010D8D0001040E955DD8A4C7EF8BF020
:101770002EC11BFC01012E2B020E2E5D0001D8A4F0
:10178000C4EF8BF001012E6B00010C010D8D0001E7
:10179000050E955DD8A4DCEF8BF02EC11BFC01017A
:1017A0002E2B020E2E5D0001D8A4D9EF8BF0010183
:1017B0002E6B00010C010D8D00018893BED6120026
:1017C000D89688A3D886D8B651EF8CF0EB0EDE6E93
:1017D0002A0EDE6EDE6A34EC9CF0D70EDE6E860ECC
:1017E000DE6E0A0EDE6E34EC9CF0D90EDE6E860ED6
:1017F000DE6E0E0EDE6E34EC9CF0DB0EDE6E250E21
:10180000DE6E070EDE6E34EC9CF0DF0EDE6E6A0ECE
:10181000DE6E070EDE6E34EC9CF0E30EDE6E3A0EEA
:10182000DE6E040EDE6E34EC9CF0DD0EDE6E580EC5
:10183000DE6E040EDE6E34EC9CF0470E3AEC01F0E6
:101840000101306F0C011E6B30C11DFC1DCCDEFF91
:101850001ECCDEFFDE6A010EDE6E0A0EDE6E0001B9
:1018600027EC76F00A0E51EC01F0480E3AEC01F04C
:101870000101316F31530001D8A449EF8CF0F10E12
:10188000DE6E390EDE6E060EDE6E34EC9CF051EF2D
:101890008CF0EF0EDE6E390EDE6E060EDE6E34EC70
:1018A0009CF0010130510C011C5D0001D8B46CEFBB
:1018B0008CF00C011E6B30C11DFC1DCCDEFF1ECC5C
:1018C000DEFFDE6A010EDE6E0A0EDE6E000127EC20
:1018D00076F00A0E51EC01F00C011F510101315D4F
:1018E0000001D8B492EF8CF0010131530001D8A46B
:1018F00087EF8CF0F10EDE6E390EDE6E060EDE6EB8
:1019000034EC9CF0640E51EC01F092EF8CF0EF0E91
:10191000DE6E390EDE6E060EDE6E34EC9CF0640E6A
:1019200051EC01F0D8960C010DAFD8860001D8B665
:10193000A1EF8CF0010E246E2C0E52EC01F00C0184
:101940000D9F0001BFEC84F0010E955DD8A4D7EF88
:101950008CF0AA6A470EA96E0101305143EC01F0E8
:10196000050E51EC01F0AA6A480EA96E315143EC04
:1019700001F0050E51EC01F0010E315D0001D8A41B
:10198000C7EF8CF0CA6B30C1C9F0CEEF8CF001010B
:1019900030513C0DF3CFC9F0F4CFCAF00001D89616
:1019A00088B3D886D8B6D7EF8CF065EF31F0020E49
:1019B000955DD8A4EBEF8CF030C11CFC01013029FF
:1019C0000001D8A4E6EF8CF00101306B00010101A9
:1019D000302B0C010D8F0001030E955DD8A4FFEF95
:1019E0008CF030C11CFC0101300730530001D8A439
:1019F000FCEF8CF00101306900010C010D8F00013A
:101A0000040E955DD8A414EF8DF031C11FFC0101C7
:101A1000312B020E315D0001D8A411EF8DF00101D0
:101A2000316B00010C010D8F0001050E955DD8A4EE
:101A300029EF8DF031C11FFC0101312B020E315D08
:101A40000001D8A426EF8DF00101316B00010C01DB
:101A50000D8F00018893B4D612000C01206900019B
:101A6000B353D8A437EF8DF0B2510C01205DD8A448
:101A7000010E3B6E0001B553D8A442EF8DF0B45176
:101A80000C01205DD8A4010E3B100001D8B47EEFFC
:101A90008EF0B551B411D8A401EF8EF0B2C0DEFFC4
:101AA000B3C0DEFFDE6A010EDE6E0A0EDE6E27ECCC
:101AB00076F0B351B211D8A4AEEF8DF0040EDE6E05
:101AC00017ECC2F0820EDE6E33ECC2F00C01216B1B
:101AD0000001180E0C01215D0001D8B078EF8DF0E7
:101AE000DE6AA3ECC2F00C01212B0001D8A4F0D7D0
:101AF000050EDE6E17ECC2F0890EDE6E33ECC2F01E
:101B00000C01216B0001080E0C01215D0001D8B011
:101B100092EF8DF0DE6AA3ECC2F00C01212B0001E4
:101B2000D8A4F0D7030EDE6E17ECC2F0890EDE6E7D
:101B300033ECC2F00C01216B0001080E0C01215D99
:101B40000001D8B0ACEF8DF0DE6AA3ECC2F00C015E
:101B5000212B0001D8A4F0D7FCEF8DF0040EDE6E2F
:101B600017ECC2F0820EDE6E33ECC2F00C01216B7A
:101B70000001180E0C01215D0001D8B0C8EF8DF0F6
:101B8000DE68A3ECC2F00C01212B0001D8A4F0D731
:101B9000050EDE6E17ECC2F0890EDE6E33ECC2F07D
:101BA0000C01216B0001080E0C01215D0001D8B071
:101BB000E2EF8DF0DE68A3ECC2F00C01212B0001F6
:101BC000D8A4F0D7030EDE6E17ECC2F0890EDE6EDD
:101BD00033ECC2F00C01216B0001080E0C01215DF9
:101BE0000001D8B0FCEF8DF0DE68A3ECC2F00C0170
:101BF000212B0001D8A4F0D70A0E51EC01F07EEFA2
